:100000000C94B03B0C94DF3B0C94DF3B0C94DF3B37
:100010000C94DF3B0C94DF3B0C94DF3B0C94DF3BF8
:100020000C94DF3B0C94DF3B0C94DF3B0C94DF3BE8
:100030000C94DF3B0C947D5F0C94DF3B0C94DF3B16
:100040000C94DF3B0C94DF3B0C94DF3B0C94DF3BC8
:100050000C94DF3B0C9489600C94DF3B0C94DF3BE9
:100060000C94DF3B0C94F1CB0C94DF3B0C941DCC37
:100070000C94DF3B0C94899A0C94DF3B0C94DF3B8F
:100080000C94D75B0C94DF3B0C94DF3B0C94DF3B70
:100090000C94DF3B0C94DF3B0C94DF3B0C94DF3B78
:1000A0000C94DF3B0C94DF3B0C94DF3B0C94DF3B68
:1000B0000C94DF3B0C94DF3B0C94DF3B0C94DF3B58
:1000C0000C94DF3B0C94DF3B0C94DF3B0C94DF3B48
:1000D0000C94DF3B0C94DF3B0C94DF3B0C94DF3B38
:1000E0000C94DF3BF1562657295710573357E357E7
:1000F000E35710578657E3578A578F57A457A95786
:100100006D5772577C5710578157E357F65668570B
:10011000AE57D657E357B357546865205265706C95
:10012000696361743072007A7A7A7979797978784A
:10013000787878777777777676767675757575755A
:100140007474747474737373737272727272717183
:1001500071717170707070706F6F6F6F6F6E6E6EA7
:100160006E6E6D6D6D6D6D6D6C6C6C6C6C6B6B6BC8
:100170006B6B6A6A6A6A6A6A6969696969696868E7
:100180006868686767676767676666666666666504
:10019000656565656564646464646464636363631E
:1001A0006363626262626262626161616161616035
:1001B0006060606060605F5F5F5F5F5F5F5E5E5E4C
:1001C0005E5E5E5E5D5D5D5D5D5D5D5C5C5C5C5C60
:1001D0005C5C5C5B5B5B5B5B5B5B5A5A5A5A5A5A72
:1001E0005A5A595959595959595958585858585883
:1001F0005858575757575757575756565656565693
:1002000056565555555555555555555454545454A1
:1002100054545454535353535353535353525252AD
:1002200052525252525251515151515151515151B8
:10023000505050505050505050504F4F4F4F4F4FC4
:100240004F4F4F4F4E4E4E4E4E4E4E4E4E4E4D4DCC
:100250004D4D4D4D4D4D4D4D4C4C4C4C4C4C4C4CD6
:100260004C4C4C4B4B4B4B4B4B4B4B4B4B4B4A4ADD
:100270004A4A4A4A4A4A4A4A4A4A494949494949E4
:1002800049494949494948484848484848484848E8
:1002900048484747474747474747474747474646EE
:1002A00046464646464646464646464545454545F3
:1002B00045454545454545454444444444444444F6
:1002C00044444444444343434343434343434343F9
:1002D00043434342424242424242424242424242FB
:1002E00042424141414141414141414141414141FC
:1002F00040404040404040404040404040404040FE
:100300003F3F3F3F3F3F3F3F3F3F3F3F3F3F3F3FFD
:100310003E3E3E3E3E3E3E3E3E3E3E3E3E3E3E3EFD
:100320003D3D3D3D3D3D3D3D3D3D3D3D3D3D3D3DFD
:100330003D3C3C3C3C3C3C3C3C3C3C3C3C3C3C3CFC
:100340003C3C3B3B3B3B3B3B3B3B3B3B3B3B3B3BFB
:100350003B3B3B3B3A3A3A3A3A3A3A3A3A3A3A3AF9
:100360003A3A3A3A3A3A39393939393939393939F7
:1003700039393939393939393939383838383838F3
:1003800038383838383838383838383838383737EF
:1003900037373737373737373737373737373737ED
:1003A00037373636363636363636363636363636EB
:1003B00036363636363636363535353535353535E5
:1003C00035353535353535353535353535353434DF
:1003D00034343434343434343434343434343434DD
:1003E00034343434343333333333333333333333D8
:1003F00033333333333333333333333333323232D0
:1004000032323232323232323232323232323232CC
:1004100032323232323231313131313131313131C6
:1004200031313131313131313131313131313131BC
:1004300030303030303030303030303030303030BC
:1004400030303030303030303030302F2F2F2F2FB1
:100450002F2F2F2F2F2F2F2F2F2F2F2F2F2F2F2FAC
:100460002F2F2F2F2F2F2F2F2E2E2E2E2E2E2E2EA4
:100470002E2E2E2E2E2E2E2E2E2E2E2E2E2E2E2E9C
:100480002E2E2E2E2E2D2D2D2D2D2D2D2D2D2D2D97
:100490002D2D2D2D2D2D2D2D2D2D2D2D2D2D2D2D8C
:1004A0002D2D2D2D2C2C2C2C2C2C2C2C2C2C2C2C88
:1004B0002C2C2C2C2C2C2C2C2C2C2C2C2C2C2C2C7C
:1004C0002C2C2C2C2B2B2B2B2B2B2B2B2B2B2B2B78
:1004D0002B2B2B2B2B2B2B2B2B2B2B2B2B2B2B2B6C
:1004E0002B2B2B2B2B2B2A2A2A2A2A2A2A2A2A2A66
:1004F0002A2A2A2A2A2A2A2A2A2A2A2A2A2A2A2A5C
:100500002A2A2A2A2A2A2A2A2A2A29292929292951
:10051000292929292929292929292929292929294B
:10052000292929292929292929292929292929283C
:10053000282828282828282828282828282828283B
:10054000282828282828282828282828282828282B
:100550002828282828282727272727272727272725
:10056000272727272727272727272727272727271B
:10057000272727272727272727272727272727260C
:10058000262626262626262626262626262626260B
:1005900026262626262626262626262626262626FB
:1005A00026262626262626262626252525252525F1
:1005B00025252525252525252525252525252525EB
:1005C00025252525252525252525252525252525DB
:1005D00025252525252525252424242424242424D3
:1005E00024242424242424242424242424242424CB
:1005F00024242424242424242424242424242424BB
:1006000024242424242424242323232323232323B2
:1006100023232323232323232323232323232323AA
:10062000232323232323232323232323232323239A
:10063000232323232323232323232322222222228F
:10064000222222222222222222222222222222228A
:10065000222222222222222222222222222222227A
:10066000222222222222222222222222222222226A
:100670002221212121212121212121212121212169
:10068000212121212121212121212121212121215A
:10069000212121212121212121212121212121214A
:1006A000212121212121212121212120202020203F
:1006B000202020202020202020202020202020203A
:1006C000202020202020202020202020202020202A
:1006D000202020202020202020202020202020201A
:1006E00020202020202020201F1F1F1F1F1F1F1F12
:1006F0001F1F1F1F1F1F1F1F1F1F1F1F1F1F1F1F0A
:100700001F1F1F1F1F1F1F1F1F1F1F1F1F1F1F1FF9
:100710001F1F1F1F1F1F1F1F1F1F1F1F1F1F1F1FE9
:100720001F1F1F1F1F1F1F1E0000000000000000D2
:1007300000000000000000000000000000000000B9
:1007400000000000000000000000000000000000A9
:100750000000000000000000000000000000000099
:100760000000000000000000127A5F76E4729B6FC8
:10077000826C9369CC662964A861465F025DD85A91
:10078000C758CE56EB541D536151B84F204E984C6C
:100790001F4BB44957480647C14588445943354221
:1007A0001B410940013F013E093D193C303B4D3A98
:1007B00072399D38CE37053741368335CA34153402
:1007C0006633BB3215327231D4303A30A32F102F3A
:1007D000812EF52D6C2DE62C642CE42B672BED2A55
:1007E000762A012A8E291E29B1284528DC2775275B
:1007F0001027AD264C26ED258F253425DA248224BA
:100800002B24D62383233123E12292224422F82170
:10081000AD2163211B21D3208D2048200520C21F3C
:10082000811F401F011FC21E851E481E0C1ED21DA7
:10083000981D5F1D271DEF1CB91C831C4E1C1A1C24
:10084000E71BB41B821B511B201BF11AC11A931A00
:10085000651A371A0B1ADF19B31988195E1934197A
:100860000A19E118B91891186A1843181D18F717D2
:10087000D217AD178817641740171D17FA16D81628
:10088000B61694167316521632161216F215D315A2
:10089000B4159515771558153B151D150015E4145D
:1008A000C714AB148F14741458143D142314081473
:1008B000EE13D413BB13A11388136F1356133E13F7
:1008C00026130E13F612DF12C812B1129A128312F7
:1008D0006D12571241122B1216120012EB11D61183
:1008E000C111AD119911841170115C1149113511AB
:1008F00022110F11FC10E910D610C410B2109F1075
:100900008D107B106A1058104710351024101310EA
:100910000210F20FE10FD10FC00FB00FA00F900F18
:10092000800F710F610F520F420F330F240F150FFD
:10093000060FF70EE90EDA0ECC0EBE0EAF0EA10EAC
:10094000930E850E780E6A0E5C0E4F0E420E340E1C
:10095000270E1A0E0D0E000EF30DE70DDA0DCE0D5B
:10096000C10DB50DA90D9C0D900D840D780D6C0D6C
:10097000610D550D490D3E0D320D270D1C0D100D4D
:10098000050DFA0CEF0CE40CD90CCF0CC40CB90C0F
:10099000AF0CA40C9A0C8F0C850C7B0C710C670CA3
:1009A0005D0C530C490C3F0C350C2B0C220C180C15
:1009B0000E0C050CFB0BF20BE90BE00BD60BCD0B71
:1009C000C40BBB0BB20BA90BA00B970B8F0B860BA9
:1009D0007D0B750B6C0B630B5B0B530B4A0B420BC4
:1009E0003A0B310B290B210B190B110B090B010BC6
:1009F000F90AF10AE90AE20ADA0AD20ACA0AC30AB9
:100A0000BB0AB40AAC0AA50A9D0A960A8F0A870A8D
:100A1000800A790A720A6B0A640A5D0A560A4F0A4A
:100A2000480A410A3A0A330A2C0A250A1F0A180AF8
:100A3000110A0B0A040AFE09F709F109EA09E40997
:100A4000DD09D709D109CA09C409BE09B809B10924
:100A5000AB09A5099F09990993098D09870981099E
:100A60007B0975096F096A0964095E095809530908
:100A70004D09470942093C09360931092B09260964
:100A800020091B09160910090B0905090009FB08B3
:100A9000F608F008EB08E608E108DC08D608D108FB
:100AA000CC08C708C208BD08B808B308AE08A90832
:100AB000A408A0089B08960891088C08870883085A
:100AC0007E087908750870086B08670862085D0879
:100AD0005908540850084B08470842083E0839088E
:100AE000350830082C08280823081F081B0816089A
:100AF00012080E080A0805080108FD07F907F5079E
:100B0000F107EC07E807E407E007DC07D807D4079C
:100B1000D007CC07C807C407C007BC07B807B4078D
:100B2000B107AD07A907A507A1079D079A07960773
:100B300092078E078B07870783077F077C07780755
:100B4000740771076D076A07660762075F075B072F
:100B50005807540751074D074A07460743073F0701
:100B60003C073807350732072E072B0728072407CD
:100B700021071D071A071707140710070D070A0793
:100B8000070703070007FD06FA06F706F306F00657
:100B9000ED06EA06E706E406E106DD06DA06D70614
:100BA000D406D106CE06CB06C806C506C206BF06C9
:100BB000BC06B906B606B306B006AD06AA06A80678
:100BC000A506A2069F069C0699069606940691061F
:100BD0008E068B0688068506830680067D067A06C5
:100BE0007806750672066F066D066A066706650664
:100BF00062065F065D065A065706550652065006FF
:100C00004D064A0648064506430640063D063B0695
:100C100038063606330631062E062C062906270628
:100C2000240622061F061D061B06180616061306B6
:100C300011060E060C060A06070605060206000641
:100C4000FE05FB05F905F705F405F205F005ED05D0
:100C5000EB05E905E705E405E205E005DE05DB0552
:100C6000D905D705D505D205D005CE05CC05C905D2
:100C7000C705C505C305C105BF05BC05BA05B8054F
:100C8000B605B405B205B005AD05AB05A905A705C8
:100C9000A505A305A1059F059D059B05990597053C
:100CA0009505930591058E058C058A0588058605B1
:100CB0008405820580057E057C057B057905770521
:100CC0007505730571056F056D056B05690567058C
:100CD00065056305610560055E055C055A055805F7
:100CE00056055405520551054F054D054B0549055F
:100CF000470546054405420540053E053C053B05C4
:100D00003905370535053405320530052E052D0525
:100D10002B052905270526052405220520051F0585
:100D20001D051B05190518051605140513051105E4
:100D30000F050E050C050A0509050705050504053F
:100D400002050005FF04FD04FC04FA04F804F7049E
:100D5000F504F304F204F004EF04ED04EB04EA04F8
:100D6000E804E704E504E404E204E004DF04DD044D
:100D7000DC04DA04D904D704D604D404D304D1049F
:100D8000D004CE04CD04CB04C904C804C604C504F1
:100D9000C404C204C104BF04BE04BC04BB04B9043F
:100DA000B804B604B504B304B204B004AF04AE048E
:100DB000AC04AB04A904A804A604A504A404A204DA
:100DC000A1049F049E049D049B049A049804970424
:100DD000960494049304920490048F048E048C046B
:100DE0008B048904880487048504840483048104B3
:100DF00080047F047D047C047B04790478047704F8
:100E0000760474047304720470046F046E046D0439
:100E10006B046A046904670466046504640462047C
:100E2000610460045F045D045C045B045A045804BC
:100E300057045604550453045204510450044F04FB
:100E40004D044C044B044A0448044704460445043A
:100E500044044304410440043F043E043D043B0475
:100E60003A043904380437043604340433043204B1
:100E7000310430042F042E042C042B042A042904EA
:100E80002804270426042404230422042104200423
:100E90001F041E041D041C041A041904180417045A
:100EA00016041504140413041204110410040E048F
:100EB0000D040C040B040A040904080407040604C6
:100EC000050404040304020401040004FE03FD03FA
:100ED000FC03FB03FA03F903F803F703F603F50336
:100EE000F403F303F203F103F003EF03EE03ED0366
:100EF000EC03EB03EA03E903E803E703E603E50396
:100F0000E403E303E203E103E003DF03DE03DD03C5
:100F1000DC03DB03DA03D903D803D703D603D503F5
:100F2000D403D303D203D203D103D003CF03CE0320
:100F3000CD03CC03CB03CA03C903C803C703C6034D
:100F4000C503C403C303C203C203C103C003BF0379
:100F5000BE03BD03BC03BB03BA03B903B803B703A5
:100F6000B703B603B503B403B303B203B103B003CD
:100F7000AF03AF03AE03AD03AC03AB03AA03A903F6
:100F8000A803A703A703A603A503A403A303A2031F
:100F9000A103A103A0039F039E039D039C039B0346
:100FA0009B039A039903980397039603950395036C
:100FB0009403930392039103900390038F038E0392
:100FC0008D038C038B038B038A03890388038703B8
:100FD00087038603850384038303820382038103DB
:100FE00080037F037E037E037D037C037B037A0300
:100FF0007A03790378037703770376037503740321
:101000007303730372037103700370036F036E0342
:101010006D036C036C036B036A0369036903680364
:101020006703660366036503640363036303620384
:101030006103600360035F035E035D035D035C03A4
:101040005B035A035A0359035803570357035603C4
:1010500055035503540353035203520351035003E2
:101060004F034F034E034D034D034C034B034A0301
:101070004A0349034803480347034603460345031D
:1010800044034303430342034103410340033F033B
:101090003F033E033D033D033C033B033A033A0356
:1010A0003903380338033703360336033503340373
:1010B00034033303320332033103300330032F038D
:1010C0002E032E032D032C032C032B032A032A03A8
:1010D00029032803280327032603260325032503C2
:1010E00024032303230322032103210320031F03DB
:1010F0001F031E031D031D031C031C031B031A03F4
:101100001A0319031803180317031703160315030B
:101110001503140313031303120312031103100323
:1011200010030F030E030E030D030D030C030B033B
:101130000B030A030A030903080308030703070351
:101140000603050305030403040303030203020368
:10115000010301030003FF02FF02FE02FE02FD0283
:10116000FD02FC02FB02FB02FA02FA02F902F8029B
:10117000F802F702F702F602F602F502F402F402B0
:10118000F302F302F202F202F102F002F002EF02C5
:10119000EF02EE02EE02ED02ED02EC02EB02EB02D8
:1011A000EA02EA02E902E902E802E702E702E602ED
:1011B000E602E502E502E402E402E302E302E202FF
:1011C000E102E102E002E002DF02DF02DE02DE0213
:1011D000DD02DD02DC02DC02DB02DA02DA02D90225
:1011E000D902D802D802D702D702D602D602D50237
:1011F000D502D402D402D302D302D202D202D10247
:10120000D002D002CF02CF02CE02CE02CD02CD025A
:10121000CC02CC02CB02CB02CA02CA02C902C9026A
:10122000C802C802C702C702C602C602C502C5027A
:10123000C402C402C302C302C202C202C102C1028A
:10124000C002C002BF02BF02BE02BE02BD02BD029A
:10125000BC02BC02BB02BB02BA02BA02B902B902AA
:10126000B802B802B702B702B602B602B502B502BA
:10127000B502B402B402B302B302B202B202B102C6
:10128000B102B002B002AF02AF02AE02AE02AD02D6
:10129000AD02AC02AC02AC02AB02AB02AA02AA02E3
:1012A000A902A902A802A802A702A702A602A602F2
:1012B000A602A502A502A402A402A302A302A202FE
:1012C000A202A102A102A002A002A0029F029F020C
:1012D0009E029E029D029D029C029C029C029B0219
:1012E0009B029A029A029902990298029802980225
:1012F0009702970296029602950295029502940231
:10130000940293029302920292029102910291023C
:10131000900290028F028F028E028E028E028D0248
:101320008D028C028C028B028B028B028A028A0253
:10133000890289028902880288028702870286025E
:101340008602860285028502840284028402830268
:101350008302820282028102810281028002800273
:101360007F027F027F027E027E027D027D027D027D
:101370007C027C027B027B027B027A027A02790287
:101380007902790278027802770277027702760290
:10139000760275027502750274027402730273029A
:1013A00073027202720271027102710270027002A3
:1013B0006F026F026F026E026E026E026D026D02AC
:1013C0006C026C026C026B026B026A026A026A02B5
:1013D00069026902690268026802670267026702BD
:1013E00066026602650265026502640264026402C6
:1013F00063026302630262026202610261026102CD
:101400006002600260025F025F025E025E025E02D4
:101410005D025D025D025C025C025C025B025B02DB
:101420005A025A025A0259025902590258025802E3
:1014300058025702570256025602560255025502EA
:1014400055025402540254025302530253025202F0
:1014500052025102510251025002500250024F02F8
:101460004F024F024E024E024E024D024D024D02FD
:101470004C024C024C024B024B024B024A024A0203
:10148000490249024902480248024802470247020B
:101490004702460246024602450245024502440210
:1014A0004402440243024302430242024202420215
:1014B0004102410241024002400240023F023F021B
:1014C0003F023E023E023E023D023D023D023C0220
:1014D0003C023C023B023B023B023A023A023A0225
:1014E0003902390239023902380238023802370229
:1014F000370237023602360236023502350235022D
:101500003402340234023302330233023202320232
:101510003202310231023102310230023002300235
:101520002F022F022F022E022E022E022D022D023A
:101530002D022C022C022C022C022B022B022B023D
:101540002A022A022A022902290229022802280242
:101550002802280227022702270226022602260244
:101560002502250225022502240224022402230248
:10157000230223022202220222022202210221024B
:1015800021022002200220021F021F021F021F024E
:101590001E021E021E021D021D021D021D021C0251
:1015A0001C021C021B021B021B021B021A021A0253
:1015B0001A02190219021902180218021802180256
:1015C0001702170217021602160216021602150259
:1015D000150215021402140214021402130213025B
:1015E000130213021202120212021102110211025C
:1015F00011021002100210020F020F020F020F025E
:101600000E020E020E020D020D020D020D020C0260
:101610000C020C020C020B020B020B020A020A0261
:101620000A020A0209020902090209020802080262
:101630000802070207020702070206020602060264
:101640000602050205020502050204020402040264
:101650000302030203020302020202020202020266
:101660000102010201020102000200020002000266
:10167000FF01FF01FF01FE01FE01FE01FE01FD0170
:10168000FD01FD01FD01FC01FC01FC01FC01FB0170
:10169000FB01FB01FB01FA01FA01FA01FA01F90170
:1016A000F901F901F901F801F801F801F801F70170
:1016B000F701F701F701F601F601F601F601F50170
:1016C000F501F501F501F401F401F401F401F30170
:1016D000F301F301F301F201F201F201F201F10170
:1016E000F101F101F101F001F001F001F001EF0170
:1016F000EF01EF01EF01EE01EE01EE01EE01ED0170
:10170000ED01ED01ED01EC01EC01EC01EC01EB016F
:10171000EB01EB01EB01EA01EA01EA01EA01E9016F
:10172000E901E901E901E901E801E801E801E8016D
:10173000E701E701E701E701E601E601E601E6016D
:10174000E501E501E501E501E401E401E401E4016D
:10175000E401E301E301E301E301E201E201E2016B
:10176000E201E101E101E101E101E101E001E0016A
:10177000E001E001DF01DF01DF01DF01DE01DE0169
:10178000DE01DE01DE01DD01DD01DD01DD01DC0167
:10179000DC01DC01DC01DC01DB01DB01DB01DB0165
:1017A000DA01DA01DA01DA01D901D901D901D90165
:1017B000D901D801D801D801D801D701D701D70163
:1017C000D701D701D601D601D601D601D501D50161
:1017D000D501D501D501D401D401D401D401D4015E
:1017E000D301D301D301D301D201D201D201D2015D
:1017F000D201D101D101D101D101D001D001D0015B
:10180000D001D001CF01CF01CF01CF01CF01CE0157
:10181000CE01CE01CE01CD01CD01CD01CD01CD0155
:10182000CC01CC01CC01CC01CC01CB01CB01CB0153
:10183000CB01CB01CA01CA01CA01CA01C901C90150
:10184000C901C901C901C801C801C801C801C8014D
:10185000C701C701C701C701C701C601C601C6014B
:10186000C601C601C501C501C501C501C401C40148
:10187000C401C401C401C301C301C301C301C30145
:10188000C201C201C201C201C201C101C101C10143
:10189000C101C101C001C001C001C001C001BF013F
:1018A000BF01BF01BF01BF01BE01BE01BE01BE013C
:1018B000BE01BD01BD01BD01BD01BD01BC01BC0139
:1018C000BC01BC01BC01BB01BB01BB01BB01BB0135
:1018D000BA01BA01BA01BA01BA01BA01B901B90132
:1018E000B901B901B901B801B801B801B801B8012D
:1018F000B701B701B701B701B701B601B601B6012B
:10190000B601B601B501B501B501B501B501B40126
:10191000B401B401B401B401B401B301B301B30122
:10192000B301B301B201B201B201B201B201B1011E
:10193000B101B101B101B101B101B001B001B0011A
:10194000B001B001AF01AF01AF01AF01AF01AE0116
:10195000AE01AE01AE01AE01AE01AD01AD01AD0112
:10196000AD01AD01AC01AC01AC01AC01AC01AC010D
:10197000AB01AB01AB01AB01AB01AA01AA01AA010A
:10198000AA01AA01AA01A901A901A901A901A90104
:10199000A801A801A801A801A801A801A701A70101
:1019A000A701A701A701A601A601A601A601A601FC
:1019B000A601A501A501A501A501A501A501A401F7
:1019C000A401A401A401A401A301A301A301A301F3
:1019D000A301A301A201A201A201A201A201A201ED
:1019E000A101A101A101A101A101A001A001A001EA
:1019F000A001A001A0019F019F019F019F019F01E4
:101A00009F019E019E019E019E019E019E019D01DE
:101A10009D019D019D019D019D019C019C019C01D9
:101A20009C019C019C019B019B019B019B019B01D3
:101A30009B019A019A019A019A019A019A019901CE
:101A400099019901990199019801980198019801CA
:101A500098019801970197019701970197019701C4
:101A600097019601960196019601960196019501BE
:101A700095019501950195019501940194019401B9
:101A800094019401940193019301930193019301B3
:101A900093019201920192019201920192019101AE
:101AA00091019101910191019101900190019001A9
:101AB00090019001900190018F018F018F018F01A2
:101AC0008F018F018E018E018E018E018E018E019C
:101AD0008D018D018D018D018D018D018D018C0197
:101AE0008C018C018C018C018C018B018B018B0191
:101AF0008B018B018B018A018A018A018A018A018B
:101B00008A018A0189018901890189018901890183
:101B1000880188018801880188018801880187017E
:101B20008701870187018701870186018601860178
:101B30008601860186018601850185018501850171
:101B4000850185018501840184018401840184016A
:101B50008401830183018301830183018301830164
:101B6000820182018201820182018201820181015E
:101B70008101810181018101810180018001800158
:101B800080018001800180017F017F017F017F0151
:101B90007F017F017F017E017E017E017E017E014A
:101BA0007E017E017D017D017D017D017D017D0143
:101BB0007D017C017C017C017C017C017C017C013C
:101BC0007B017B017B017B017B017B017B017A0136
:101BD0007A017A017A017A017A017A01790179012F
:101BE0007901790179017901790178017801780128
:101BF0007801780178017801770177017701770121
:101C00007701770177017601760176017601760119
:101C10007601760175017501750175017501750112
:101C2000750174017401740174017401740174010B
:101C30007301730173017301730173017301730104
:101C400072017201720172017201720172017101FD
:101C500071017101710171017101710170017001F6
:101C60007001700170017001700170016F016F01EE
:101C70006F016F016F016F016F016E016E016E01E7
:101C80006E016E016E016E016D016D016D016D01E0
:101C90006D016D016D016D016C016C016C016C01D8
:101CA0006C016C016C016C016B016B016B016B01D0
:101CB0006B016B016B016A016A016A016A016A01C9
:101CC0006A016A016A0169016901690169016901C1
:101CD00069016901680168016801680168016801BA
:101CE00068016801670167016701670167016701B2
:101CF00067016701660166016601660166016601AA
:101D000066016601650165016501650165016501A1
:101D10006501650164016401640164016401640199
:101D20006401630163016301630163016301630192
:101D3000630162016201620162016201620162018A
:101D40006201610161016101610161016101610182
:101D5000610160016001600160016001600160017A
:101D600060015F015F015F015F015F015F015F0172
:101D70005F015F015E015E015E015E015E015E0169
:101D80005E015E015D015D015D015D015D015D0161
:101D90005D015D015C015C015C015C015C015C0159
:101DA0005C015C015B015B015B015B015B015B0151
:101DB0005B015B015B015A015A015A015A015A0148
:101DC0005A015A015A015901590159015901590140
:101DD0005901590159015801580158015801580138
:101DE000580158015801580157015701570157012F
:101DF0005701570157015701560156015601560127
:101E0000560156015601560156015501550155011D
:101E10005501550155015501550154015401540115
:101E2000540154015401540154015401530153010C
:101E30005301530153015301530153015301520103
:101E400052015201520152015201520152015101FB
:101E500051015101510151015101510151015101F2
:101E600050015001500150015001500150015001EA
:101E700050014F014F014F014F014F014F014F01E1
:101E80004F014F014E014E014E014E014E014E01D8
:101E90004E014E014E014D014D014D014D014D01CF
:101EA0004D014D014D014D014C014C014C014C01C6
:101EB0004C014C014C014C014C014B014B014B01BD
:101EC0004B014B014B014B014B014B014A014A01B4
:101ED0004A014A014A014A014A014A014A014901AB
:101EE00049014901490149014901490149014901A2
:101EF0004901480148014801480148014801480199
:101F0000480148014701470147014701470147018F
:101F10004701470147014601460146014601460186
:101F2000460146014601460146014501450145017C
:101F30004501450145014501450145014401440173
:101F40004401440144014401440144014401440169
:101F50004301430143014301430143014301430161
:101F60004301420142014201420142014201420158
:101F7000420142014201410141014101410141014E
:101F80004101410141014101410140014001400144
:101F90004001400140014001400140013F013F013B
:101FA0003F013F013F013F013F013F013F013F0131
:101FB0003E013E013E013E013E013E013E013E0129
:101FC0003E013E013D013D013D013D013D013D011F
:101FD0003D013D013D013D013C013C013C013C0115
:101FE0003C013C013C013C013C013C013B013B010B
:101FF0003B013B013B013B013B013B013B013B0101
:102000003A013A013A013A013A013A013A013A01F8
:102010003A013A01390139013901390139013901EE
:1020200039013901390139013901380138013801E3
:1020300038013801380138013801380138013701D9
:1020400037013701370137013701370137013701D0
:1020500037013601360136013601360136013601C7
:1020600036013601360136013501350135013501BC
:1020700035013501350135013501350134013401B2
:1020800034013401340134013401340134013401A8
:10209000340133013301330133013301330133019F
:1020A0003301330133013201320132013201320195
:1020B000320132013201320132013201310131018A
:1020C0003101310131013101310131013101310180
:1020D0003101300130013001300130013001300177
:1020E0003001300130012F012F012F012F012F016D
:1020F0002F012F012F012F012F012F012E012E0162
:102100002E012E012E012E012E012E012E012E0157
:102110002E012D012D012D012D012D012D012D014E
:102120002D012D012D012D012C012C012C012C0143
:102130002C012C012C012C012C012C012C012B0138
:102140002B012B012B012B012B012B012B012B012F
:102150002B012B012B012A012A012A012A012A0124
:102160002A012A012A012A012A012A012901290119
:10217000290129012901290129012901290129010F
:102180002901280128012801280128012801280106
:1021900028012801280128012801270127012701FA
:1021A00027012701270127012701270127012701EF
:1021B00026012601260126012601260126012601E7
:1021C00026012601260126012501250125012501DB
:1021D00025012501250125012501250125012401D0
:1021E00024012401240124012401240124012401C7
:1021F00024012401240123012301230123012301BC
:1022000023012301230123012301230123012201AF
:1022100022012201220122012201220122012201A6
:10222000220122012201210121012101210121019B
:10223000210121012101210121012101210120018F
:102240002001200120012001200120012001200186
:102250002001200120011F011F011F011F011F017B
:102260001F011F011F011F011F011F011F011E016F
:102270001E011E011E011E011E011E011E011E0166
:102280001E011E011E011D011D011D011D011D015B
:102290001D011D011D011D011D011D011D011C014F
:1022A0001C011C011C011C011C011C011C011C0146
:1022B0001C011C011C011C011B011B011B011B013A
:1022C0001B011B011B011B011B011B011B011B012E
:1022D0001A011A011A011A011A011A011A011A0126
:1022E0001A011A011A011A011A0119011901190119
:1022F000190119011901190119011901190119010E
:102300001901190118011801180118011801180103
:1023100018011801180118011801180117011701F7
:1023200017011701170117011701170117011701ED
:1023300017011701170116011601160116011601E2
:1023400016011601160116011601160116011601D5
:1023500015011501150115011501150115011501CD
:1023600015011501150115011501140114011401C0
:1023700014011401140114011401140114011401B5
:1023800014011401130113011301130113011301AB
:10239000130113011301130113011301130112019E
:1023A0001201120112011201120112011201120195
:1023B0001201120112011201120111011101110188
:1023C000110111011101110111011101110111017D
:1023D0001101110110011001100110011001100173
:1023E0001001100110011001100110011001100165
:1023F0000F010F010F010F010F010F010F010F015D
:102400000F010F010F010F010F010E010E010E014F
:102410000E010E010E010E010E010E010E010E0144
:102420000E010E010E010D010D010D010D010D0139
:102430000D010D010D010D010D010D010D010D012C
:102440000D010C010C010C010C010C010C010C0123
:102450000C010C010C010C010C010C010C010B0115
:102460000B010B010B010B010B010B010B010B010C
:102470000B010B010B010B010B010A010A010A01FF
:102480000A010A010A010A010A010A010A010A01F4
:102490000A010A010A0109010901090109010901E9
:1024A00009010901090109010901090109010901DC
:1024B00009010801080108010801080108010801D3
:1024C00008010801080108010801080108010801C4
:1024D00007010701070107010701070107010701BC
:1024E00007010701070107010701070106010601AE
:1024F00006010601060106010601060106010601A4
:102500000601060106010601060105010501050196
:10251000050105010501050105010501050105018B
:102520000501050105010401040104010401040180
:102530000401040104010401040104010401040173
:102540000401040103010301030103010301030169
:10255000030103010301030103010301030103015B
:102560000301020102010201020102010201020152
:102570000201020102010201020102010201020143
:10258000010101010101010101010101010101013B
:10259000010101010101010101010101010100012C
:1025A0000001000100010001000100010001000123
:1025B000000100010001000100010001FF00FF0017
:1025C000FF00FF00FF00FF00FF00FF00FF00FF0013
:1025D000FF00FF00FF00FF00FF00FF00FE00FE0005
:1025E000FE00FE00FE00FE00FE00FE00FE00FE00FB
:1025F000FE00FE00FE00FE00FE00FD00FD00FD00EE
:10260000FD00FD00FD00FD00FD00FD00FD00FD00E2
:10261000FD00FD00FD00FD00FD00FC00FC00FC00D5
:10262000FC00FC00FC00FC00FC00FC00FC00FC00CA
:10263000FC00FC00FC00FC00FC00FB00FB00FB00BD
:10264000FB00FB00FB00FB00FB00FB00FB00FB00B2
:10265000FB00FB00FB00FB00FB00FA00FA00FA00A5
:10266000FA00FA00FA00FA00FA00FA00FA00FA009A
:10267000FA00FA00FA00FA00FA00F900F900F9008D
:10268000F900F900F900F900F900F900F900F90082
:10269000F900F900F900F900F900F800F800F80075
:1026A000F800F800F800F800F800F800F800F8006A
:1026B000F800F800F800F800F800F700F700F7005D
:1026C000F700F700F700F700F700F700F700F70052
:1026D000F700F700F700F700F700F600F600F60045
:1026E000F600F600F600F600F600F600F600F6003A
:1026F000F600F600F600F600F600F600F500F5002C
:10270000F500F500F500F500F500F500F500F50021
:10271000F500F500F500F500F500F500F400F40013
:10272000F400F400F400F400F400F400F400F40009
:10273000F400F400F400F400F400F400F400F300FA
:10274000F300F300F300F300F300F300F300F300F1
:10275000F300F300F300F300F300F300F300F300E1
:10276000F200F200F200F200F200F200F200F200D9
:10277000F200F200F200F200F200F200F200F200C9
:10278000F200F100F100F100F100F100F100F100C0
:10279000F100F100F100F100F100F100F100F100B1
:1027A000F100F100F100F000F000F000F000F000A6
:1027B000F000F000F000F000F000F000F000F00099
:1027C000F000F000F000F000EF00EF00EF00EF008D
:1027D000EF00EF00EF00EF00EF00EF00EF00EF0081
:1027E000EF00EF00EF00EF00EF00EE00EE00EE0074
:1027F000EE00EE00EE00EE00EE00EE00EE00EE0069
:10280000EE00EE00EE00EE00EE00EE00EE00ED0059
:10281000ED00ED00ED00ED00ED00ED00ED00ED0050
:10282000ED00ED00ED00ED00ED00ED00ED00ED0040
:10283000ED00EC00EC00EC00EC00EC00EC00EC0037
:10284000EC00EC00EC00EC00EC00EC00EC00EC0028
:10285000EC00EC00EC00EB00EB00EB00EB00EB001D
:10286000EB00EB00EB00EB00EB00EB00EB00EB0010
:10287000EB00EB00EB00EB00EB00EA00EA00EA0003
:10288000EA00EA00EA00EA00EA00EA00EA00EA00F8
:10289000EA00EA00EA00EA00EA00EA00EA00E900E9
:1028A000E900E900E900E900E900E900E900E900E0
:1028B000E900E900E900E900E900E900E900E900D0
:1028C000E900E900E800E800E800E800E800E800C6
:1028D000E800E800E800E800E800E800E800E800B8
:1028E000E800E800E800E800E700E700E700E700AC
:1028F000E700E700E700E700E700E700E700E700A0
:10290000E700E700E700E700E700E700E700E60090
:10291000E600E600E600E600E600E600E600E60087
:10292000E600E600E600E600E600E600E600E60077
:10293000E600E600E500E500E500E500E500E5006D
:10294000E500E500E500E500E500E500E500E5005F
:10295000E500E500E500E500E500E400E400E40052
:10296000E400E400E400E400E400E400E400E40047
:10297000E400E400E400E400E400E400E400E40037
:10298000E300E300E300E300E300E300E300E3002F
:10299000E300E300E300E300E300E300E300E3001F
:1029A000E300E300E300E300E200E200E200E20013
:1029B000E200E200E200E200E200E200E200E20007
:1029C000E200E200E200E200E200E200E200E100F8
:1029D000E100E100E100E100E100E100E100E100EF
:1029E000E100E100E100E100E100E100E100E100DF
:1029F000E100E100E100E000E000E000E000E000D4
:102A0000E000E000E000E000E000E000E000E000C6
:102A1000E000E000E000E000E000E000E000DF00B7
:102A2000DF00DF00DF00DF00DF00DF00DF00DF00AE
:102A3000DF00DF00DF00DF00DF00DF00DF00DF009E
:102A4000DF00DF00DF00DE00DE00DE00DE00DE0093
:102A5000DE00DE00DE00DE00DE00DE00DE00DE0086
:102A6000DE00DE00DE00DE00DE00DE00DE00DD0077
:102A7000DD00DD00DD00DD00DD00DD00DD00DD006E
:102A8000DD00DD00DD00DD00DD00DD00DD00DD005E
:102A9000DD00DD00DD00DD00DC00DC00DC00DC0052
:102AA000DC00DC00DC00DC00DC00DC00DC00DC0046
:102AB000DC00DC00DC00DC00DC00DC00DC00DC0036
:102AC000DB00DB00DB00DB00DB00DB00DB00DB002E
:102AD000DB00DB00DB00DB00DB00DB00DB00DB001E
:102AE000DB00DB00DB00DB00DB00DA00DA00DA0011
:102AF000DA00DA00DA00DA00DA00DA00DA00DA0006
:102B0000DA00DA00DA00DA00DA00DA00DA00DA00F5
:102B1000DA00DA00D900D900D900D900D900D900EB
:102B2000D900D900D900D900D900D900D900D900DD
:102B3000D900D900D900D900D900D900D900D800CE
:102B4000D800D800D800D800D800D800D800D800C5
:102B5000D800D800D800D800D800D800D800D800B5
:102B6000D800D800D800D800D800D700D700D700A8
:102B7000D700D700D700D700D700D700D700D7009D
:102B8000D700D700D700D700D700D700D700D7008D
:102B9000D700D700D700D600D600D600D600D60082
:102BA000D600D600D600D600D600D600D600D60075
:102BB000D600D600D600D600D600D600D600D60065
:102BC000D500D500D500D500D500D500D500D5005D
:102BD000D500D500D500D500D500D500D500D5004D
:102BE000D500D500D500D500D500D500D400D4003F
:102BF000D400D400D400D400D400D400D400D40035
:102C0000D400D400D400D400D400D400D400D40024
:102C1000D400D400D400D400D400D300D300D30017
:102C2000D300D300D300D300D300D300D300D3000C
:102C3000D300D300D300D300D300D300D300D300FC
:102C4000D300D300D300D200D200D200D200D200F1
:102C5000D200D200D200D200D200D200D200D200E4
:102C6000D200D200D200D200D200D200D200D200D4
:102C7000D200D200D100D100D100D100D100D100CA
:102C8000D100D100D100D100D100D100D100D100BC
:102C9000D100D100D100D100D100D100D100D100AC
:102CA000D100D000D000D000D000D000D000D000A3
:102CB000D000D000D000D000D000D000D000D00094
:102CC000D000D000D000D000D000D000D000D00084
:102CD000CF00CF00CF00CF00CF00CF00CF00CF007C
:102CE000CF00CF00CF00CF00CF00CF00CF00CF006C
:102CF000CF00CF00CF00CF00CF00CF00CF00CE005D
:102D0000CE00CE00CE00CE00CE00CE00CE00CE0053
:102D1000CE00CE00CE00CE00CE00CE00CE00CE0043
:102D2000CE00CE00CE00CE00CE00CE00CE00CD0034
:102D3000CD00CD00CD00CD00CD00CD00CD00CD002B
:102D4000CD00CD00CD00CD00CD00CD00CD00CD001B
:102D5000CD00CD00CD00CD00CD00CD00CC00CC000D
:102D6000CC00CC00CC00CC00CC00CC00CC00CC0003
:102D7000CC00CC00CC00CC00CC00CC00CC00CC00F3
:102D8000CC00CC00CC00CC00CC00CC00CC00CB00E4
:102D9000CB00CB00CB00CB00CB00CB00CB00CB00DB
:102DA000CB00CB00CB00CB00CB00CB00CB00CB00CB
:102DB000CB00CB00CB00CB00CB00CB00CB00CA00BC
:102DC000CA00CA00CA00CA00CA00CA00CA00CA00B3
:102DD000CA00CA00CA00CA00CA00CA00CA00CA00A3
:102DE000CA00CA00CA00CA00CA00CA00CA00C90094
:102DF000C900C900C900C900C900C900C900C9008B
:102E0000C900C900C900C900C900C900C900C9007A
:102E1000C900C900C900C900C900C900C900C9006A
:102E2000C800C800C800C800C800C800C800C80062
:102E3000C800C800C800C800C800C800C800C80052
:102E4000C800C800C800C800C800C800C800C80042
:102E5000C800C700C700C700C700C700C700C70039
:102E6000C700C700C700C700C700C700C700C7002A
:102E7000C700C700C700C700C700C700C700C7001A
:102E8000C700C700C600C600C600C600C600C60010
:102E9000C600C600C600C600C600C600C600C60002
:102EA000C600C600C600C600C600C600C600C600F2
:102EB000C600C600C600C600C500C500C500C500E6
:102EC000C500C500C500C500C500C500C500C500DA
:102ED000C500C500C500C500C500C500C500C500CA
:102EE000C500C500C500C500C500C500C400C400BC
:102EF000C400C400C400C400C400C400C400C400B2
:102F0000C400C400C400C400C400C400C400C400A1
:102F1000C400C400C400C400C400C400C400C40091
:102F2000C300C300C300C300C300C300C300C30089
:102F3000C300C300C300C300C300C300C300C30079
:102F4000C300C300C300C300C300C300C300C30069
:102F5000C300C300C200C200C200C200C200C2005F
:102F6000C200C200C200C200C200C200C200C20051
:102F7000C200C200C200C200C200C200C200C20041
:102F8000C200C200C200C200C100C100C100C10035
:102F9000C100C100C100C100C100C100C100C10029
:102FA000C100C100C100C100C100C100C100C10019
:102FB000C100C100C100C100C100C100C100C0000A
:102FC000C000C000C000C000C000C000C000C00001
:102FD000C000C000C000C000C000C000C000C000F1
:102FE000C000C000C000C000C000C000C000C000E1
:102FF000C000C000BF00BF00BF00BF00BF00BF00D7
:10300000BF00BF00BF00BF00BF00BF00BF00BF00C8
:10301000BF00BF00BF00BF00BF00BF00BF00BF00B8
:10302000BF00BF00BF00BF00BF00BF00BE00BE00AA
:10303000BE00BE00BE00BE00BE00BE00BE00BE00A0
:10304000BE00BE00BE00BE00BE00BE00BE00BE0090
:10305000BE00BE00BE00BE00BE00BE00BE00BE0080
:10306000BE00BE00BD00BD00BD00BD00BD00BD0076
:10307000BD00BD00BD00BD00BD00BD00BD00BD0068
:10308000BD00BD00BD00BD00BD00BD00BD00BD0058
:10309000BD00BD00BD00BD00BD00BD00BC00BC004A
:1030A000BC00BC00BC00BC00BC00BC00BC00BC0040
:1030B000BC00BC00BC00BC00BC00BC00BC00BC0030
:1030C000BC00BC00BC00BC00BC00BC00BC00BC0020
:1030D000BC00BC00BB00BB00BB00BB00BB00BB0016
:1030E000BB00BB00BB00BB00BB00BB00BB00BB0008
:1030F000BB00BB00BB00BB00BB00BB00BB00BB00F8
:10310000BB00BB00BB00BB00BB00BB00BA00BA00E9
:10311000BA00BA00BA00BA00BA00BA00BA00BA00DF
:10312000BA00BA00BA00BA00BA00BA00BA00BA00CF
:10313000BA00BA00BA00BA00BA00BA00BA00BA00BF
:10314000BA00BA00BA00B900B900B900B900B900B4
:10315000B900B900B900B900B900B900B900B900A7
:10316000B900B900B900B900B900B900B900B90097
:10317000B900B900B900B900B900B900B900B90087
:10318000B900B800B800B800B800B800B800B8007E
:10319000B800B800B800B800B800B800B800B8006F
:1031A000B800B800B800B800B800B800B800B8005F
:1031B000B800B800B800B800B800B800B700B70051
:1031C000B700B700B700B700B700B700B700B70047
:1031D000B700B700B700B700B700B700B700B70037
:1031E000B700B700B700B700B700B700B700B70027
:1031F000B700B700B700B700B600B600B600B6001B
:10320000B600B600B600B600B600B600B600B6000E
:10321000B600B600B600B600B600B600B600B600FE
:10322000B600B600B600B600B600B600B600B600EE
:10323000B600B600B500B500B500B500B500B500E4
:10324000B500B500B500B500B500B500B500B500D6
:10325000B500B500B500B500B500B500B500B500C6
:10326000B500B500B500B500B500B500B500B500B6
:10327000B500B400B400B400B400B400B400B400AD
:10328000B400B400B400B400B400B400B400B4009E
:10329000B400B400B400B400B400B400B400B4008E
:1032A000B400B400B400B400B400B400B400B4007E
:1032B000B300B300B300B300B300B300B300B30076
:1032C000B300B300B300B300B300B300B300B30066
:1032D000B300B300B300B300B300B300B300B30056
:1032E000B300B300B300B300B300B300B300B20047
:1032F000B200B200B200B200B200B200B200B2003E
:10330000B200B200B200B200B200B200B200B2002D
:10331000B200B200B200B200B200B200B200B2001D
:10332000B200B200B200B200B200B200B100B1000F
:10333000B100B100B100B100B100B100B100B10005
:10334000B100B100B100B100B100B100B100B100F5
:10335000B100B100B100B100B100B100B100B100E5
:10336000B100B100B100B100B100B100B000B000D7
:10337000B000B000B000B000B000B000B000B000CD
:10338000B000B000B000B000B000B000B000B000BD
:10339000B000B000B000B000B000B000B000B000AD
:1033A000B000B000B000B000B000B000B000AF009E
:1033B000AF00AF00AF00AF00AF00AF00AF00AF0095
:1033C000AF00AF00AF00AF00AF00AF00AF00AF0085
:1033D000AF00AF00AF00AF00AF00AF00AF00AF0075
:1033E000AF00AF00AF00AF00AF00AF00AF00AE0066
:1033F000AE00AE00AE00AE00AE00AE00AE00AE005D
:10340000AE00AE00AE00AE00AE00AE00AE00AE004C
:10341000AE00AE00AE00AE00AE00AE00AE00AE003C
:10342000AE00AE00AE00AE00AE00AE00AE00AE002C
:10343000AD00AD00AD00AD00AD00AD00AD00AD0024
:10344000AD00AD00AD00AD00AD00AD00AD00AD0014
:10345000AD00AD00AD00AD00AD00AD00AD00AD0004
:10346000AD00AD00AD00AD00AD00AD00AD00AD00F4
:10347000AD00AD00AC00AC00AC00AC00AC00AC00EA
:10348000AC00AC00AC00AC00AC00AC00AC00AC00DC
:10349000AC00AC00AC00AC00AC00AC00AC00AC00CC
:1034A000AC00AC00AC00AC00AC00AC00AC00AC00BC
:1034B000AC00AC00AC00AB00AB00AB00AB00AB00B1
:1034C000AB00AB00AB00AB00AB00AB00AB00AB00A4
:1034D000AB00AB00AB00AB00AB00AB00AB00AB0094
:1034E000AB00AB00AB00AB00AB00AB00AB00AB0084
:1034F000AB00AB00AB00AB00AB00AB00AA00AA0076
:10350000AA00AA00AA00AA00AA00AA00AA00AA006B
:10351000AA00AA00AA00AA00AA00AA00AA00AA005B
:10352000AA00AA00AA00AA00AA00AA00AA00AA004B
:10353000AA00AA00AA00AA00AA00AA00AA00AA003B
:10354000A900A900A900A900A900A900A900A90033
:10355000A900A900A900A900A900A900A900A90023
:10356000A900A900A900A900A900A900A900A90013
:10357000A900A900A900A900A900A900A900A90003
:10358000A900A900A900A800A800A800A800A800F8
:10359000A800A800A800A800A800A800A800A800EB
:1035A000A800A800A800A800A800A800A800A800DB
:1035B000A800A800A800A800A800A800A800A800CB
:1035C000A800A800A800A800A800A800A800A700BC
:1035D000A700A700A700A700A700A700A700A700B3
:1035E000A700A700A700A700A700A700A700A700A3
:1035F000A700A700A700A700A700A700A700A70093
:10360000A700A700A700A700A700A700A700A70082
:10361000A700A700A700A600A600A600A600A60077
:10362000A600A600A600A600A600A600A600A6006A
:10363000A600A600A600A600A600A600A600A6005A
:10364000A600A600A600A600A600A600A600A6004A
:10365000A600A600A600A600A600A600A600A5003B
:10366000A500A500A500A500A500A500A500A50032
:10367000A500A500A500A500A500A500A500A50022
:10368000A500A500A500A500A500A500A500A50012
:10369000A500A500A500A500A500A500A500A50002
:1036A000A500A500A500A500A400A400A400A400F6
:1036B000A400A400A400A400A400A400A400A400EA
:1036C000A400A400A400A400A400A400A400A400DA
:1036D000A400A400A400A400A400A400A400A400CA
:1036E000A400A400A400A400A400A400A400A400BA
:1036F000A400A300A300A300A300A300A300A300B1
:10370000A300A300A300A300A300A300A300A300A1
:10371000A300A300A300A300A300A300A300A30091
:10372000A300A300A300A300A300A300A300A30081
:10373000A300A300A300A300A300A300A200A20073
:10374000A200A200A200A200A200A200A200A20069
:10375000A200A200A200A200A200A200A200A20059
:10376000A200A200A200A200A200A200A200A20049
:10377000A200A200A200A200A200A200A200A20039
:10378000A200A200A200A200A100A100A100A1002D
:10379000A100A100A100A100A100A100A100A10021
:1037A000A100A100A100A100A100A100A100A10011
:1037B000A100A100A100A100A100A100A100A10001
:1037C000A100A100A100A100A100A100A100A100F1
:1037D000A100A100A100A000A000A000A000A000E6
:1037E000A000A000A000A000A000A000A000A000D9
:1037F000A000A000A000A000A000A000A000A000C9
:10380000A000A000A000A000A000A000A000A000B8
:10381000A000A000A000A000A000A000A000A000A8
:10382000A000A0009F009F009F009F009F009F009E
:103830009F009F009F009F009F009F009F009F0090
:103840009F009F009F009F009F009F009F009F0080
:103850009F009F009F009F009F009F009F009F0070
:103860009F009F009F009F009F009F009F009F0060
:103870009F009F009E009E009E009E009E009E0056
:103880009E009E009E009E009E009E009E009E0048
:103890009E009E009E009E009E009E009E009E0038
:1038A0009E009E009E009E009E009E009E009E0028
:1038B0009E009E009E009E009E009E009E009E0018
:1038C0009E009E009D009D009D009D009D009D000E
:1038D0009D009D009D009D009D009D009D009D0000
:1038E0009D009D009D009D009D009D009D009D00F0
:1038F0009D009D009D009D009D009D009D009D00E0
:103900009D009D009D009D009D009D009D009D00CF
:103910009D009D009C009C009C009C009C009C00C5
:103920009C009C009C009C009C009C009C009C00B7
:103930009C009C009C009C009C009C009C009C00A7
:103940009C009C009C009C009C009C009C009C0097
:103950009C009C009C009C009C009C009C009C0087
:103960009C009C009C009B009B009B009B009B007C
:103970009B009B009B009B009B009B009B009B006F
:103980009B009B009B009B009B009B009B009B005F
:103990009B009B009B009B009B009B009B009B004F
:1039A0009B009B009B009B009B009B009B009B003F
:1039B0009B009B009B009B009B009A009A009A0032
:1039C0009A009A009A009A009A009A009A009A0027
:1039D0009A009A009A009A009A009A009A009A0017
:1039E0009A009A009A009A009A009A009A009A0007
:1039F0009A009A009A009A009A009A009A009A00F7
:103A00009A009A009A009A009A009A009A009900E7
:103A100099009900990099009900990099009900DE
:103A200099009900990099009900990099009900CE
:103A300099009900990099009900990099009900BE
:103A400099009900990099009900990099009900AE
:103A5000990099009900990099009900990099009E
:103A60009900990098009800980098009800980094
:103A70009800980098009800980098009800980086
:103A80009800980098009800980098009800980076
:103A90009800980098009800980098009800980066
:103AA0009800980098009800980098009800980056
:103AB0009800980098009800980097009700970049
:103AC000970097009700970097009700970097003E
:103AD000970097009700970097009700970097002E
:103AE000970097009700970097009700970097001E
:103AF000970097009700970097009700970097000E
:103B000097009700970097009700970097009700FD
:103B100097009600960096009600960096009600F4
:103B200096009600960096009600960096009600E5
:103B300096009600960096009600960096009600D5
:103B400096009600960096009600960096009600C5
:103B500096009600960096009600960096009600B5
:103B600096009600960096009600950095009500A8
:103B7000950095009500950095009500950095009D
:103B8000950095009500950095009500950095008D
:103B9000950095009500950095009500950095007D
:103BA000950095009500950095009500950095006D
:103BB000950095009500950095009500950095005D
:103BC0009500950095009400940094009400940052
:103BD0009400940094009400940094009400940045
:103BE0009400940094009400940094009400940035
:103BF0009400940094009400940094009400940025
:103C00009400940094009400940094009400940014
:103C10009400940094009400940094009400940004
:103C200093009300930093009300930093009300FC
:103C300093009300930093009300930093009300EC
:103C400093009300930093009300930093009300DC
:103C500093009300930093009300930093009300CC
:103C600093009300930093009300930093009300BC
:103C700093009300930093009300930092009200AE
:103C800092009200920092009200920092009200A4
:103C90009200920092009200920092009200920094
:103CA0009200920092009200920092009200920084
:103CB0009200920092009200920092009200920074
:103CC0009200920092009200920092009200920064
:103CD0009200920092009200920091009100910057
:103CE000910091009100910091009100910091004C
:103CF000910091009100910091009100910091003C
:103D0000910091009100910091009100910091002B
:103D1000910091009100910091009100910091001B
:103D2000910091009100910091009100910091000B
:103D300091009100910091009100900090009000FE
:103D400090009000900090009000900090009000F3
:103D500090009000900090009000900090009000E3
:103D600090009000900090009000900090009000D3
:103D700090009000900090009000900090009000C3
:103D800090009000900090009000900090009000B3
:103D9000900090009000900090008F008F008F00A6
:103DA0008F008F008F008F008F008F008F008F009B
:103DB0008F008F008F008F008F008F008F008F008B
:103DC0008F008F008F008F008F008F008F008F007B
:103DD0008F008F008F008F008F008F008F008F006B
:103DE0008F008F008F008F008F008F008F008F005B
:103DF0008F008F008F008F008F008F008E008E004D
:103E00008E008E008E008E008E008E008E008E0042
:103E10008E008E008E008E008E008E008E008E0032
:103E20008E008E008E008E008E008E008E008E0022
:103E30008E008E008E008E008E008E008E008E0012
:103E40008E008E008E008E008E008E008E008E0002
:103E50008E008E008E008E008E008E008E008E00F2
:103E60008D008D008D008D008D008D008D008D00EA
:103E70008D008D008D008D008D008D008D008D00DA
:103E80008D008D008D008D008D008D008D008D00CA
:103E90008D008D008D008D008D008D008D008D00BA
:103EA0008D008D008D008D008D008D008D008D00AA
:103EB0008D008D008D008D008D008D008D008D009A
:103EC0008D008D008C008C008C008C008C008C0090
:103ED0008C008C008C008C008C008C008C008C0082
:103EE0008C008C008C008C008C008C008C008C0072
:103EF0008C008C008C008C008C008C008C008C0062
:103F00008C008C008C008C008C008C008C008C0051
:103F10008C008C008C008C008C008C008C008C0041
:103F20008C008C008C008C008C008B008B008B0034
:103F30008B008B008B008B008B008B008B008B0029
:103F40008B008B008B008B008B008B008B008B0019
:103F50008B008B008B008B008B008B008B008B0009
:103F60008B008B008B008B008B008B008B008B00F9
:103F70008B008B008B008B008B008B008B008B00E9
:103F80008B008B008B008B008B008B008B008B00D9
:103F90008B008A008A008A008A008A008A008A00D0
:103FA0008A008A008A008A008A008A008A008A00C1
:103FB0008A008A008A008A008A008A008A008A00B1
:103FC0008A008A008A008A008A008A008A008A00A1
:103FD0008A008A008A008A008A008A008A008A0091
:103FE0008A008A008A008A008A008A008A008A0081
:103FF0008A008A008A008A008A0089008900890074
:104000008900890089008900890089008900890068
:104010008900890089008900890089008900890058
:104020008900890089008900890089008900890048
:104030008900890089008900890089008900890038
:104040008900890089008900890089008900890028
:104050008900890089008900890089008900890018
:10406000890089008900880088008800880088000D
:104070008800880088008800880088008800880000
:1040800088008800880088008800880088008800F0
:1040900088008800880088008800880088008800E0
:1040A00088008800880088008800880088008800D0
:1040B00088008800880088008800880088008800C0
:1040C00088008800880088008800880088008800B0
:1040D00088008700870087008700870087008700A7
:1040E0008700870087008700870087008700870098
:1040F0008700870087008700870087008700870088
:104100008700870087008700870087008700870077
:104110008700870087008700870087008700870067
:104120008700870087008700870087008700870057
:104130008700870087008700870087008700860048
:10414000860086008600860086008600860086003F
:10415000860086008600860086008600860086002F
:10416000860086008600860086008600860086001F
:10417000860086008600860086008600860086000F
:1041800086008600860086008600860086008600FF
:1041900086008600860086008600860086008600EF
:1041A00086008600860086008600860086008500E0
:1041B00085008500850085008500850085008500D7
:1041C00085008500850085008500850085008500C7
:1041D00085008500850085008500850085008500B7
:1041E00085008500850085008500850085008500A7
:1041F0008500850085008500850085008500850097
:104200008500850085008500850085008500850086
:104210008500850085008500850085008500850076
:10422000840084008400840084008400840084006E
:10423000840084008400840084008400840084005E
:10424000840084008400840084008400840084004E
:10425000840084008400840084008400840084003E
:10426000840084008400840084008400840084002E
:10427000840084008400840084008400840084001E
:10428000840084008400840084008400840084000E
:104290008400830083008300830083008300830005
:1042A00083008300830083008300830083008300F6
:1042B00083008300830083008300830083008300E6
:1042C00083008300830083008300830083008300D6
:1042D00083008300830083008300830083008300C6
:1042E00083008300830083008300830083008300B6
:1042F00083008300830083008300830083008300A6
:10430000830083008300820082008200820082009A
:10431000820082008200820082008200820082008D
:10432000820082008200820082008200820082007D
:10433000820082008200820082008200820082006D
:10434000820082008200820082008200820082005D
:10435000820082008200820082008200820082004D
:10436000820082008200820082008200820082003D
:10437000820082008200820082008200820081002E
:104380008100810081008100810081008100810025
:104390008100810081008100810081008100810015
:1043A0008100810081008100810081008100810005
:1043B00081008100810081008100810081008100F5
:1043C00081008100810081008100810081008100E5
:1043D00081008100810081008100810081008100D5
:1043E00081008100810081008100810081008100C5
:1043F00081008100810080008000800080008000BA
:1044000080008000800080008000800080008000AC
:10441000800080008000800080008000800080009C
:10442000800080008000800080008000800080008C
:10443000800080008000800080008000800080007C
:10444000800080008000800080008000800080006C
:10445000800080008000800080008000800080005C
:10446000800080008000800080008000800080004C
:104470007F007F007F007F007F007F007F007F0044
:104480007F007F007F007F007F007F007F007F0034
:104490007F007F007F007F007F007F007F007F0024
:1044A0007F007F007F007F007F007F007F007F0014
:1044B0007F007F007F007F007F007F007F007F0004
:1044C0007F007F007F007F007F007F007F007F00F4
:1044D0007F007F007F007F007F007F007F007F00E4
:1044E0007F007F007F007F007F007F007E007E00D6
:1044F0007E007E007E007E007E007E007E007E00CC
:104500007E007E007E007E007E007E007E007E00BB
:104510007E007E007E007E007E007E007E007E00AB
:104520007E007E007E007E007E007E007E007E009B
:104530007E007E007E007E007E007E007E007E008B
:104540007E007E007E007E007E007E007E007E007B
:104550007E007E007E007E007E007E007E007E006B
:104560007E007E007E007E007E007D007D007D005E
:104570007D007D007D007D007D007D007D007D0053
:104580007D007D007D007D007D007D007D007D0043
:104590007D007D007D007D007D007D007D007D0033
:1045A0007D007D007D007D007D007D007D007D0023
:1045B0007D007D007D007D007D007D007D007D0013
:1045C0007D007D007D007D007D007D007D007D0003
:1045D0007D007D007D007D007D007D007D007D00F3
:1045E0007D007D007D007D007D007C007C007C00E6
:1045F0007C007C007C007C007C007C007C007C00DB
:104600007C007C007C007C007C007C007C007C00CA
:104610007C007C007C007C007C007C007C007C00BA
:104620007C007C007C007C007C007C007C007C00AA
:104630007C007C007C007C007C007C007C007C009A
:104640007C007C007C007C007C007C007C007C008A
:104650007C007C007C007C007C007C007C007C007A
:104660007C007C007C007C007C007C007B007B006C
:104670007B007B007B007B007B007B007B007B0062
:104680007B007B007B007B007B007B007B007B0052
:104690007B007B007B007B007B007B007B007B0042
:1046A0007B007B007B007B007B007B007B007B0032
:1046B0007B007B007B007B007B007B007B007B0022
:1046C0007B007B007B007B007B007B007B007B0012
:1046D0007B007B007B007B007B007B007B007B0002
:1046E0007B007B007B007B007B007B007B007B00F2
:1046F0007A007A007A007A007A007A007A007A00EA
:104700007A007A007A007A007A007A007A007A00D9
:104710007A007A007A007A007A007A007A007A00C9
:104720007A007A007A007A0083048800000014007E
:104730008C000000000000000030F8FFFF000000C7
:1047400000000000008E00000000000000000000DB
:10475000000000000000000000005729040018833A
:1047600004DC0500001400840369010000140090BB
:104770001F891F950000000046696E6420746865FB
:104780002034206B6E6F6273206F6E2000950100E5
:10479000000074686520626F74746F6D206F66200E
:1047A000746865202020009501000000706C617421
:1047B000666F726D20616E64207469676874656EDF
:1047C000009507000000666F7572206F72206669A1
:1047D0007665207475726E732E0095000000004996
:1047E000276D20676F696E6720746F206D6F766527
:1047F0002020200095010000007468652065787411
:10480000727564657220746F20202020200095014D
:10481000000000766172696F757320706F73697440
:10482000696F6E73202020009507000000666F728C
:104830002061646A7573746D656E742E0095000056
:104840000000496E206561636820706F7369746948
:104850006F6E2C20202000950100000077652077E6
:10486000696C6C206E65656420746F2020202020A8
:1048700000950100000061646A7573742032206B3A
:104880006E6F627320617420202000950700000085
:104890007468652073616D652074696D652E00957F
:1048A000000000004E6F7A7A6C657320617265209B
:1048B0006174207468652020009501000000726911
:1048C00067687420686569676874207768656E201A
:1048D0002020009501000000796F752063616E2033
:1048E0006A75737420736C696465206100950700B4
:1048F00000007368656574206F6620706170657272
:104900000095000000006265747765656E2074682C
:1049100065206E6F7A7A6C6520200095010000009A
:10492000616E642074686520706C6174666F726D6E
:104930002E20202000950100000047726162206156
:10494000207368656574206F662020202020009504
:1049500007000000706170657220746F20617373CE
:104960006973742075732E009502000000506C6509
:104970006173652077616974008403690100001424
:104980000083048800000014008C00000000000078
:10499000000030F8FFFF00000000000000008E0063
:1049A0000000000000000000000000000000000007
:1049B00000000057290400188304DC0500001400DF
:1049C0008CE5370000941B00000000000000000090
:1049D00000000000009502000000506C65617365E6
:1049E0002077616974008EE6370000941B0000D0C8
:1049F00007000000000000000000000D4503001843
:104A00008E00000000CAE4FFFFD007000000000095
:104A100000000000002A0D3B00188E00000000C9B5
:104A2000E4FFFF0000000000000000000000000D97
:104A300045030018950000000041646A75737420F6
:104A40007468652066726F6E742074776F009501CC
:104A50000000006B6E6F627320756E74696C20705D
:104A6000617065722020200095010000006A757356
:104A70007420736C69646573206265747765656E14
:104A8000200095070000006E6F7A7A6C6520616ED9
:104A90006420706C6174666F726D00950200000096
:104AA000506C656173652077616974008E00000049
:104AB00000CAE4FFFFD00700000000000000000073
:104AC000000D450300188E000000007A1A0000D087
:104AD00007000000000000000000005181280018BD
:104AE0008E000000007A1A000000000000000000A4
:104AF00000000000000D4503001895000000004173
:104B0000646A75737420746865206261636B2074D5
:104B1000776F200095010000006B6E6F6273207547
:104B20006E74696C207061706572202020009501A0
:104B30000000006A75737420736C69646573206289
:104B400065747765656E200095070000006E6F7ACA
:104B50007A6C6520616E6420706C6174666F726D32
:104B6000009502000000506C6561736520776169F3
:104B700074008E000000007A1A0000D007000000C8
:104B8000000000000000000D450300188EC6240040
:104B90000000000000D0070000000000000000003E
:104BA00000A82F2200188EC624000000000000007C
:104BB00000000000000000000000000D4503001888
:104BC000950000000041646A757374207468652064
:104BD00072696768742074776F0095010000006B3C
:104BE0006E6F627320756E74696C2070617065728F
:104BF0002020200095010000006A75737420736CFA
:104C000069646573206265747765656E2000950739
:104C10000000006E6F7A7A6C6520616E6420706CA3
:104C20006174666F726D009502000000506C6561E2
:104C300073652077616974008EC62400000000004F
:104C400000D007000000000000000000000D450338
:104C500000188E3ADBFFFF00000000D007000000C4
:104C6000000000000000008B7C3700188E3ADBFF4C
:104C7000FF00000000000000000000000000000035
:104C8000000D45030018950000000041646A75732B
:104C90007420746865206C6566742074776F2000DA
:104CA00095010000006B6E6F627320756E74696C05
:104CB0002070617065722020200095010000006A5C
:104CC00075737420736C69646573206265747765AD
:104CD000656E200095070000006E6F7A7A6C652083
:104CE000616E6420706C6174666F726D0095020075
:104CF0000000506C656173652077616974008E3ABD
:104D0000DBFFFF00000000D00700000000000000F3
:104D10000000000D450300188E0000000000000098
:104D200000D0070000000000000000000045BE1B8E
:104D300000188E00000000000000000000000000CD
:104D4000000000000000000D450300189500000061
:104D500000436865636B20746861742070617065DE
:104D600072202020200095010000006A75737420D5
:104D7000736C69646573206265747765656E200085
:104D800095070000006E6F7A7A6C6520616E642072
:104D9000706C6174666F726D00891F950000000071
:104DA00046696E64207468652034206B6E6F627390
:104DB000206F6E2000950100000074686520626F0E
:104DC00074746F6D206F66207468652020200095D4
:104DD00001000000706C6174666F726D20616E641A
:104DE000207469676874656E009507000000666F3F
:104DF0007572206F722066697665207475726E73A5
:104E00002E00950000000049276D20676F696E67CE
:104E100020746F206D6F76652020200095010000C2
:104E20000074686520657874727564657220746FAB
:104E30002020202020009501000000766172696F1B
:104E4000757320706F736974696F6E732020200012
:104E50009507000000666F722061646A7573746D57
:104E6000656E742E009500000000496E2065616338
:104E70006820706F736974696F6E2C202020009514
:104E80000100000077652077696C6C206E656564B1
:104E900020746F2020202020009501000000616414
:104EA0006A7573742032206B6E6F62732061742098
:104EB00020200095070000007468652073616D650F
:104EC0002074696D652E0095000000004E6F7A7A9F
:104ED0006C657320617265206174207468652020A0
:104EE0000095010000007269676874206865696751
:104EF0006874207768656E2020200095010000000E
:104F0000796F752063616E206A75737420736C69A4
:104F10006465206100950700000073686565742072
:104F20006F66207061706572009500000000626518
:104F3000747765656E20746865206E6F7A7A6C652B
:104F40002020009501000000616E642074686520D7
:104F5000706C6174666F726D2E20202000950100C8
:104F60000000477261622061207368656574206F7C
:104F700066202020202000950700000070617065E9
:104F80007220746F206173736973742075732E00BF
:104F90009502000000506C6561736520776169744B
:104FA00000840369010000140083048800000014D9
:104FB000008C000000000000000030F8FFFF00003F
:104FC0000000000000008E00000000000000000053
:104FD0000000000000000000000000572904001835
:104FE0008304DC05000014008CE5370000941B00EE
:104FF000000000000000000000000000009502001A
:105000000000506C656173652077616974008EE5FE
:10501000370000941B0000D00700000000000000D3
:105020000000000D450300188E12060000CAE4FFC0
:10503000FFD00700000000000000000000DADF37AA
:1050400000188E11060000CAE4FFFF0000000000F7
:10505000000000000000000D45030018950000004E
:105060000041646A757374207468652066726F6E9F
:10507000742074776F0095010000006B6E6F62738F
:1050800020756E74696C207061706572202020003C
:1050900095010000006A75737420736C6964657310
:1050A000206265747765656E200095070000006ECC
:1050B0006F7A7A6C6520616E6420706C6174666FC3
:1050C000726D009502000000506C65617365207779
:1050D000616974008E11060000C9E4FFFFD007006B
:1050E0000000000000000000000D450300188E11B4
:1050F0000600007A1A0000D007000000000000003F
:1051000000000051812800188E120600007A1A0053
:10511000000000000000000000000000000D45033A
:105120000018950000000041646A7573742074686B
:1051300065206261636B2074776F20009501000029
:10514000006B6E6F627320756E74696C2070617095
:1051500065722020200095010000006A757374209C
:10516000736C69646573206265747765656E200091
:1051700095070000006E6F7A7A6C6520616E64207E
:10518000706C6174666F726D009502000000506C67
:10519000656173652077616974008E110600007B7C
:1051A0001A0000D007000000000000000000000D01
:1051B000450300188E2A27000000000000D00700D9
:1051C000000000000000000000CFF91F00188E2A28
:1051D00027000000000000000000000000000000A8
:1051E0000000000D45030018950000000041646AAE
:1051F00075737420746865207269676874207477A9
:105200006F0095010000006B6E6F627320756E7405
:10521000696C20706170657220202000950100008B
:10522000006A75737420736C6964657320626574B9
:105230007765656E200095070000006E6F7A7A6CC6
:105240006520616E6420706C6174666F726D00958C
:1052500002000000506C656173652077616974001D
:105260008E2A27000000000000D007000000000088
:1052700000000000000D450300188EF8E4FFFF0059
:10528000000000D007000000000000000000001730
:10529000F03100188EF9E4FFFF000000000000006C
:1052A0000000000000000000000D450300189500FC
:1052B00000000041646A75737420746865206C6531
:1052C00066742074776F200095010000006B6E6F8C
:1052D000627320756E74696C207061706572202035
:1052E000200095010000006A75737420736C696476
:1052F0006573206265747765656E20009507000010
:10530000006E6F7A7A6C6520616E6420706C6174D7
:10531000666F726D009502000000506C65617365E8
:105320002077616974008EF9E4FFFF00000000D06F
:1053300007000000000000000000000D45030018F9
:105340008E1106000000000000D0070000000000E1
:1053500000000000000BF81800188E110600000075
:105360000000000000000000000000000000000D30
:10537000450300189500000000436865636B2074C6
:105380006861742070617065722020202000950192
:105390000000006A75737420736C69646573206221
:1053A00065747765656E200095070000006E6F7A62
:1053B0007A6C6520616E6420706C6174666F726DCA
:1053C00000891F99000000005265704720427569EE
:1053D0006C64009600FF860088001F026E00880142
:1053E0001F026E00860088000302DC00860188012F
:1053F0000302DC00840369010000140083048800B8
:10540000000014008C000000000000000030F8FFD5
:10541000FF00000000000000008E000000000000FF
:1054200000000000000000000000000000005729FC
:105430000400188304DC0500001400901F8E1E2356
:10544000000028E5FFFF60EA000000000000000007
:1054500000009B1762001891000091010091030069
:105460009104008600860087006400FFFF8D0064C1
:1054700000FFFF8601860187016400FFFF8D006445
:1054800000FFFF91007F91017F91037F91047F8E48
:105490001F23000028E5FFFFC800000000000000F7
:1054A00000000000E6C361001888010A01038801BA
:1054B0000401FF8E1E23000027E5FFFFC800000047
:1054C000000000007FFEFFFF003E4900188C1E23F5
:1054D000000028E5FFFFC800000000000000810177
:1054E000000086008E31E0FFFFB8E9FFFF68010091
:1054F000000000000000000000229C3200188E31E5
:10550000E0FFFFB7E9FFFF68010000E3FFFFFF00D6
:105510000000001C5800001889888E31E0FFFFB79A
:10552000E9FFFFF0000000EDFFFFFF00000000605A
:10553000180000188E31E0FFFFB7E9FFFFF0000010
:1055400000E3FFFFFF00000000F22B0000188E7B3D
:10555000D1FFFFB7E9FFFFF00000009CFEFFFF0056
:10556000000000862F3000188E31E0FFFF6EEDFF47
:10557000FFF0000000300000000000000012720B7D
:1055800000188E31E0FFFF6EEDFFFFF0000000E33A
:10559000FFFFFF00000000F12B0000188E29D5FF4F
:1055A000FF6EEDFFFFF00000009CFEFFFF0000001B
:1055B00000A5232400188E30E0FFFF25F1FFFFF047
:1055C000000000300000000000000031C808001892
:1055D0008E31E0FFFF24F1FFFFF0000000E3FFFF4A
:1055E000FF00000000F12B0000188E29D5FFFF25D9
:1055F000F1FFFFF00000009CFEFFFF00000000A58F
:10560000232400188E31E0FFFFDCF4FFFFF00000E0
:1056100000300000000000000031C80800188E3182
:10562000E0FFFFDBF4FFFFF0000000E3FFFFFF00FF
:10563000000000F22B0000188E29D5FFFFDCF4FFDC
:10564000FFF00000009CFEFFFF00000000A52324E7
:1056500000188E31E0FFFF92F8FFFFF000000030ED
:105660000000000000000031C80800188E31E0FF83
:10567000FF93F8FFFFF0000000E3FFFFFF000000D2
:1056800000F22B0000188E28D5FFFF92F8FFFFF0E4
:105690000000009CFEFFFF00000000A5232400186E
:1056A0008E31E0FFFF49FCFFFFF0000000300000FA
:1056B000000000000031C80800188E31E0FFFF49EB
:1056C000FCFFFFF0000000E3FFFFFF00000000F21E
:1056D0002B0000188E29D5FFFF4AFCFFFFF00000C9
:1056E000009CFEFFFF00000000A5232400188E315F
:1056F000E0FFFF00000000F00000003000000000AC
:1057000000000031C80800188E31E0FFFF000000E3
:1057100000F0000000E3FFFFFF00000000F22B009C
:1057200000188E28D5FFFF00000000F00000009C4C
:10573000FEFFFF00000000A5232400188E31E0FFCB
:10574000FFB6030000F00000003000000000000081
:105750000031C80800188E31E0FFFFB7030000F0E9
:10576000000000E3FFFFFF00000000F22B00001824
:105770008E29D5FFFFB7030000F00000009CFEFF5C
:10578000FF00000000A5232400188E31E0FFFF6E0B
:10579000070000F0000000300000000000000031B1
:1057A000C80800188E31E0FFFF6D070000F0000010
:1057B00000E3FFFFFF00000000F22B0000188E281E
:1057C000D5FFFF6E070000F00000009CFEFFFF0009
:1057D000000000A5232400188E31E0FFFF240B00F9
:1057E00000F0000000300000000000000031C80898
:1057F00000188E31E0FFFF250B0000F0000000E3F1
:10580000FFFFFF00000000F12B0000188E29D5FFDC
:10581000FF240B0000F00000009CFEFFFF000000D2
:1058200000A5232400188E31E0FFFFDB0E0000F0FE
:10583000000000300000000000000031C80800181F
:105840008E31E0FFFFDC0E0000F0000000E3FFFF00
:10585000FF00000000F12B0000188E29D5FFFFDBB0
:105860000E0000F00000009CFEFFFF00000000A5FD
:10587000232400188E30E0FFFF92120000F0000099
:1058800000300000000000000031C80800188E3110
:10589000E0FFFF92120000F0000000E3FFFFFF00B6
:1058A000000000F12B0000188E29D5FFFF92120096
:1058B00000F00000009CFEFFFF00000000A5232474
:1058C00000188E31E0FFFF49160000F000000030A4
:1058D0000000000000000031C80800188E31E0FF11
:1058E000FF49160000F0000000E3FFFFFF0000008A
:1058F00000F12B0000188E29D5FFFF49160000F09B
:105900000000009CFEFFFF00000000A523240018FB
:105910008EAEEEFFFFA5F8FFFF680100003000002B
:10592000000000000018821D00188EAEEEFFFFA5DB
:10593000F8FFFFF0000000D0FFFFFF00000000AE06
:10594000250000188EAEEEFFFFA5F8FFFFF0000067
:1059500000E3FFFFFF00000000F12B0000188EAEF7
:10596000EEFFFF5B070000F00000009CFEFFFF0061
:10597000000000862F3000188E65F2FFFFA5F8FFAB
:10598000FFF0000000300000000000000012720B69
:1059900000188E64F2FFFFA5F8FFFFF0000000E39F
:1059A000FFFFFF00000000F12B0000188E65F2FFE2
:1059B000FFAE030000F00000009CFEFFFF000000AF
:1059C00000A5232400188E1CF6FFFFA5F8FFFFF0AA
:1059D000000000300000000000000031C80800187E
:1059E0008E1CF6FFFFA5F8FFFFF0000000E3FFFFAD
:1059F000FF00000000F12B0000188E1BF6FFFFAE29
:105A0000030000F00000009CFEFFFF00000000A566
:105A1000232400188ED3F9FFFFA5F8FFFFF0000044
:105A200000300000000000000031C80800188ED2CD
:105A3000F9FFFFA5F8FFFFF0000000E3FFFFFF0004
:105A4000000000F12B0000188ED3F9FFFFAE030019
:105A500000F00000009CFEFFFF00000000A52324D2
:105A600000188E89FDFFFFA5F8FFFFF00000003051
:105A70000000000000000031C80800188E89FDFFFA
:105A8000FFA5F8FFFFF0000000E3FFFFFF000000AC
:105A900000F12B0000188E89FDFFFFAD030000F020
:105AA0000000009CFEFFFF00000000A5232400185A
:105AB0008E40010000A6F8FFFFF00000003000005B
:105AC000000000000031C80800188E40010000A549
:105AD000F8FFFFF0000000E4FFFFFF00000000F10E
:105AE0002B0000188E41010000AD030000F0000003
:105AF000009BFEFFFF00000000A5232400188EF687
:105B0000040000A5F8FFFFF00000003000000000D6
:105B100000000031C80800188EF7040000A6F8FF46
:105B2000FFF0000000E4FFFFFF00000000F12B0089
:105B300000188EF7040000AD030000F00000009B89
:105B4000FEFFFF00000000A5232400188EAE080011
:105B500000A5F8FFFFF0000000300000000000008A
:105B60000031C80800188EAE080000A5F8FFFFF04D
:105B7000000000E4FFFFFF00000000F12B00001810
:105B80008EAD080000AE030000F00000009BFEFF99
:105B9000FF00000000A5232400188E650C0000A55E
:105BA000F8FFFFF0000000300000000000000031AE
:105BB000C80800188E640C0000A5F8FFFFF0000074
:105BC00000E4FFFFFF00000000F12B0000188E65CD
:105BD0000C0000AE030000F00000009BFEFFFF0081
:105BE000000000A5232400188E1B100000A5F8FF5C
:105BF000FFF0000000310000000000000031C80884
:105C000000188E1B100000A5F8FFFFF0000000E355
:105C1000FFFFFF00000000F12B0000188E1C100099
:105C200000AD030000F00000009BFEFFFF0000003D
:105C300000A5232400188ED2130000A6F8FFFFF061
:105C4000000000310000000000000031C80800180A
:105C50008ED2130000A5F8FFFFF0000000E3FFFF65
:105C6000FF00000000F12B0000188ED2130000ADE1
:105C7000030000F00000009BFEFFFF00000000A5F5
:105C8000232400188E89170000A5F8FFFFF00000FC
:105C900000310000000000000031C80800188E89A3
:105CA000170000A6F8FFFFF0000000E3FFFFFF0071
:105CB000000000F12B0000188E89170000AD0300D2
:105CC00000F00000009CFEFFFF00000000A5232460
:105CD00000188E401B0000A5F8FFFFF00000003008
:105CE0000000000000000031C80800188E401B00B2
:105CF00000A5F8FFFFF0000000E3FFFFFF00000039
:105D000000F12B0000188E3F1B0000AE030000F0D6
:105D10000000009CFEFFFF00000000A523240018E7
:105D20008E401B0000AD030000F0000000300000BA
:105D30000000000000D99200001889088601891827
:105D40008C401B0000AD030000F0000000000000CC
:105D500000810100008E54ECFFFFF0E9FFFF6801B5
:105D600000000000000000000000A3602800188E62
:105D700053ECFFFFEFE9FFFF6801000000000000A7
:105D800064010000B33E04001889908E54ECFFFFBC
:105D9000F0E9FFFFF000000000000000EDFFFFFF52
:105DA00060180000188E53ECFFFFF0E9FFFFF000D1
:105DB000000000000000E3FFFFFFF22B0000188E40
:105DC0005CF7FFFFEFE9FFFFF000000000000000BC
:105DD0009CFEFFFFA5232400188E53ECFFFF9DEDD2
:105DE000FFFFF00000000000000030000000EFC5E1
:105DF0000800188E54ECFFFF9DEDFFFFF00000003F
:105E000000000000E3FFFFFFF12B0000188E5CF79D
:105E1000FFFF9DEDFFFFF0000000000000009CFE72
:105E2000FFFFA5232400188E53ECFFFF4BF1FFFF6B
:105E3000F00000000000000030000000EFC5080086
:105E4000188E54ECFFFF4AF1FFFFF0000000000045
:105E50000000E3FFFFFFF12B0000188E5BF7FFFF50
:105E60004BF1FFFFF0000000000000009CFEFFFF70
:105E7000A5232400188E54ECFFFFF7F4FFFFF00079
:105E800000000000000030000000EFC50800188E80
:105E900053ECFFFFF8F4FFFFF000000000000000EB
:105EA000E3FFFFFFF22B0000188E5CF7FFFFF8F412
:105EB000FFFFF0000000000000009CFEFFFFA52394
:105EC0002400188E54ECFFFFA5F8FFFFF00000003F
:105ED0000000000030000000EFC50800188E53ECF1
:105EE000FFFFA5F8FFFFF000000000000000E3FF47
:105EF000FFFFF22B0000188E5CF7FFFFA6F8FFFFF4
:105F0000F0000000000000009CFEFFFFA52324001D
:105F1000188E53ECFFFF52FCFFFFF0000000000062
:105F2000000030000000EFC50800188E54ECFFFFA1
:105F300053FCFFFFF000000000000000E3FFFFFF44
:105F4000F22B0000188E5CF7FFFF52FCFFFFF00001
:105F50000000000000009CFEFFFFA5232400188E17
:105F600053ECFFFF00000000F00000000000000004
:105F700030000000EFC50800188E54ECFFFF000051
:105F80000000F000000000000000E3FFFFFFF22B24
:105F90000000188E5BF7FFFF00000000F00000001B
:105FA000000000009CFEFFFFA5232400188E54EC87
:105FB000FFFFAE030000F000000000000000300012
:105FC0000000EFC50800188E53ECFFFFAD03000082
:105FD000F000000000000000E3FFFFFFF22B0000D4
:105FE000188E5CF7FFFFAE030000F0000000000019
:105FF00000009CFEFFFFA5232400188E54ECFFFF39
:106000005A070000F000000000000000300000000F
:10601000EFC50800188E53ECFFFF5B070000F0008F
:10602000000000000000E3FFFFFFF22B0000188ECD
:106030005CF7FFFF5B070000F000000000000000BD
:106040009CFEFFFFA5232400188E54ECFFFF080BD5
:106050000000F00000000000000030000000EFC56C
:106060000800188E53ECFFFF080B0000F000000042
:1060700000000000E3FFFFFFF12B0000188E5CF72B
:10608000FFFF090B0000F0000000000000009CFE74
:10609000FFFFA5232400188E53ECFFFFB50E000070
:1060A000F00000000000000030000000EFC5080014
:1060B000188E54ECFFFFB60E0000F0000000000048
:1060C0000000E3FFFFFFF12B0000188E5CF7FFFFDD
:1060D000B50E0000F0000000000000009CFEFFFF75
:1060E000A5232400188E53ECFFFF63120000F0007C
:1060F00000000000000030000000EFC50800188E0E
:1061000054ECFFFF63120000F000000000000000EC
:10611000E3FFFFFFF12B0000188E5BF7FFFF631218
:106120000000F0000000000000009CFEFFFFA5231F
:106130002400188E54ECFFFF11160000F000000040
:106140000000000030000000EFC50800188E53EC7E
:10615000FFFF10160000F000000000000000E3FF49
:10616000FFFFF12B0000188E5CF7FFFF10160000F8
:10617000F0000000000000009CFEFFFFA5232400AB
:10618000188E09FBFFFF9DEDFFFF68010000000076
:10619000000030000000BEA41E00188E09FBFFFFA7
:1061A0009DEDFFFFF000000000000000D0FFFFFFAA
:1061B000AE250000188E09FBFFFF9DEDFFFFF000EC
:1061C000000000000000E3FFFFFFF12B0000188E2D
:1061D0000AFBFFFFA6F8FFFFF00000000000000030
:1061E0009CFEFFFFA5232400188EB6FEFFFF9DED49
:1061F000FFFFF00000000000000030000000EFC5CD
:106200000800188EB7FEFFFF9DEDFFFFF0000000B5
:1062100000000000E3FFFFFFF12B0000188EB6FE28
:10622000FFFFA5F8FFFFF0000000000000009CFE4B
:10623000FFFFA5232400188E640200009DEDFFFFE0
:10624000F00000000000000030000000EFC5080072
:10625000188E640200009DEDFFFFF00000000000BA
:106260000000E3FFFFFFF12B0000188E6402000026
:10627000A5F8FFFFF0000000000000009CFEFFFFFB
:10628000A5232400188E110600009DEDFFFFF000ED
:1062900000000000000030000000EFC50800188E6C
:1062A000110600009DEDFFFFF0000000000000005F
:1062B000E3FFFFFFF12B0000188E12060000A5F887
:1062C000FFFFF0000000000000009CFEFFFFA52380
:1062D0002400188EBE0900009DEDFFFFF0000000B5
:1062E0000000000030000000EFC50800188EBF0954
:1062F00000009DEDFFFFF000000000000000E3FF44
:10630000FFFFF12B0000188EBF090000A6F8FFFF69
:10631000F0000000000000009CFEFFFFA523240009
:10632000188E6C0D00009DEDFFFFF00000000000D6
:10633000000030000000EFC50800188E6C0D000052
:106340009DEDFFFFF000000000000000E4FFFFFFF4
:10635000F12B0000188E6C0D0000A5F8FFFFF00077
:106360000000000000009BFEFFFFA5232400188E04
:106370001A1100009DEDFFFFF0000000000000007A
:1063800030000000EFC50800188E191100009DEDC7
:10639000FFFFF000000000000000E4FFFFFFF12B12
:1063A0000000188E1A110000A5F8FFFFF000000091
:1063B000000000009BFEFFFFA5232400188EC614DA
:1063C00000009DEDFFFFF000000000000000300025
:1063D0000000EFC50800188EC71400009DEDFFFFF8
:1063E000F000000000000000E4FFFFFFF12B0000C0
:1063F000188EC7140000A5F8FFFFF0000000000091
:1064000000009BFEFFFFA5232400188E75180000D6
:106410009DEDFFFFF00000000000000030000000D4
:10642000EFC50800188E741800009DEDFFFFF00006
:10643000000000000000E4FFFFFFF12B0000188EB9
:1064400074180000A6F8FFFFF00000000000000034
:106450009BFEFFFFA5232400188E221C00009DED4B
:10646000FFFFF00000000000000031000000EFC559
:106470000800188E221C00009DEDFFFFF0000000B8
:1064800000000000E3FFFFFFF12B0000188E211C2D
:106490000000A5F8FFFFF0000000000000009BFED8
:1064A000FFFFA5232400188ECF1F00009DEDFFFFE6
:1064B000F00000000000000031000000EFC50800FF
:1064C000188ECF1F00009DEDFFFFF00000000000C0
:1064D0000000E3FFFFFFF12B0000188ECF1F00002C
:1064E000A5F8FFFFF0000000000000009BFEFFFF8A
:1064F000A5232400188E7D2300009DEDFFFFF000F2
:1065000000000000000031000000EFC50800188EF8
:106510007C2300009DEDFFFFF00000000000000064
:10652000E3FFFFFFF12B0000188E7D230000A5F88C
:10653000FFFFF0000000000000009CFEFFFFA5230D
:106540002400188E2A2700009DEDFFFFF0000000B8
:106550000000000030000000EFC50800188E2A2758
:1065600000009DEDFFFFF000000000000000E3FFD1
:10657000FFFFF12B0000188E2A270000A6F8FFFF6E
:10658000F0000000000000009CFEFFFFA523240097
:106590001889108E29270000A5F8FFFF30F20000AF
:1065A000000000000000000036F864001888010AAE
:1065B000010288010401FF891F8600880003020090
:1065C000008601880103020000860088001F020087
:1065D0000088011F020000891F4B00280616124E7A
:1065E0006F205344206361726420666F756E64008F
:1065F00065786974206D656E7500536F756E640003
:106600002D2D3E00202020004F4E20004F464600FA
:106610004C454420436F6C6F722020202020005294
:106620004544202020004F52414E4745200050490C
:106630004E4B202000475245454E2000424C5545C8
:10664000202000505552504C450057484954452091
:1066500000435553544F4D00546F6F6C20436F757A
:106660006E74200053494E474C45004455414C2020
:10667000200048656174204C4544730048656C7087
:106680002054657874202000416363656C657261F5
:106690007465004D6F6E69746F72204D6F64650094
:1066A00046696C616D656E74204F7074696F6E73AE
:1066B00000507265686561742053657474696E6713
:1066C00073004C6576656C204275696C6420506C73
:1066D00061746500486F6D652041786573004A6F8D
:1066E00067204D6F646500456E61626C6520537470
:1066F00065707065727320200044697361626C6517
:106700002053746570706572730053746F7020420B
:106710006C696E6B696E672100426C696E6B204C10
:10672000454473202020202020200052756E2053E5
:106730007461727475702053637269707400566569
:106740007273696F6E204E756D6265720047656E7B
:106750006572616C2053657474696E67730052656D
:1067600073746F72652044656661756C7473004361
:10677000616C696272617465204E6F7A7A6C6573C0
:10678000005072696E742066726F6D205344005021
:10679000726568656174005574696C6974696573C4
:1067A0000043616E63656C20746869732070726960
:1067B0006E743F005175697420746869732070723B
:1067C0006F636573733F004E6F00556E5061757354
:1067D0006500506175736500596573005265736596
:1067E000742053657474696E677320746F2000445D
:1067F000656661756C742076616C7565733F0050D9
:106800007265686561742053657474696E6773207E
:1068100020202000526967687420546F6F6C20201C
:106820002020202020202020004C65667420546FFA
:106830006F6C202020202020202020202000506C61
:106840006174666F726D2020202020202020004877
:10685000656174696E673A20202020202020202066
:106860002020200048656174696E673A00202D2D54
:1068700025006572726F72210020202020202020C8
:1068800020202020202020202020202020004578AB
:106890007472756465723A2020202D2D2D2F2D2DB8
:1068A0002D4300522045787472756465723A202D2C
:1068B0002D2D2F2D2D2D43004C204578747275649D
:1068C00065723A202D2D2D2F2D2D2D4300506C61FA
:1068D00074666F726D3A2020202D2D2D2F2D2D2DB9
:1068E0004300200020204E412020202000776169B5
:1068F00074696E6720002F20202043004320202051
:106900002000446F6E65210047414D45204F56459C
:1069100052210020202020204A6F67206D6F64657F
:106920002020202020202000202020202020202087
:10693000582B202020202020202020200020202034
:10694000202020284261636B29202020592D3E20E1
:1069500020002020202020202020582D2020202012
:10696000202020202020002020202020202020590E
:106970002B202020202020202020200020203C2D03
:106980005820284261636B2920205A2D3E20202068
:10699000002020202020202020592D2020202020D1
:1069A00020202020200020202020202020205A2DC0
:1069B000202020202020202020200020203C2D5995
:1069C00020284261636B29202020202020202000E5
:1069D00020202020202020205A2B20202020202072
:1069E00020202020004C6F61642072696768740069
:1069F0004C6F616400556E6C6F61642072696768EA
:106A00007400556E6C6F6164004C6F6164206C653E
:106A1000667400556E6C6F6164206C65667400442A
:106A2000696420706C617374696320657874727531
:106A30006465200066726F6D20746865206E6F7AE1
:106A40007A6C653F00446F6573206D79206E6F7AB4
:106A50007A6C650068656967687420636865636B54
:106A6000206F75743F004D792068656967687420F0
:106A7000697320676F6F6421004C657427732074FD
:106A8000727920616761696E2E00486F77276420F4
:106A9000697420676F3F2052656164792000746FCC
:106AA000207472792061207072696E743F202020FA
:106AB00020004D7920657874727564657273206169
:106AC0007265202020206E6F742068656174696E85
:106AD000672075702E2020202020436865636B207E
:106AE0006D79202020202020202020202020636F6E
:106AF0006E6E656374696F6E7321202020202020E4
:106B0000202000507265737320646F776E206F6E63
:106B100020746865202020677265792072696E672D
:106B20007320617420746F70206F667468652065CF
:106B3000787472756465727320616E6420202070B1
:106B4000756C6C2074686520626C61636B2E2E2EF0
:106B500020202000507265737320646F776E206F61
:106B60006E20746865202020677265792072696ED6
:106B70006720617420746F70206F662074686520D0
:106B8000657874727564657220616E6420202020BF
:106B900070756C6C2074686520626C61636B2E2E5E
:106BA0002E2020200049276D2068656174696E677A
:106BB000207570206D792020206578747275646569
:106BC00072212020202020202020202020506C65B1
:106BD00061736520776169742E2020202020202099
:106BE00020202020202020202020202020202020A5
:106BF0002020202020006775696465207475626517
:106C000073206F75742E204E6F77666565642066FD
:106C1000696C616D656E742066726F6D202074689A
:106C200065206261636B207468726F756768207499
:106C30006865747562657320756E74696C2069741B
:106C40002E2E2E20202000677569646520747562E1
:106C500065206F75742E20204E6F77666565642001
:106C600066696C616D656E742066726F6D2020744C
:106C70006865206261636B207468726F7567682055
:106C80007468657475626520756E74696C206974CA
:106C90002E2E2E20202000706F7073206F757420B0
:106CA000696E2066726F6E742E202049276D2068F1
:106CB000656174696E67207570206D79202020658C
:106CC0007874727564657220736F207765206361D4
:106CD0006E20206C6F6164207468652066696C6149
:106CE0006D656E742E2E2E0054686973206D696771
:106CF00068742074616B65206120202066657720B0
:106D00006D696E757465732E202020202020202050
:106D1000416E64207761746368206F75742C2074F1
:106D2000686520206E6F7A7A6C652077696C6C20BC
:106D300067657420484F54210048656174696E6727
:106D40002050726F67726573733A202020202020D4
:106D50002020202020202020202020202020202033
:106D60002020202020202020202020202020202023
:106D70002020202020202020202020202020202013
:106D8000202020202020202020004F4B2049276D4C
:106D9000207265616479212020202020202046690E
:106DA000727374207765276C6C206C6F616420743B
:106DB0006865726967687420657874727564657255
:106DC0002E2020202020507573682066696C616D2C
:106DD000656E7420696E2E2E2E20004772656174D8
:106DE00021204E6F77207765276C6C202020206C47
:106DF0006F616420746865206C65667420202020B3
:106E000020202065787472756465722E2050757329
:106E10006820202020202066696C616D656E7420DA
:106E2000646F776E2E2E2E20202020004F4B20499D
:106E3000276D207265616479212020202020202088
:106E4000506F70207468652067756964652074757B
:106E5000626520206F666620616E642070757368BD
:106E6000207468652020202066696C616D656E74F1
:106E700020646F776E2E2E2E20202020004F4B2076
:106E800049276D207265616479212020202020200F
:106E900020506F7020746865206775696465207480
:106EA00075626520206F666620616E642070756C67
:106EB0006C202020202020202066696C616D656E8A
:106EC000742067656E746C792E2E2E2020007468F5
:106ED000726F756768207468652067726579202015
:106EE000202072696E6720756E74696C20796F75E9
:106EF000206665656C20746865206D6F746F722004
:106F000074756767696E6720202074686520706CEF
:106F1000617374696320696E2E2E2E202020005725
:106F200068656E2066696C616D656E74206973209A
:106F3000202020657874727564696E67206F75749F
:106F4000206F66207468656E6F7A7A6C652C2050AD
:106F50007265737320274D27202020746F2073746F
:106F60006F7020657874727564696E672E202000DA
:106F70005768656E2066696C616D656E7420697313
:106F800020202020657874727564696E67206F75A3
:106F900074206F66207468656E6F7A7A6C652C2039
:106FA000507265737320274D27202020746F206551
:106FB00078697420202020202020202020202020DC
:106FC000005768656E206D792066696C616D656E2D
:106FD000742069732072656C65617365642C202070
:106FE000202020202020202020507265737320272D
:106FF0004D2720746F20657869742E202020202072
:107000002020202020202020202020202020202080
:107010002000477265617421202049276C6C207321
:10702000746F7020202072756E6E696E67206D79A6
:107030002065787472756465722E50726573732062
:107040004D20746F20636F6E74696E75652E2020FD
:107050002020202020202020202020202020202030
:107060002020004F4B212049276C6C206B656570F8
:10707000206D79202020206D6F746F722072756EE4
:107080006E696E672E20596F7520206D6179206EB4
:1070900065656420746F20707573682020202068F7
:1070A00061726465722E2E2E202020202020202048
:1070B000202020005765276C6C206B656570206769
:1070C0006F696E672E2020204C657473207472796E
:1070D00020746865206C6566742020206578747261
:1070E000756465722E205075736820202020202042
:1070F00066696C616D656E7420646F776E2E2E2EDE
:1071000020202020005765276C6C206B656570205F
:10711000676F696E672E202020496620796F75277A
:10712000726520686176696E672020202074726F16
:1071300075626C652C20636865636B206F757420C5
:10714000206D616B6572626F742E636F6D2F686561
:107150006C70202020004D79206D6F746F72207448
:10716000696D6564206F7574202061667465722096
:1071700035206D696E757465732E20202020507245
:10718000657373204D20746F20657869742E2020FC
:1071900020202020202020202020202020202020EF
:1071A0002020202020200053656C656374206265D8
:1071B0007374206C696E65732E0058204178697372
:1071C000204C696E6500592041786973204C696EC6
:1071D000650049276D20676F696E6720746F2070A6
:1071E00072696E7420206120736572696573206F07
:1071F00066206C696E657320736F77652063616EBE
:107200002066696E64206D792020202020206E6F1A
:107210007A7A6C6520616C69676E6D656E742E207C
:107220002020004C6F6F6B20666F722074686520A1
:10723000626573742020206D617463686564206CDE
:10724000696E6520696E2065616368617869732085
:107250007365742E204C696E657320617265206EB3
:10726000756D626572656420312D313320616E6405
:107270002E2E2E006C696E65206F6E65206973205E
:1072800065787472612020206C6F6E672E205468C0
:107290006520592061786973207365746973206C67
:1072A000656674206F6E2074686520706C6174650B
:1072B000616E642058206178697320697320726957
:1072C0006768742E00477265617421202049277613
:1072D000652073617665642020746865736520732A
:1072E000657474696E677320616E64202049276C31
:1072F0006C20757365207468656D20746F20202084
:10730000206D616B65206E696365207072696E74B3
:1073100073212020200057656C636F6D652120204C
:107320002020202020202020202049276D20746844
:1073300065205265706C696361746F722E205072A3
:107340006573732074686520726564204D20746FC6
:107350002020676574207374617274656421202035
:10736000202020202020004120626C696E6B696E15
:107370006720274D27206D65616E7349276D207743
:10738000616974696E6720616E642077696C6C63F3
:107390006F6E74696E7565207768656E20796F759C
:1073A0002020207072657373207468652062757484
:1073B000746F6E2E2E2E20004120736F6C69642036
:1073C000274D27206D65616E7320202049276D2091
:1073D000776F726B696E6720616E642077696C6C81
:1073E000757064617465206D792073746174757350
:1073F000202020207768656E2049276D2066696E01
:1074000069736865642E2E2E004F7572206E657844
:10741000742073746570732077696C6C2067657471
:10742000206D652073657420757020746F20202096
:10743000207072696E74212046697273742C2077F3
:1074400065276C6C20726573746F7265206D79208E
:107450006275696C642E2E2E2000706C6174666FEC
:10746000726D20736F2069742773202020206E694D
:10747000636520616E64206C6576656C2E204974AE
:10748000277370726F6261626C7920612062697427
:10749000206F6666202066726F6D20736869707059
:1074A000696E672E2E2E2020202000416161682CFD
:1074B0002074686174206665656C73202020206DDF
:1074C000756368206265747465722E202020202008
:1074D0002020204C6574277320676F206F6E206119
:1074E0006E64206C6F6164736F6D6520706C617386
:1074F0007469632120202020202020005765276CFC
:107500006C2074727920616761696E2120202020CF
:10751000202020202020202020202020202020206B
:10752000202020202020202020202020202020205B
:10753000202020202020202020202020202020204B
:1075400020202020202020202020202000576527D8
:107550006C6C206B65657020676F696E67202020FA
:1075600020616E64206C6F616420736F6D652020F4
:107570002020202020706C61737469632120466F85
:10758000722068656C7020676F746F206D616B6529
:1075900072626F742E636F6D2F68656C7000576533
:1075A000276C6C20676F20746F20746865206D6194
:1075B000696E6D656E752E20496620796F75206E37
:1075C00065656420202068656C7020676F20746F8B
:1075D0003A2020202020202020206D616B657262DF
:1075E0006F742E636F6D2F68656C702020200041D2
:1075F0007765736F6D6521202020202020202020BA
:107600002020205765276C6C20676F20746F2074D2
:107610006865205344202063617264204D656E7557
:1076200020616E6420796F7520202063616E207365
:10763000656C6563742061207072696E742120002E
:10764000436F6F6C210053746172742050726568CF
:107650006561742100526967687420546F6F6C0013
:107660004578747275646572004C65667420546F59
:107670006F6C00506C6174666F726D0020205468EE
:1076800065205265706C696361746F7220202020E0
:1076900000202020202D2D2D2D2D2D2D2D2D2D2088
:1076A00020202020200020202020202020202020FA
:1076B00020202020202020202020004669726D7785
:1076C0006172652056657273696F6E20352E2000D9
:1076D000010049033600FF006B00D100A000B80094
:1076E000D500A6000A0199003F018E0074018400B4
:1076F000A9017C00DE01740013026C0048026500E1
:107700007D025D00B2025600E7024E001C034600F7
:1077100051033D0086033200BB032200F003030047
:10772000AE44B24C104E184EA250EA518B59E45957
:107730002B61336371715D755378CD7913886C89D2
:1077400098957A96219AB89AA19B5F9C8EA107A2E0
:107750001AA57DA841C6B4C735C916CB6DCB4FCC91
:1077600011241FBECFEFD1E2DEBFCDBF18E0A0E0F5
:10777000B2E0EAEDFDE901E00BBF02C007900D9217
:10778000A634B107D9F71AE1A6E4B8E001C01D920A
:10779000A933B107E1F717E7C0E6D7E700E006C075
:1077A00022970109FE010BBF0E942ACDC032D107EA
:1077B00080E00807A9F70E94D4590C94EBCE0C94F2
:1077C0000000EF92FF920F931F937B018C0120E04A
:1077D00030E040E05FE40E94ED3F87FD11C0C8014A
:1077E000B70120E030E040E05FE40E94843D0E9469
:1077F000DD409B01AC01205030404040504806C065
:10780000C801B7010E94DD409B01AC01B901CA016A
:107810001F910F91FF90EF900895A0E0B0E0E3E199
:10782000FCE30C94F7CCFC01EA018081823008F47F
:1078300038C1DB019C91923008F430C1843059F496
:10784000943009F02EC1918111968C91119798175F
:1078500009F021C126C1943009F420C19230B1F45D
:10786000823009F01EC1CA01AF0128E0DA010D9093
:10787000AD01DC010D92CD012150C1F7DB01119664
:107880008C9111979181892389830AC1823009F4EF
:1078900005C1C280D380DB0112966D907C90139756
:1078A00024813581468157811496ED90FD900D918C
:1078B0001C911797C601861997095C0197FF04C0B0
:1078C000AA24BB24A81AB90AB0E2AB16B1040CF082
:1078D00061C0181619066CF5370148010A2C04C05E
:1078E00096948794779467940A94D2F781E090E015
:1078F000A0E0B0E00A2C04C0880F991FAA1FBB1F8C
:107900000A94D2F70197A109B1098E219F21A023E2
:10791000B123EE24FF248701E3940097A105B1056C
:1079200019F4EE24FF248701E628F72808291929ED
:107930003CC00097D1F1CA0CDB1C39014A010A2C6A
:1079400004C096948794779467940A94D2F781E060
:1079500090E0A0E0B0E00A2C04C0880F991FAA1F95
:10796000BB1F0A94D2F70197A109B109822393237F
:10797000A423B52321E030E040E050E00097A105CA
:10798000B10519F420E030E0A9012629372948295A
:1079900059290BC06C147D0424F4EE24FF248701C4
:1079A00004C0630120E030E0A9018181FB019181E5
:1079B000891709F445C0882349F0D801C701821B03
:1079C000930BA40BB50B9C01AD0104C02E193F090C
:1079D000400B510B57FD04C01982DB82CA820BC0D9
:1079E00081E08983DB82CA8250954095309521954C
:1079F0003F4F4F4F5F4F2C833D834E835F830DC0BE
:107A0000880F991FAA1FBB1F8C839D83AE83BF83E2
:107A10008A819B8101979B838A838C819D81AE8122
:107A2000BF819C01AD0121503040404050402F3F6C
:107A3000EFEF3E07EFEF4E07EFE35E0708F30BC0F3
:107A40008983DB82CA822E0D3F1D401F511F2C836C
:107A50003D834E835F8383E088832C813D814E810B
:107A60005F8157FF1DC0DA01C90181709070A0705D
:107A7000B0705695479537952795822B932BA42B5D
:107A8000B52B8C839D83AE83BF838A819B810196B6
:107A90009B838A8305C0E8E8F4E003C0FB0101C0D2
:107AA000FE01CF01CDB7DEB7EEE00C9413CDA0E21E
:107AB000B0E0EDE5FDE30C94FFCC69837A838B8322
:107AC0009C832D833E834F83588789E0E82EF12CD9
:107AD000EC0EFD1ECE010196B7010E94CF428E0131
:107AE0000F5E1F4FCE010596B8010E94CF42C7011D
:107AF000B801AE01475E5F4F0E940D3C0E940142FB
:107B0000A096E6E00C941BCDA0E2B0E0EAE8FDE32D
:107B10000C94FFCC69837A838B839C832D833E8373
:107B20004F8358878E01075F1F4FCE010196B80122
:107B30000E94CF4291E1E92EF12CEC0EFD1ECE0108
:107B40000596B7010E94CF428A8991E089278A8BE6
:107B5000C801B701AE01475E5F4F0E940D3C0E9415
:107B60000142A096E6E00C941BCDA0E2B0E0EBEB66
:107B7000FDE30C94F3CC69837A838B839C832D8300
:107B80003E834F835887CE010196BE01675F7F4FCA
:107B90000E94CF42CE010596BE016F5E7F4F0E94CC
:107BA000CF429985923078F089898230C0F0943044
:107BB00019F4823041F4CBC0843019F4923079F456
:107BC000C6C0923051F481E02A859A89291709F4B8
:107BD00080E08A87CE010996BCC0823051F481E0F2
:107BE0002A859A89291709F480E08A8BCE0141966B
:107BF000B0C06D847E848F849888ED88FE880F895C
:107C0000188DE0E2F0E080E090E0DC01AA24BB24E3
:107C1000650120E030E0A901B30161707070611569
:107C20007105D1F02E0D3F1D401F511F150126017A
:107C3000280E391E4A1E5B1E81E090E0A0E0B0E0F5
:107C40002E153F054007510718F080E090E0DC0159
:107C5000820D931DA41DB51DAA0CBB1CCC1CDD1CE4
:107C600017FF09C061E0262E312C412C512CA2288F
:107C7000B328C428D528319749F0EE0CFF1C001F0B
:107C8000111F9694879477946794C6CF6B897C89EB
:107C9000EB85FC856E0F7F1F6E5F7F4F7C8F6B8F38
:107CA00061E0EA857A89E71709F460E06A8F6B8DF5
:107CB0007C8D10C0FC01E170F070309729F0569572
:107CC0004795379527955068B695A79597958795C9
:107CD0006F5F7F4FB7FDEECF0CC0880F991FAA1FB3
:107CE000BB1F57FD8160220F331F441F551F61507A
:107CF00070408030E0E09E07E0E0AE07E0E4BE07C1
:107D000060F36B8F7C8F6FE7E62EF12C012D112D28
:107D1000E822F9220A231B2360E4E616F104010598
:107D2000110561F487FD0AC0211531054105510592
:107D300029F0805C9F4FAF4FBF4F80788D8F9E8F13
:107D4000AF8FB8A383E0898FCE01499602C088E83F
:107D500094E00E940142A096E2E10C940FCDA8E1CC
:107D6000B0E0E5EBFEE30C94FBCC69837A838B8374
:107D70009C832D833E834F8358878E01075F1F4F5F
:107D8000CE010196B8010E94CF4281E1E82EF12C8C
:107D9000EC0EFD1ECE010596B7010E94CF429985DB
:107DA000923008F483C08989823008F47BC02A8528
:107DB0003A8923272A87943011F0923021F49817BA
:107DC00009F06CC071C0843039F41D861E861F8690
:107DD000188A1C861B866AC0823019F484E0898761
:107DE00065C08B859C852B893C89821B930B9C8766
:107DF0008B872D853E854F855889ED88FE880F89B4
:107E0000188D2E153F054007510738F4220F331FF8
:107E1000441F551F01979C878B876FE170E0A12C51
:107E2000B12CC12CA0E4DA2E80E090E0DC012E150C
:107E30003F054007510740F08A299B29AC29BD29FD
:107E40002E193F09400B510BD694C794B794A794B1
:107E5000220F331F441F551F6150704041F76FE7D9
:107E6000E62EF12C012D112DE822F9220A231B23E5
:107E700060E4E616F1040105110561F487FD0AC00E
:107E8000211531054105510529F0805C9F4FAF4F09
:107E9000BF4F80788D879E87AF87B88B8E01075F35
:107EA0001F4F04C0870102C008E814E0C8010E9407
:107EB00001426896EAE00C9417CDA8E1B0E0E3E651
:107EC000FFE30C94FFCC69837A838B839C832D839F
:107ED0003E834F8358878E01075F1F4FCE01019667
:107EE000B8010E94CF4281E1E82EF12CEC0EFD1E7C
:107EF000CE010596B7010E94CF428985823040F0BD
:107F00008989823028F0C801B7010E94384301C036
:107F100081E06896E6E00C941BCDA8E1B0E0E3E9CF
:107F2000FFE30C94FFCC69837A838B839C832D833E
:107F30003E834F8358878E01075F1F4FCE01019606
:107F4000B8010E94CF4281E1E82EF12CEC0EFD1E1B
:107F5000CE010596B7010E94CF428985823040F05C
:107F60008989823028F0C801B7010E94384301C0D6
:107F700081E06896E6E00C941BCDA8E1B0E0E3EC6C
:107F8000FFE30C94FFCC69837A838B839C832D83DE
:107F90003E834F8358878E01075F1F4FCE010196A6
:107FA000B8010E94CF4281E1E82EF12CEC0EFD1EBB
:107FB000CE010596B7010E94CF428985823040F0FC
:107FC0008989823028F0C801B7010E94384301C076
:107FD0008FEF6896E6E00C941BCDA8E1B0E0E3EFEC
:107FE000FFE30C94FFCC69837A838B839C832D837E
:107FF0003E834F8358878E01075F1F4FCE01019646
:10800000B8010E94CF4281E1E82EF12CEC0EFD1E5A
:10801000CE010596B7010E94CF428985823040F09B
:108020008989823028F0C801B7010E94384301C015
:108030008FEF6896E6E00C941BCDA8E1B0E0E3E298
:10804000F0E40C94FFCC69837A838B839C832D832B
:108050003E834F8358878E01075F1F4FCE010196E5
:10806000B8010E94CF4281E1E82EF12CEC0EFD1EFA
:10807000CE010596B7010E94CF428985823040F03B
:108080008989823028F0C801B7010E94384301C0B5
:1080900081E06896E6E00C941BCDA8E1B0E0E3E552
:1080A000F0E40C94FFCC69837A838B839C832D83CB
:1080B0003E834F8358878E01075F1F4FCE01019685
:1080C000B8010E94CF4281E1E82EF12CEC0EFD1E9A
:1080D000CE010596B7010E94CF428985823040F0DB
:1080E0008989823028F0C801B7010E94384301C055
:1080F00081E06896E6E00C941BCDA8E0B0E0E3E8F0
:10810000F0E40C94FFCC7B018C0183E08983D801DF
:10811000C7018827B7FD83959927AA27BB27282F52
:108120008A83E114F1040105110519F482E08983C1
:1081300037C08EE190E09C838B83222389F080E01E
:10814000E81680E0F80680E0080780E8180769F183
:1081500010950095F094E094E11CF11C011D111D97
:10816000ED82FE820F831887C801B7010E94A741E4
:108170009C01215030401216130694F4022E04C0C4
:10818000EE0CFF1C001F111F0A94D2F7ED82FE8235
:108190000F8318878EE190E0821B930B9C838B8367
:1081A000CE0101960E94014204C060E070E080E0D0
:1081B0009FEC2896E6E00C941BCDACE0B0E0E3EE3B
:1081C000F0E40C9403CD69837A838B839C83CE0186
:1081D0000196BE016B5F7F4F0E94CF428D8182303E
:1081E00081F1823070F1843021F48E81882369F12D
:1081F0000AC02F81388537FD24C06E812F313105AB
:108200003CF0662311F120E030E040E050E821C06E
:108210008EE190E0821B930B29853A854B855C8526
:1082200004C056954795379527958A95D2F76623CA
:1082300081F050954095309521953F4F4F4F5F4FBE
:1082400008C020E030E0A90104C02FEF3FEF4FEF5E
:108250005FE7B901CA012C96E2E00C941FCDA8E0BB
:10826000B0E0E5E3F1E40C94FDCC7B018C011A82D3
:10827000611571058105910519F482E089835FC05C
:1082800083E089838EE1C82ED12CDC82CB82ED8203
:10829000FE820F831887C801B7010E94A741FC0125
:1082A0003197F7FF3AC0AA27BB27AE1BBF0B21E0CF
:1082B00030E040E050E00A2E04C0220F331F441F7C
:1082C000551F0A94D2F721503040404050402E2193
:1082D0003F214023512361E070E080E090E02115D0
:1082E00031054105510519F460E070E0CB0104C08F
:1082F00016950795F794E794AA95D2F7E62AF72AF8
:10830000082B192BED82FE820F8318878EE190E0F7
:108310008E1B9F0B9C838B8312C0309781F00E2E97
:1083200004C0EE0CFF1C001F111F0A94D2F7ED824F
:10833000FE820F831887CE1ADF0ADC82CB82CE0141
:1083400001960E9401422896E8E00C9419CDAF9264
:10835000BF92CF92DF92EF92FF920F931F937B0118
:108360008C0180E0E81680E0F80681E0080780E0F4
:10837000180758F4EFEFEE16F1040105110509F0A6
:1083800090F480E090E0DC0117C0F0E0EF16F0E040
:10839000FF06F0E00F07F1E01F0750F480E190E0E6
:1083A000A0E0B0E009C088E090E0A0E0B0E004C048
:1083B00088E190E0A0E0B0E020E230E040E050E072
:1083C000281B390B4A0B5B0B5701680104C0D6947C
:1083D000C794B794A7948A95D2F7D601C501805760
:1083E0009B4FFC018081281B310941095109C901BA
:1083F0001F910F91FF90EF90DF90CF90BF90AF90C3
:108400000895EF92FF920F931F93CF93DF93FC0198
:10841000248135814681578161818081823020F4B9
:108420004061EFEFF0E0A3C0843009F49BC08230DC
:1084300009F492C0211531054105510509F48FC099
:108440000280F381E02D8FEFE238F8070CF05AC07C
:10845000C2E8DFEFCE1BDF0BCA31D1056CF5790125
:108460008A010C2E04C016950795F794E7940A9498
:10847000D2F781E090E0A0E0B0E00C2E04C0880FBD
:10848000991FAA1FBB1F0A94D2F70197A109B1092E
:1084900082239323A423B52321E030E040E050E081
:1084A0000097A105B10519F420E030E0A9012E29BB
:1084B0003F29402B512B03C020E030E0A901DA0115
:1084C000C9018F779070A070B07080349105A105BC
:1084D000B10539F427FF09C0205C3F4F4F4F5F4F74
:1084E00004C0215C3F4F4F4F5F4FE1E0F0E0203090
:1084F00080E0380780E0480780E4580728F5E0E08E
:10850000F0E022C0E038F1056CF5E158FF4FDA01E8
:10851000C9018F779070A070B07080349105A1056B
:10852000B10539F427FF09C0205C3F4F4F4F5F4F23
:1085300004C0215C3F4F4F4F5F4F57FF05C056951A
:10854000479537952795319687E056954795379506
:1085500027958A95D1F70BC0E0E0F0E005C0E0E098
:10856000F0E005C0EFEFF0E020E030E0A9018E2F51
:10857000879588278795942F9F77679566276795B6
:10858000E695E22EA92FA82BFE2FF62B622F732F34
:108590008A2F9F2FCDB7DEB7E6E00C941BCDDC0110
:1085A000FB012C9111963C91119712968C91129788
:1085B000482F4F7750E0982F991F9927991F1396AE
:1085C0006C911397862F880F892B90E0661F662782
:1085D000661F6183009739F5211531054105510565
:1085E00011F482E029C082E89FEF9383828367E0E1
:1085F000220F331F441F551F6A95D1F783E08083F4
:1086000009C0220F331F441F551F82819381019798
:1086100093838283203080E0380780E0480780E43D
:10862000580778F320C08F3F910579F42115310563
:108630004105510519F484E08083089544FF03C087
:1086400081E0808310C010820EC08F5790409383CA
:10865000828383E0808387E0220F331F441F551FEE
:108660008A95D1F7506424833583468357830895D0
:10867000FC01DB019081923008F449C08C9182307A
:1086800008F445C0943051F461818430B1F51196FD
:108690002C91119730E0261B310941C0843021F024
:1086A000923041F48230B1F111968C911197882368
:1086B000A1F12DC06181823001F111968C91119749
:1086C0006817D9F42281338112968D919C9113976A
:1086D0008217930794F028173907BCF0248135815D
:1086E0004681578114968D919D910D90BC91A02D3E
:1086F00082179307A407B50718F4662341F00DC04D
:10870000281739074A075B0728F4662331F021E070
:1087100030E005C020E030E002C02FEF3FEFC9019C
:10872000089510924E08E4E0F1E08081807E80831D
:10873000E5E0F1E08081807E808308956F927F92F2
:108740008F929F92AF92BF92CF92DF92EF92FF9261
:108750000F931F93DF93CF93CDB7DEB7A8970FB6D4
:10876000F894DEBF0FBECDBF8C01FC018181882350
:1087700009F0CDC08281882309F4BAC0C8010296ED
:108780000E9444CB882309F4C2C0B2C0809146083D
:108790008823E9F4C8010C9640E856E968E970E0DE
:1087A0000E9427CB81E08093460811C07E01089487
:1087B000E11CF11CC7010E9423CBD8011C96F701D4
:1087C0008AE001900D928150E1F7109246083CE05A
:1087D000E32EF12CE00EF11EC7010E9444CB88234A
:1087E00099F085E0F801808381E081838E01055F47
:1087F0001F4FC8010E9423CBD701F8018AE00190E6
:108800000D928150E1F783C0A1FC10C08091470810
:108810008823F1F4C801469640E856E968E970E01B
:108820000E9427CB81E08093470812C025E1E22E09
:10883000F12CEC0EFD1EC7010E9423CBD8015696E9
:10884000F7018AE001900D928150E1F710924708FC
:1088500096E1E92EF12CE00EF11EC7010E9444CBF7
:10886000882399F086E0F801808381E081838E017E
:10887000015E1F4FC8010E9423CBD701F8018AE097
:1088800001900D928150E1F742C060904E08D614DD
:1088900061F16D24EE24FF247724CC24C39493014A
:1088A0000E2C02C0359527950A94E2F720FF16C0DA
:1088B00095010E2C02C0359527950A94E2F720FD0C
:1088C0000DC0F8018181882349F4E082C182C4018E
:1088D00040E452E460E070E00E9427CB0894E11C81
:1088E000F11CF5E0EF16F104D1F6D0924E080FC05E
:1088F00082E0882E912C800E911EC4010E946ACBCA
:10890000D0900301AD2CBB24D0FE40CF4FCFA89612
:108910000FB6F894DEBF0FBECDBFCF91DF911F9190
:108920000F91FF90EF90DF90CF90BF90AF909F900E
:108930008F907F906F900895FC01DB01F894818106
:10894000908111827894882321F09C9311961C9237
:10895000119708958FE180934E08089588E498E078
:108960006CE779E140E00E94E9C808958091510ADE
:108970009091520A009729F481E08093580A80E090
:1089800008958091530A9091540A20914F0A309192
:10899000500AB9010E948FCCE091550AF091560A15
:1089A000E80FF91F8091530A9091540A0196B9017A
:1089B0000E948FCC9093540A8093530A8091510A5D
:1089C0009091520A01979093520A8093510A8081A4
:1089D0000895F8948091510A9091520A20914F0A7B
:1089E0003091500A281B390B7894C901089580935F
:1089F0005B0A089581E080935C0A089580915B0A88
:108A000008952091510A3091520A81E021153105D3
:108A100009F080E008950E94B64408951F930E94D3
:108A2000B644182F0E94B644982F812F1F910895A5
:108A30001F93DF93CF9300D0CDB7DEB70E94B6442B
:108A40008A830E94B64489830E94B644182F0E94EC
:108A5000B644982F6A817981812F0F900F90CF9122
:108A6000DF911F9108952F923F924F925F926F92E4
:108A70007F928F929F92AF92BF92CF92DF92EF92AE
:108A8000FF920F931F93DF93CF93CDB7DEB7E59798
:108A90000FB6F894DEBF0FBECDBF7C010E94EF661B
:108AA000882309F0BDC0F70180818B3809F059C0D7
:108AB0008091510A9091520A8931910508F4B0C011
:108AC00081E29BE00E94CF5B0E94B64481E090E08F
:108AD00090935E0A80935D0A0E9418455B016C01C9
:108AE0000E9418456DA77EA78FA798AB0E941845D6
:108AF0001B012C010E94184569AB7AAB8BAB9CAB78
:108B00000E9418457B018C010E94184569837A8375
:108B10008B839C8300D000D095E0692E712C6C0E65
:108B20007D1EEDB7FEB7E182F28203831483C30199
:108B3000B601A5010DA51EA52FA538A972016101D9
:108B400089A89AA8ABA8BCA80E949C710F900F900E
:108B50000F900F90C301BE016F5F7F4F0E94BB6FEC
:108B60005FC08E3809F05CC08091510A9091520A22
:108B70008A31910508F454C081E29BE00E94CF5BEA
:108B80000E94B64481E090E090935E0A80935D0A73
:108B90000E9418455B016C010E9418456DA77EA7D5
:108BA0008FA798AB0E9418451B012C010E94184505
:108BB00069AB7AAB8BAB9CAB0E9418457B018C01F7
:108BC0000E94184569837A838B839C830E940B459E
:108BD0008DAB00D000D089E1682E712C6C0E7D1E0B
:108BE000EDB7FEB7E182F28203831483C301B601BD
:108BF000A5010DA51EA52FA538A97201610189A89F
:108C00009AA8ABA8BCA80E949C710F900F900F90DF
:108C10000F90C301BE016F5F7F4F4DA90E943E7050
:108C2000E5960FB6F894DEBF0FBECDBFCF91DF91B2
:108C30001F910F91FF90EF90DF90CF90BF90AF907A
:108C40009F908F907F906F905F904F903F902F906C
:108C500008951092520A1092510A1092540A1092DA
:108C6000530A1092570A1092580A10925E0A1092F4
:108C70005D0A089581E020915D0A30915E0A2630F8
:108C8000310509F080E008950F931F93CF93DF9390
:108C90000E94B644182F0E94B644082F0E94B64482
:108CA000093009F4C1C00A3090F4053009F4BCC0A1
:108CB000063030F4033009F1043009F0BBC0B4C011
:108CC000073009F4B4C0083008F0AEC0B0C00C30B2
:108CD00009F459C00D3038F40A3009F48DC00B3056
:108CE00009F0A8C097C0073109F446C00F3109F454
:108CF00066C00D3009F09EC057C0113019F4C1EDA7
:108D0000DBE002C0CAE3DBE00E940E45BC01CE01FD
:108D100049960E94AC9E84E09FE00E94879F882332
:108D200009F48EC084E09FE00E94A19F882309F08F
:108D300087C0113019F421ED3BE002C02AE33BE08B
:108D4000C90149960E94A19F882309F079C081E05A
:108D500080935A0A113019F481ED9BE002C08AE336
:108D60009BE0499661E004C08AE39BE0499660E09D
:108D70000E94E19F81E05FC080915B0A91E08927BA
:108D800080935B0AF7CF113019F4C1EDDBE002C02C
:108D9000CAE3DBE00E940B45682F70E061707070E1
:108DA000CE010E946351E6CF0E940B45682F70E010
:108DB0006170707081E29BE00E94EC60DBCF81E229
:108DC0009BE061E00E94E7600E940E45BC0184E0E8
:108DD0009FE00E94AC9E84E09FE00E94A19F11E072
:108DE000182710935A0A83E59BE0612F0E94E19FA8
:108DF0008AEE9BE0612FBCCF0E94B64421E030E0B8
:108E000030935E0A20935D0A682F70E06170707085
:108E100084E007C00E94B644682F70E061707070F3
:108E200083E00E94BA81A6CF0E94B644A3CF0E94DD
:108E30001845A0CF80E0DF91CF911F910F91089549
:108E4000113009F091CF81ED9BE090CFFC01462FCE
:108E5000828193812081318182179307A0F46281FE
:108E6000738184819581860F971FB9010E948FCCF1
:108E7000A681B781A80FB91F4C9382819381019677
:108E800093838283089581E080870895682F8FE41B
:108E90009AE00E94264708952F923F924F925F9248
:108EA0006F927F928F929F92AF92BF92CF92DF92FA
:108EB000EF92FF920F931F93DF93CF93CDB7DEB75F
:108EC000CF56D0400FB6F894DEBF0FBECDBF0E9484
:108ED000CF76882309F18091510A9091520A20910E
:108EE0004F0A3091500A2817390709F415C50E9416
:108EF0001D77882309F410C50E942077682F8FE41E
:108F00009AE00E942647E7CF8091510A9091520A39
:108F1000009711F40E942F770E94D688882309F1C8
:108F20008091510A9091520A20914F0A3091500A33
:108F30002817390709F4F6C40E94DC88882309F44D
:108F4000F1C40E94EA88682F8FE49AE00E942647C5
:108F5000E7CF8091510A9091520A009711F40E9434
:108F6000698980915A0A882391F084E09FE00E94E9
:108F70004C9F882361F083E59BE060E00E94E19FC5
:108F80008AEE9BE060E00E94E19F10925A0A809175
:108F90005B0A882309F0CCC480915C0A882309F01D
:108FA000C7C480915D0A90915E0A8330910581F477
:108FB0000E94D979882341F089E69AE00E9444CB47
:108FC000882331F00E94D76710925E0A10925D0AE2
:108FD00080915D0A90915E0A81309105D9F50E94D9
:108FE000D979882329F410925E0A10925D0A32C062
:108FF0008091510A9091520A009761F181E29BE0C1
:109000000E94CF5B8091530A9091540A60914F0A5D
:109010007091500A0E948FCCE091550AF091560A47
:10902000E80FF91F808189838B3811F08E3829F47D
:10903000CE0101960E9433450DC0893859F48091C4
:10904000510A9091520A8230910520F00E94B64454
:109050000E94B64480915D0A90915E0A823091052B
:1090600051F48FE59AE00E9444CB882321F01092BE
:109070005E0A10925D0A80915D0A90915E0A8430CA
:10908000910571F583E79AE00E9444CB882341F073
:1090900081E29BE060E072E040E00E94725C1CC0F4
:1090A0008091590A813019F481ED9BE002C08AE376
:1090B0009BE049960E94879F882371F08091590A0E
:1090C000813019F481ED9BE002C08AE39BE0499670
:1090D0000E944C9F882321F010925E0A10925D0A34
:1090E00080915D0A90915E0A85309105F1F483E7E5
:1090F0009AE00E9444CB882341F081E29BE065E343
:1091000072E040E00E94725C0CC084E09FE00E942C
:10911000879F882331F084E09FE00E944C9F882342
:1091200021F010925E0A10925D0A80915D0A909182
:109130005E0A8630910561F58DE79AE00E9444CB86
:10914000882351F08091880A81FF1EC081E29BE054
:1091500060E00E94F55D1CC084EA9CE00E9412A5BC
:109160008823B1F08091880A82FF04C084EA9CE0E1
:109170000E9432A381E29BE060E070E040E050E0BA
:109180000E943D5C0E94C77410925E0A10925D0AB4
:1091900080915D0A90915E0A009709F0C9C38091A1
:1091A000510A9091520A009709F4C2C381E29BE0F0
:1091B0000E94CF5B8091530A9091540AE0914F0A2C
:1091C000F091500A2091550A3091560ABF010E9431
:1091D0008FCC820F931FDC018C9189838138C9F475
:1091E0008091510A9091520A8131910508F4A0C3EF
:1091F0000E94B64481E090E090935E0A80935D0AFD
:109200000E9418450E9418450E9418450E94184562
:109210008FC38B3811F08E3829F4CE0101960E944D
:10922000334586C3863889F48091510A9091520A59
:109230008230910508F47CC30E94B6440E94B64473
:109240008093590A0E94CB6773C3893839F580919E
:10925000510A9091520A8230910508F469C30E9424
:10926000B6440E94B644A82EAA1CAA24AA1C00E058
:1092700010E0C82EDD24C601002E02C0959587950A
:109280000A94E2F780FF04C0802F6A2D0E94BA8101
:109290000F5F1F4F0530110571F74AC3823821F562
:1092A0008091510A9091520A8D30910508F440C383
:1092B0000E94B6440E9418453B014C010E9418458B
:1092C0001B012C010E9418456B017C01FAE1AF2EB5
:1092D000B12CAC0EBD1EC501B401A30192018101E8
:1092E0000E94D071C50144C08C3809F044C08091FF
:1092F000510A9091520A8531910508F419C30E94D0
:10930000B6440E9418456B017C010E9418451B0160
:109310002C010E9418454B015C010E941845AE9635
:109320006CAF7DAF8EAF9FAFAE970E94184500D057
:1093300000D0EEE26E2E712C6C0E7D1EEDB7FEB7E6
:109340006183728383839483C301B701A601920171
:10935000810175016401AE968CAC9DACAEACBFAC26
:10936000AE970E949C710F900F900F900F90C301C9
:109370000E945669DDC28538E9F48091510A9091C6
:10938000520A8530910508F4D3C282E090E09093B0
:109390005E0A80935D0A0E94B6440E94184528EE3A
:1093A00033E040E050E00E9470CCAB01BC018FE59F
:1093B0009AE022C18439B9F58091510A9091520AFC
:1093C0008530910508F4B4C20E94B6440E94B644A8
:1093D0008093870A0E940E458C010E94B6448093B8
:1093E000880A0115110581F0B80180E090E020E4C1
:1093F00032E44FE050E00E9470CCAB01BC018DE73D
:109400009AE00E9427CB85C08E010A5F1F4FC801DA
:109410000E9423CBADE7BAE0F8018AE001900D92FB
:109420008150E1F776C0853909F088C08091510AF2
:109430009091520A8630910508F47AC20E94B6448F
:109440000E94B644C82E0E94B644882E0E94B6449C
:10945000A82E0E94B644082FC0FC04C083E89EE0FA
:109460000E941FC28092850EA092860E41E0C1FE2E
:1094700040E083E89EE06FE47AE00E94F2C5E0916C
:10948000F20CFF27E7FDF095EE0FFF1FEC51F34FB5
:1094900020813181FEE023383F0731F084EA9CE0EF
:1094A00063E87EE00E948BA2002341F0C2FC06C06C
:1094B00083E89EE0602F41E00E9463C2C2FE38C292
:1094C000002389F0602F70E080E090E020E432E437
:1094D0004FE050E00E9470CCAB01BC018DE79AE0F8
:1094E0000E9427CB0EC08E01005F1F4FC8010E9453
:1094F00023CBADE7BAE0F8018AE001900D928150EC
:10950000E1F781E08093870A8091880A84708093D4
:10951000880A81E29BE069E170E04FE050E00E9440
:109520003D5C84EA9CE06091870A0E940DA586E07C
:1095300090E090935E0A80935D0AFAC1982F935849
:10954000923098F58091510A9091520A8830910595
:1095500008F4EEC10E94B6440E940B45082F0E94F9
:1095600018456B017C010E940E4523E030E03093EA
:109570005E0A20935D0ABC0180E090E020E432E4C2
:109580004FE050E00E9470CCAB01BC0189E69AE04C
:109590000E9427CB81E09981943809F080E0602F08
:1095A000A70196010E949B80C3C1873841F5809135
:1095B000510A9091520A8630910508F4B9C184E0AD
:1095C00090E090935E0A80935D0A0E94B6440E94E8
:1095D000B6448093590A0E940E450E940E45BC0174
:1095E00080E090E020E432E44FE050E00E9470CC54
:1095F000AB01BC0183E79AE00E9427CB99C18D386B
:1096000099F48091510A9091520A8630910508F49C
:109610008FC185E090E090935E0A80935D0A0E947E
:10962000B6440E94B644D7CF8F3809F048C0809125
:10963000510A9091520A8230910508F479C10E9432
:10964000B6440E940B456EE0A62EB12C00E010E05F
:10965000C82EDD2452E4652E712C6C0E7D1E42E076
:10966000842E912C8C0E9D1EC601002E02C0959555
:1096700087950A94E2F780FF18C0C3010E94AA7B75
:10968000C301B8010E94F271FC0180819181A28125
:10969000B3818A839B83AC83BD83F894C401B501F5
:1096A00044E050E00E949ACE78940F5F1F4F84E010
:1096B00090E0A80EB91E05301105B1F639C1803908
:1096C00009F03FC08091510A9091520A8230910571
:1096D00008F42EC10E94B6440E940B45C82E36E500
:1096E000A32EB12CAC0EBD1EC5010E94AA7B2EE09C
:1096F000622E712C00E010E0DD248A2CAB2CC60118
:10970000002E02C0959587950A94E2F780FF0CC061
:10971000F894882D9A2DB8010E94FA71B30144E0A3
:1097200050E00E9484CE78940F5F1F4FA4E0B0E019
:109730006A0E7B1E0530110511F7CE018A5A9F4F24
:1097400017CE8139C9F48091510A9091520A833021
:10975000910508F4EDC00E94B6440E940B45C82E46
:109760000E940B45082F8C2D602F0E94EC818C2DC0
:10977000602F0E94EC81DCC0823949F58091510A4A
:109780009091520A8630910508F4D2C00E94B644E6
:109790000E940B45082F0E940B45E0968FAFE09783
:1097A0000E940B45AF968FAFAF970E940B45C82E16
:1097B0000E940B458C2D0E945375802FE0966FAD53
:1097C000E097AF964FADAF970E94B574B1C08339A3
:1097D000B9F48091510A9091520A8630910508F4AB
:1097E000A7C00E94B6440E940E456C010E940E451F
:1097F0008C010E940B45C601B8010E94796198C096
:10980000883819F58091510A9091520A8430910557
:1098100008F48EC08091530A9091540A0091510A25
:109820001091520A0396BF010E948FCC820F931FA2
:10983000FC01808190E004960817190708F478C0AD
:109840000E94B6440E94444673C0863999F48091C0
:10985000510A9091520A8330910508F469C00E9420
:10986000B6440E940B45082F0E940B45802F0E9492
:10987000D3A15EC08739C9F48091510A9091520AF0
:109880008230910508F454C00E94B6440E940B45F2
:10989000882311F484E006C0813019F40E945762D5
:1098A00047C082E00E94386243C0883999F48091B1
:1098B000510A9091520A82309105D0F10E94B6442B
:1098C0000E940B450E94E24F81E29BE060E00E9413
:1098D000F55D2EC0893981F48091510A9091520A28
:1098E0008530910528F10E94B6440E9418458FE406
:1098F0009AE00E9423591CC08A39D1F48091510A00
:109900009091520A8230910598F00E94B6440E94CC
:10991000B6440E9489540CC00E941D77882309F424
:10992000F3CAFACA0E94DC88882309F412CB19CB47
:10993000C159DF4F0FB6F894DEBF0FBECDBFCF9138
:10994000DF911F910F91FF90EF90DF90CF90BF902C
:10995000AF909F908F907F906F905F904F903F90CF
:109960002F90089589E89AE06CE779E140E00E9441
:10997000E9C880E092E09093500A80934F0A1092D9
:10998000520A1092510A1092540A1092530A8FE40C
:1099900098E09093560A8093550A1092570A1092B5
:1099A000580A8FE59AE00E9423CB89E69AE00E944C
:1099B00023CB83E79AE00E9423CB8DE79AE00E94B5
:1099C00023CB0895FC018281882349F4A081B181D1
:1099D0009C918481982381E019F480E0089580E0CF
:1099E0000895FC01A081B181662331F012968C911B
:1099F00012979481892B05C012968C9112979581AC
:109A0000892312968C9312970895EF92FF920F93E9
:109A10001F93DF93CF93CDB7DEB768970FB6F89457
:109A2000DEBF0FBECDBF7C018E010F5F1F4FC8018F
:109A300064E779E140E00E94E9C8C8010E94E24C75
:109A4000882361F58E01095F1F4FC80164E779E142
:109A500041E00E94E9C8C80161E00E94F14C8E011A
:109A6000035F1F4FC80162E779E144E00E94E9C843
:109A7000C8010E94E24C882321F0C7010E945B4D7F
:109A80000DC08E010D5E1F4FC80164E779E141E012
:109A90000E94E9C8C80160E00E94F14C68960FB6C8
:109AA000F894DEBF0FBECDBFCF91DF911F910F9114
:109AB000FF90EF900895EF92FF920F931F93DF9323
:109AC000CF93CDB7DEB768970FB6F894DEBF0FBE61
:109AD000CDBF7C018E010F5F1F4FC80164E779E1A4
:109AE00040E00E94E9C8C80160E00E94F14C8E018C
:109AF000095F1F4FC80164E779E140E00E94E9C8AF
:109B0000C80161E00E941EC9F70110828E01035F47
:109B10001F4FC80162E779E144E00E94E9C8C8012B
:109B20000E94E24C882319F0C7010E94054D8E0166
:109B30000D5E1F4FC80164E779E141E00E94E9C86A
:109B4000C80160E00E94F14C68960FB6F894DEBF41
:109B50000FBECDBFCF91DF911F910F91FF90EF907E
:109B60000895CF92DF92EF92FF920F931F93DF93AE
:109B7000CF93CDB7DEB768970FB6F894DEBF0FBEB0
:109B8000CDBF7C0194E7C92E99E1D92E8E010F5FDC
:109B90001F4FC801B60141E00E94E9C8C80160E05A
:109BA0000E94F14C8E01095F1F4FC801B60141E0D0
:109BB0000E94E9C8C80161E00E941EC98E01035FCE
:109BC0001F4F82E7C82E89E1D82EC801B60144E0B4
:109BD0000E94E9C8C80160E00E94F14C8E010D5E50
:109BE0001F4FC801B60144E00E94E9C8C80160E007
:109BF0000E941EC9C7010E945B4DF70111821282AB
:109C0000138268960FB6F894DEBF0FBECDBFCF911A
:109C1000DF911F910F91FF90EF90DF90CF9008950B
:109C20008FE89AE06CE779E140E00E94E9C8089586
:109C30008BEB9AE06CE779E140E00E94E9C885E9A6
:109C40009AE00E9450C80895DF93CF9300D0CDB71B
:109C5000DEB7BC0181E0898382E38A83CE0101966D
:109C600042E050E00E949ACE0F900F90CF91DF918A
:109C70000895CF93DF93EC0140E050E060EE70E494
:109C80000E94379DCE01029646E656E666EA7EE3DE
:109C90000E94379DCE01049640E050E060E172E4FE
:109CA0000E94379DDF91CF9108950F931F93CF931B
:109CB000DF93EB018B01085E1F4F009719F4CB0176
:109CC00067E002C0CB0168E30E94A4CEC80162E352
:109CD0000E94A4CECE010A960E94394ECE01409633
:109CE0000E94394ECE014A960E94244ECE0106961D
:109CF00064EF71E00E94BACECE01029665E070E09A
:109D00000E94BACECE01049664EF71E00E94BACEF2
:109D1000CE0108966CE271E00E94BACEDF91CF913D
:109D20001F910F910895CF93DF93EC0140EA56E81D
:109D300061E070E00E94B2CECE01049649E150E0AD
:109D400060E070E00E94B2CECE01089643EE5FE084
:109D500060E070E00E94B2CEBE01605F7F4F80ED98
:109D600096E740E550E00E949ACEDF91CF910895AA
:109D70000F931F93DF93CF9300D00F92CDB7DEB731
:109D80008C0160E00E94A4CEC801029661E00E94AE
:109D9000A4CE8FEF89831B821A82B8016C5F7F4F3C
:109DA000CE01019643E050E00E949ACE0F900F90B2
:109DB0000F90CF91DF911F910F9108950F931F93F3
:109DC000DF93CF9300D000D0CDB7DEB7082F162F8A
:109DD00080E491E067E04C830E94A4CE09831A835B
:109DE0004C814B83CE01019664E471E043E050E086
:109DF0000E949ACE0F900F900F900F90CF91DF910D
:109E00001F910F910895EF92FF920F931F93CF939D
:109E1000DF937B018C01EA01CA01B7010E94BACE2F
:109E2000CE010496B8010E94BACEDF91CF911F9166
:109E30000F91FF90EF900895AC016BE770E084EF15
:109E400091E00E94034F0895CF93DF93EC016CEDF6
:109E500070E00E94BACECE0102966CED70E00E94D6
:109E6000BACECE0104966EE670E00E94BACECE0164
:109E7000069665E00E94A4CEDF91CF9108958EE60C
:109E800091E060E00E94A4CE80E791E068EB7BE087
:109E90000E94BACE82E791E068EB7BE00E94BACEE6
:109EA00084E791E068EB7BE00E94BACE86E791E020
:109EB00068EE73E00E94BACE88E791E068EB7BE041
:109EC0000E94BACE8AE791E068EB7BE00E94BACEAE
:109ED0008CE791E040E050E060EA71E40E94379D39
:109EE00080E891E040E050E060E87FE30E94379D29
:109EF00082E891E040E050E060E771E40E94379D25
:109F000084E891E040E050E060E771E40E94379D12
:109F100086E891E06FE070E00E94BACE88E891E0B8
:109F200060E80E94A4CE089582E490E061E00E947F
:109F3000979C91E0813009F090E0892F0895DF939C
:109F4000CF93CDB7DEB764970FB6F894DEBF0FBEE0
:109F5000CDBFDE011196EEEAF5E084E101900D92AD
:109F60008150E1F70E94944F882381F085EE97E3BA
:109F7000A0E0B0E089839A83AB83BC838AE79AE14F
:109F8000A0E0B0E08D839E83AF83B887CE010196B9
:109F90006EE070E044E150E00E949ACE64960FB605
:109FA000F894DEBF0FBECDBFCF91DF910895682F2B
:109FB000833008F061E082E490E00E94A4CE0E9429
:109FC0009F4F0895DF93CF93CDB7DEB729970FB694
:109FD000F894DEBF0FBECDBFDE011596E9EAF5E0CD
:109FE00085E001900D928150E1F781EC93E29A8334
:109FF000898384E193ED9C838B838AE692E062E21D
:10A0000070E044E150E00E949ACECE01059666E0F1
:10A0100070E045E050E00E949ACE84E090E06FE965
:10A020000E94A4CE8CE090E06BE10E94A4CE0E943E
:10A030009F4F85E995E06CE871E044E150E00E94B3
:10A040009ACE0E943F4F80E691E061E00E94A4CE4C
:10A0500084E790E00E94934E88E591E00E94244FAF
:10A06000CE01019664E470E044E050E00E949ACE94
:10A0700080E090E060E071E00E94554E81E090E069
:10A080006CE171E00E94554E80E491E00E94B84E70
:10A090008AE491E00E941C4F86E591E060E00E9416
:10A0A000A4CE29960FB6F894DEBF0FBECDBFCF91D8
:10A0B000DF91089580E491E00E94B84E8AE491E037
:10A0C0000E941C4F88E591E00E94244F80E691E0B9
:10A0D00061E00E94A4CE0895DF93CF93CDB7DEB7A1
:10A0E0002C970FB6F894DEBF0FBECDBF19821A822F
:10A0F0001B821C821D821E821F82188619861A8668
:10A100001B861C86CE01019662E671E04CE050E0B1
:10A110000E949ACE2C960FB6F894DEBF0FBECDBF2C
:10A12000CF91DF91089582E090E06BE10E94A4CE90
:10A1300082E490E061E00E94A4CE0E946C500E94F4
:10A14000E24F089581EC9AE06CE779E140E00E94EB
:10A15000E9C808952F923F925F926F927F928F92FB
:10A160009F92AF92BF92CF92DF92EF92FF920F93A6
:10A170001F93DF93CF93CDB7DEB72E970FB6F8942A
:10A18000DEBF0FBECDBF5C01562E1A013E872D8764
:10A19000380147012EE6E22E29E1F22E6E010894E5
:10A1A000C11CD11CC601B70142E00E94E9C88E0162
:10A1B000095F1F4FC801B70145E00E94E9C8C5010A
:10A1C000B301A60198010E94F4CA86EC95E0F5015E
:10A1D000978B868B508E99E1692E712C6A0C7B1CB3
:10A1E000A5014A5E5F4F8AE0E82EF12CE80CF91CCD
:10A1F000C301B50100E211EA27E030E0CC24C394AA
:10A200000E946C9EC50186589F4FB1010E9403C9F0
:10A21000F501E058FF4F5082A401465E5F4FC50133
:10A220008F579F4FB3012D853E850E94899BF50175
:10A23000EB56FF4F918280822E960FB6F894DEBFC8
:10A240000FBECDBFCF91DF911F910F91FF90EF9087
:10A25000DF90CF90BF90AF909F908F907F906F9046
:10A260005F903F902F9008950F931F93CF93DF93AC
:10A27000EC018C0106581F4FC80160E00E94F14CB0
:10A28000C80161E00E941EC9CE0149960E94729DDC
:10A29000CE010E9459CACE018F579F4F0E94539BF7
:10A2A000DF91CF911F910F910895CF93DF93EC0130
:10A2B00049960E945DA0CE018F579F4F0E940F9B31
:10A2C000DF91CF9108958F579F4F662319F00E9419
:10A2D000019B08950E944E9B0895882321F0809150
:10A2E0008000806803C0809180008F73809380001D
:10A2F0000895882321F08091A000806803C0809198
:10A30000A0008F738093A0000895EF92FF920F93A7
:10A310001F93DF93CF93CDB7DEB72C970FB6F8948A
:10A32000DEBF0FBECDBFF62EEFB6F894FC018281E2
:10A330008823F9F4862F81508E3F90F080E00E94B0
:10A340007951CE01019664E779E143E00E94E9C8C2
:10A3500061E0FF2DFF3F09F060E0CE01019621C0D2
:10A3600070E07093A9006093A80081E00E94795189
:10A3700023C0813009F5862F81508E3FA8F080E000
:10A380000E946D518E01095F1F4FC80168E679E197
:10A3900045E00E94E9C861E08F2D8F3F09F060E041
:10A3A000C8010E94F14C08C070E07093890060936E
:10A3B000880081E00E946D51EFBE2C960FB6F89494
:10A3C000DEBF0FBECDBFCF91DF911F910F91FF90E8
:10A3D000EF90089587EC9AE06CE779E140E00E9405
:10A3E000E9C80895CF93DF93EC010E94FE4491E009
:10A3F00089270E94F744CE0161E80E9498C8DF9146
:10A40000CF910895FC0183A194A1009741F023A16D
:10A4100034A181E02430310519F480E0089580E012
:10A420000895CF92DF92EF92FF920F931F93CF93F5
:10A43000DF93EC018B018881882399F17E01DC2E6A
:10A44000CF2CCE0160E00E9438C887FF2AC00E944E
:10A45000D276882321F0CE010E94D57608C00E94D2
:10A46000CF76882321F40E94D688882321F1C80161
:10A4700061E80E9498C813C08D2D9C2D6C2F0E94FE
:10A4800038C80E9446472196CE15DF05ACF3C801B7
:10A4900061E802C0C80162E80E9498C8789481E02F
:10A4A00001C080E0DF91CF911F910F91FF90EF905D
:10A4B000DF90CF900895F894E8800E94E944FF244B
:10A4C0008E159F0538F3C0E0D0E0DECF86E090E047
:10A4D0009093110B8093100B81E08093140B0895DF
:10A4E000CF93DF93EB0161E00E943DC88A31910573
:10A4F00040F4CE0161E80E9498C8CE0160E070E0AF
:10A5000007C0CE0161E80E9498C8CE0169EF71E0F2
:10A510000E949BC8DF91CF910895EF92FF920F9315
:10A520001F93DF93CF93CDB7DEB764970FB6F89440
:10A53000DEBF0FBECDBF8B01F8947E010894E11CF5
:10A54000F11CC7010E949669C80161E80E9498C881
:10A55000C70160E070E00E94F271FC01408151810E
:10A5600062817381C8010E94B1C8C70161E070E0D7
:10A570000E94F271FC014081518162817381C801A6
:10A580000E94B1C8C70162E070E00E94F271FC0154
:10A590004081518162817381C8010E94B1C8C701A5
:10A5A00063E070E00E94F271FC01408151816281A0
:10A5B0007381C8010E94B1C8C70164E070E00E94C5
:10A5C000F271FC014081518162817381C8010E9456
:10A5D000B1C8C80160E070E00E949BC8789464969E
:10A5E0000FB6F894DEBF0FBECDBFCF91DF911F91A4
:10A5F0000F91FF90EF9008950F931F93CF93DF93E8
:10A60000EB018C010D5F1F4FCB0161E80E9498C8E0
:10A61000C8010E94FC77682FCE010E9498C8DF9184
:10A62000CF911F910F9108956F927F928F929F9279
:10A63000AF92BF92CF92DF92EF92FF920F931F9350
:10A64000DF93CF930F92CDB7DEB77C018B01CDB6F0
:10A65000DEB68DB69EB6ADB6BEB6CB0161E80E9441
:10A6600098C8C70161E00E9438C8882379F00E9429
:10A670003F78BC01009751F0C8010E9498C8C801FA
:10A6800060E00E9498C83C2D292D37C08DB79EB739
:10A690004F970FB6F8949EBF0FBE8DBFEDB6FEB6B6
:10A6A0000894E11CF11CC7016FE140E050E00E94FA
:10A6B000D675BC01F7018081882329F061157105E9
:10A6C00011F48E3281F3C8010E9498C820E0E22F75
:10A6D000F0E02F3161F0EE0DFF1D6081662339F04F
:10A6E000C80129830E9498C829812F5FF0CFC80133
:10A6F00060E00E9498C83A2D2B2D832F922F0FB621
:10A70000F8949EBF0FBE8DBF0FB6F894DEBE0FBE8D
:10A71000CDBE0F90CF91DF911F910F91FF90EF90E1
:10A72000DF90CF90BF90AF909F908F907F906F9071
:10A7300008958F929F92AF92BF92CF92DF92EF9245
:10A74000FF920F931F93DF93CF93CDB7DEB7A82E61
:10A75000E92E6B018DB69EB661E00E943DC88C016A
:10A760008A2D9E2D63E00E9438C8482FA82EBB2456
:10A770008DB79EB78A199B090FB6F8949EBF0FBE7E
:10A780008DBFEDB6FEB60894E11CF11CC701B801FF
:10A7900050E00E9484CEC60161E80E9498C800E0A3
:10A7A00010E008C0F70161917F01C6010E9498C8BE
:10A7B0000F5F1F4F0A151B05ACF30FB6F8949EBE32
:10A7C0000FBE8DBECF91DF911F910F91FF90EF9043
:10A7D000DF90CF90BF90AF909F908F9008952F9271
:10A7E0003F924F925F926F927F928F929F92AF9221
:10A7F000BF92CF92DF92EF92FF920F931F93DF935E
:10A80000CF930F92CDB7DEB7C82EB92E4B012DB620
:10A810003EB661E00E943DC8A82E792E8C2D9B2D5E
:10A8200063E00E9438C8D82E482E55248DB79EB7B5
:10A83000841995090FB6F8949EBF0FBE8DBF0DB752
:10A840001EB70F5F1F4F602E1983C8016A2D772D29
:10A850004D2D50E00E9484CEE02EF12E00E010E05D
:10A860000BC0602F6C5F8C2D9B2D0E9438C8F701A8
:10A8700081937F010F5F1F4F0415150594F30FB7E8
:10A88000F894862D99816A2D772D4D2D50E00E94E8
:10A890009ACE0FBFC40161E80E9498C8C4016D2D13
:10A8A0000E9498C80FB6F8943EBE0FBE2DBE0F9002
:10A8B000CF91DF911F910F91FF90EF90DF90CF909C
:10A8C000BF90AF909F908F907F906F905F904F90D0
:10A8D0003F902F9008950F931F93CF93DF93EB0139
:10A8E00061E00E9438C8082F80FF02C00E94D7672D
:10A8F00001FF02C00E942946CE0161E80E9498C86B
:10A90000CE0160E00E9498C8DF91CF911F910F9116
:10A9100008951092110B1092100B08950F931F932E
:10A92000CF93DF938091E10A882379F401EE1AE056
:10A93000C2E2D0E0CE0160E00E94979CF8018193D2
:10A940008F012196C233D105A9F78091E10A8823AE
:10A9500069F4A1EEBAE080E090E0FC01E85EFE4F11
:10A96000E491ED9301968E309105B9F781EE9AE06E
:10A97000DF91CF911F910F91089581EF9AE0089593
:10A980008091100B9091110B0895EF92FF92CF934D
:10A99000DF9381EF9AE00E94C877EC010097F1F411
:10A9A00084E09FE060E070E00E94AC9E83E59BE065
:10A9B00060E070E00E94AC9E8AEE9BE060E070E098
:10A9C0000E94AC9E0E9429460E94F87A0E94D76796
:10A9D00082E090E09093110B8093100BCE01DF91F9
:10A9E000CF91FF90EF900895CF92DF92EF92FF9278
:10A9F0000F931F93CF93DF936C017B01CB0161E831
:10AA00000E9498C801EF1AE0C1E0D0E008C0C6017A
:10AA10006C2F0E9438C8F80181938F012196F601AE
:10AA2000808190E0C817D90794F310920F0B0E9411
:10AA3000C554682FC7010E9498C8DF91CF911F911C
:10AA40000F91FF90EF90DF90CF9008950E942189A1
:10AA5000882331F085E090E09093110B8093100BE8
:10AA60000E9429460E94D76708958091100B90910B
:10AA7000110B8130910571F484E090E09093110BFB
:10AA80008093100B87ED9AE040E452E46FE070E0B1
:10AA90000E9427CB81E08093120B0895DF92EF9202
:10AAA000FF920F931F93CF93DF938C01EB01FC0177
:10AAB0008081882309F461C1D02EE12EC80161E0B4
:10AAC0000E9438C8F82EC80162E00E9438C8873159
:10AAD00009F46DC08831A0F4833009F449C0843092
:10AAE00028F48130A1F18230A8F529C08D3009F415
:10AAF00077C0863109F481C08C3009F03EC15BC05B
:10AB0000803209F491C0813250F48A3109F44AC08C
:10AB10008E3109F480C0893109F02FC13EC08332E3
:10AB200009F499C0843220F4813209F026C18AC028
:10AB3000843209F49AC0853209F01FC1D2C0CE0117
:10AB400061E80E9498C8CE0169EF71E012C180935C
:10AB5000120B20C0CE0161E80E9498C8FF2DF13091
:10AB600019F481ED9BE002C08AE39BE0499659C04D
:10AB70008F2D813019F401ED1BE002C00AE31BE0C8
:10AB80008D2D9E2D62E00E943DC8BC01C8014996F2
:10AB90000E94AC9ECE0161E8A1C0C801BE010E9426
:10ABA0009953E9C0C801BE010E94EF53E4C0CE0131
:10ABB0000E94F251E0C0EF2DE13019F401ED1BE0ED
:10ABC00002C00AE31BE08D2D9E2D62E00E9438C872
:10ABD000682F70E061707070C8010E946351DACF15
:10ABE000C80163E00E9438C8682F70E0617070701F
:10ABF00081E29BE00E94EC60BEC0CE0161E80E9451
:10AC000098C8FF2DF13019F481ED9BE002C08AE372
:10AC10009BE0499626C0CE0161E80E9498C884E076
:10AC20009FE00E94769FA3C0CE0161E80E9498C871
:10AC30008F2D813019F481ED9BE002C08AE39BE007
:10AC4000499606C0CE0161E80E9498C884E09FE062
:10AC50000E94709F8CC0CE0161E80E9498C884E079
:10AC60009FE00E944C9F682F38C0CE0161E80E948F
:10AC700098C8EF2DE13019F481ED9BE002C08AE322
:10AC80009BE049960E9484A1882311F000E801C04E
:10AC900000E084E09FE00E9484A1882311F080E41A
:10ACA00001C080E0082BFF2DF13019F481ED9BE00D
:10ACB00002C08AE39BE049960E9489A1082B8F2D50
:10ACC000813019F421ED3BE002C02AE33BE0C901E9
:10ACD00049960E944C9F602F682BCE010E9498C815
:10ACE0004AC0CE0161E80E9498C8EF2DE13019F406
:10ACF00081ED9BE002C08AE39BE049960E947B9F26
:10AD0000BC01CE010E949BC8FF2DF13019F421ED4A
:10AD10003BE002C02AE33BE0C90149960E947F9FC5
:10AD2000BC01CE010E949BC88F2D813019F481EDAA
:10AD30009BE002C08AE39BE049960E94839FBC018E
:10AD4000CE010E949BC884E09FE00E947B9FBC01D3
:10AD5000CE010E949BC884E09FE00E947F9FBC01BF
:10AD6000CE010E949BC884E09FE00E94839FBC01AB
:10AD7000CE010E949BC881E001C080E0DF91CF91AD
:10AD80001F910F91FF90EF90DF900895CF92DF9287
:10AD9000EF92FF920F931F93DF93CF93CDB7DEB760
:10ADA00064970FB6F894DEBF0FBECDBF8C017B0158
:10ADB000FC018081882309F406C1C80160E00E947B
:10ADC00038C887FD00C1E82FF0E0EA31F10508F04E
:10ADD000FAC0EE58FF4FEE0FFF1F0590F491E02DE3
:10ADE0000994C801B7010E947052EFC0C70161E821
:10ADF0000E9498C881EFC82E8AE0D82E8601C7012C
:10AE0000F60161916F010E9498C8F8018081882342
:10AE100009F4DBC0F0E1CF16FBE0DF0679F7D5C01F
:10AE20008091100B9091110B9C01215030402230E9
:10AE3000310518F08530910531F481E29BE064E042
:10AE400070E00E94015C81E08093120BC70161E811
:10AE5000B7C0C70161E80E9498C80E94E944AC01EC
:10AE600060E070E047C0F8948E010F5F1F4FC8018B
:10AE70000E949669C70161E80E9498C8C80160E015
:10AE800070E00E94F271FC01408151816281738106
:10AE9000C7010E94B1C8C80161E070E00E94F27170
:10AEA000FC014081518162817381C7010E94B1C858
:10AEB000C80162E070E00E94F271FC0140815181A2
:10AEC00062817381C7010E94B1C8C70160E038C0C8
:10AED000C801B7010E948D5278C0C801B7010E9415
:10AEE000FC5273C0C70161E80E9498C80E94717744
:10AEF000AB01BC01C70157C0C801B7010E94F4549F
:10AF000064C0C801B7010E9414535FC0C7010E940A
:10AF1000F2515BC0C801B7010E944E5556C0C7012F
:10AF200061E80E9498C8F8940E94D979882321F496
:10AF30000E940145882311F460E001C061E0C7016F
:10AF40000E9498C8789441C0C801B7010E949953E3
:10AF50003CC0C801B7010E94EF5337C0C801B70118
:10AF60000E946B5432C0C70161E80E9498C8C701B3
:10AF700040E050E0BA010E94B1C8C70140E050E093
:10AF8000BA010E94B1C8C70140E050E0BA010E9476
:10AF9000B1C8C70140E050E0BA010E94B1C8C70182
:10AFA00040E050E0BA010E94B1C80FC0C70161E89B
:10AFB0000E9498C881E29BE00E94CA5B682FC7018B
:10AFC0000E9498C802C080E001C081E064960FB67C
:10AFD000F894DEBF0FBECDBFCF91DF911F910F91CF
:10AFE000FF90EF90DF90CF9008950F931F93DF9322
:10AFF000CF93CDB7DEB72A970FB6F894DEBF0FBE5A
:10B00000CDBF81E09AE10E940252882309F0E9C095
:10B010008091D70A882301F187ED9AE00E9444CB02
:10B020008823D1F481E08093140B8E010F5F1F4FB2
:10B03000C8010E9423CBA7EDBAE0F8018AE0019095
:10B040000D928150E1F78FEF99E6A8E18150904091
:10B05000A040E1F700C000008091120B8823A9F006
:10B060008091140B882389F41092120B8091130B9A
:10B070000E949B591092130B8DEC9AE00E9467CBB3
:10B080001092E10A1092F10AA8C08091FE199091E5
:10B09000FF19009709F18091FE199091FF198430F2
:10B0A0009105D1F08091CD0A882349F48DEC9AE086
:10B0B00040E45DE063E070E00E9427CB0DC08DECC2
:10B0C0009AE00E9444CB882339F08BED99E10E94ED
:10B0D000D5C784E08093FD198091FD19882399F0EC
:10B0E0008091FD19843029F481E29BE060E070E0FA
:10B0F00004C081E29BE063E070E00E94015C8BEDA4
:10B1000099E10E94E3C78091FE199091FF19843064
:10B11000910509F048C08DEC9AE00E9467CB81E070
:10B120009AE10E9458C88091100B9091110B2091C8
:10B13000140B8630910551F4222341F181E09AE10C
:10B1400069E80E9498C81092140B25C0222371F060
:10B1500081E09AE169E80E9498C81092140B81E29C
:10B160009BE066E070E00E94015C15C08BED99E108
:10B1700061E07AE10E941152882369F48BED99E134
:10B1800061E07AE10E94C656882329F481E09AE1C1
:10B1900065E80E9498C88BED99E10E94E3C787EDAE
:10B1A00099E10E94A8CB8091100B9091110B8230F5
:10B1B000910541F40E94CF76882321F41092110B5F
:10B1C0001092100B8091100B9091110B853091050E
:10B1D00041F40E94D688882321F41092110B10921A
:10B1E000100B2A960FB6F894DEBF0FBECDBFCF91DD
:10B1F000DF911F910F910895CF93DF93FC0182811E
:10B200009381009721F481E0818780E019C08481D7
:10B21000958120813181B9010E948FCCC681D7816F
:10B22000C80FD91F848195810196B9010E948FCCE6
:10B23000958384838281938101979383828388811C
:10B24000DF91CF910895DF92EF92FF920F931F93BA
:10B25000DF93CF93CDB7DEB76F970FB6F894DEBF0D
:10B260000FBECDBF7C018091100B9091110B8130EE
:10B27000910591F1823091051CF4009739F13DC0A0
:10B280008230910521F085309105B9F525C0DD2486
:10B290008E010F5F1F4FC7010E94FC58F801ED0D92
:10B2A000F11D8083D394FE01ED0DF11D8081882373
:10B2B00091F7C80169E772E00E94B0CD0097E9F00C
:10B2C00081EF9AE0B8010E94B9CD17C081E090E00B
:10B2D0009093110B8093100B00E0C7010E94FC5863
:10B2E000E02FF0E0EF50F54F80830F5FE02FF0E0AC
:10B2F000E051F54F8081882381F76F960FB6F8945F
:10B30000DEBF0FBECDBFCF91DF911F910F91FF9098
:10B31000EF90DF90089585E19BE06CE779E140E0F4
:10B320000E94E9C88DEC9AE00E9423CB87ED9AE059
:10B330000E9423CB0895DF93CF930F92CDB7DEB752
:10B34000682FF89484B76623A1F088E10FB6F894CB
:10B3500080936000109260000FBE14BE89E228E165
:10B3600030E00FB6F894A895209360000FBE80934C
:10B37000600069830E9440770E94D9880E944F68CC
:10B380000E94D7670E9429460E94679C0E94F87A13
:10B390000E9452CA81E29BE069810E94F55D789427
:10B3A0000F90CF91DF91089581E00E949B590E94F8
:10B3B000FB7A78940E94F5570E944C4781E29BE00B
:10B3C0000E948D5CA895F6CF8BE19BE06CE779E15C
:10B3D00040E00E94E9C80895CF93DF93EC0186E135
:10B3E00097E099838883FE01EA5AFF4F1082CE01CD
:10B3F000865A9F4F0E9423CBCE018C599F4F0E94AB
:10B400006EC31C82DF91CF910895CF93DF93EC013F
:10B4100002960E9423CBCE010C960E9423CBCE0134
:10B4200046960E9423CBDF91CF910895CF93DF936F
:10B43000EC0124EA37E0FC0121933193CF010E9413
:10B44000D2C1CE010A960E946EC3CE014B960E94D5
:10B4500023CBDF91CF910895CF93DF93EC0180EF61
:10B4600097E099838883CE0105960E944DC4CE0152
:10B470000E960E94165ACE01C9960E94BEC1CE01F8
:10B480008F5B9F4F0E94C8C1DF91CF9108952F928B
:10B490003F924F925F926F927F928F929F92AF9264
:10B4A000BF92CF92DF92EF92FF920F931F93DF93A1
:10B4B000CF93CDB7DEB7C654D0400FB6F894DEBFF9
:10B4C0000FBECDBF4C0104960E9423CBC4010E9643
:10B4D0000E9423CB04E719E17E010894E11CF11CD2
:10B4E000C701B80143E00E94E9C887E0C82ED12C0B
:10B4F000CC0EDD1EC601B80144E00E94E9C88E01F1
:10B50000035F1F4FBEE6AB2EB9E1BB2EC801B501EC
:10B5100043E00E94E9C8C401499660E0A701960192
:10B52000E12CA1E0FA2E0E94AA50F3E1EF2EF12CBB
:10B53000EC0EFD1E08E619E1C701B80145E00E94C6
:10B54000E9C8E9E1CE2ED12CCC0EDD1EC601B80132
:10B5500046E00E94E9C88E01015E1F4FC801B50197
:10B5600044E00E94E9C8C40180559F4F61E0A701F3
:10B5700096017CE1E72E71E0F72E0E94AA5097E435
:10B58000692E91E0792E680C791CC3010E94055A3E
:10B5900087E6482E81E0582E480C591C05E2C02E43
:10B5A000D12CCC0EDD1E1AE6E12E19E1F12EC601DA
:10B5B000B70144E00E94E9C8BBE2AB2EB12CAC0E4F
:10B5C000BD1EC501B70143E00E94E9C88E010F5CB2
:10B5D0001F4FC801B70142E00E94E9C8C201B6018D
:10B5E000A50198010E945AA5A7E3CA2ED12CCC0E22
:10B5F000DD1EC601B70145E00E94E9C88E01035C6B
:10B600001F4FC801B70146E00E94E9C8C4018E5926
:10B610009C4F25969FAF8EAF2597F2EE2F2EF1E02F
:10B620003F2E280C391CF401EB5FFC4F2796FFAF2F
:10B63000EEAF2797C4018D579E4FB301A20196012B
:10B6400071016F012596AEACBFAC25970E940FA289
:10B65000C1010E942EC4C4018E5F9C4F0E941ABB80
:10B6600084ED96E02796EEADFFAD2797918380831A
:10B67000C401895F9C4F0E946EC3C401885E9C4FC9
:10B680000E942C5A25968EAD9FAD25970E94EC59AD
:10B69000840101531C4FC8016FE040E00E94A1C922
:10B6A000A4014F515C4F8CEC95E0FA0191838083AB
:10B6B000C4018D519C4FB80100E513EC20E030E04F
:10B6C000E0E1EE2EE1E0FE2ECC240E946C9EF4011F
:10B6D000EC5BFB4F81E08083CA5BDF4F0FB6F894D1
:10B6E000DEBF0FBECDBFCF91DF911F910F91FF90B5
:10B6F000EF90DF90CF90BF90AF909F908F907F9012
:10B700006F905F904F903F902F9008956FB7F8948F
:10B71000FC0120813181428153816FBFB901CA018F
:10B7200008950E94FE44882311F40E940782089520
:10B73000CF93DF93EC01FC01E45BFB4F71836083EB
:10B7400062307105D9F48D519C4F0E9484A18823E9
:10B75000D1F40E94944F8823B1F0CE01C2960E948A
:10B7600084A18823A1F0CE0187539F4F0E9484A11A
:10B77000882369F008C081E08093700FC75BDB4FBE
:10B7800081E0888304C08091700F8823A1F3DF914A
:10B79000CF910895FC01E25BFB4F808108950E96E6
:10B7A00040E052ED69E47BE60E9427CB08951F92AA
:10B7B0000F920FB60F920BB60F9211242F933F9357
:10B7C0004F935F936F937F938F939F93AF93BF93A9
:10B7D000EF93FF9381E29BE00E94915BFF91EF91D9
:10B7E000BF91AF919F918F917F916F915F914F9199
:10B7F0003F912F910F900BBE0F900FBE0F901F9097
:10B800001895EF92FF920F931F93DF93CF9300D081
:10B8100000D000D0CDB7DEB77B016115710591F482
:10B820001092780F1092770F8E010F5F1F4FC80193
:10B8300068E679E147E00E94E9C8C80160E00E943B
:10B84000F14C0CC08091740F90E08617970731F08F
:10B8500082E090E09093780F8093770FE092740FDE
:10B8600026960FB6F894DEBF0FBECDBFCF91DF9105
:10B870001F910F91FF90EF9008954115510531F4FC
:10B8800010927A0F1092790F81E008C0611571054E
:10B8900041F410927A0F1092790F80E00E94F3A188
:10B8A00008956093750F4093760F81E090E0909338
:10B8B0007A0F8093790F0895CF93DF93EC0169E1BC
:10B8C00070E04FE050E00E943D5CCE018D579E4FEE
:10B8D0006FEF0E940DA5C65BDB4F81E08883DF918F
:10B8E000CF9108950F931F93DF93CF930F92CDB70E
:10B8F000DEB78C018D579E4F49830E94D3A2C801A9
:10B900000E945C5CF801E55BFB4F498140830F902E
:10B91000CF91DF911F910F910895EF92FF920F93B6
:10B920001F93CF93DF938C01FC01808D882339F125
:10B9300023E8E22E21E0F22EE00EF11EC7010E9464
:10B940006FA2E8012496CE010E9444CB8823B9F06F
:10B950008091710F9091720F009789F4C7010E9436
:10B9600070A3C7010E9475A2AB01BC01CE010E9469
:10B9700027CB81E090E09093720F8093710FF801D4
:10B98000EC5BFB4F8081882329F0C8018D519C4FCF
:10B990000E945DA09AE4E92E94E0F92EE00EF11EDB
:10B9A000F7018081882301F1E801CD57DE4FCE01F8
:10B9B0000E9412A58823C1F0C80160E070E040E059
:10B9C00050E00E943D5C0E94C774F7011082CE01D6
:10B9D0000E9432A3F801E55BFB4F8081882311F0C0
:10B9E0000E9435551092730FE8012E96CE010E94E9
:10B9F00044CB882309F457C0F801E75BFB4F8081F3
:10BA0000882309F050C00E94C0548230910509F487
:10BA10004AC00E94C0548130910509F444C0CE014F
:10BA20000E946ACBF801E25BFB4F808180648083D7
:10BA3000E801E296CE010E94709F1816190684F064
:10BA4000C80187539F4F0E94709F1816190644F033
:10BA5000C8018D519C4F0E94709F1816190684F4DE
:10BA6000C8018D579E4F64E872E00E94D3A2C801BE
:10BA70000E945C5C80E060E04FEF21E00E94D9739F
:10BA8000CE0160E070E00E94AC9EC80187539F4FDA
:10BA900060E070E00E94AC9EC8018D519C4F60E058
:10BAA00070E00E94AC9EE801C75BDB4F8881882371
:10BAB00009F470C08091730F882309F06BC00E9455
:10BAC0003761882309F066C081E08093730FC80155
:10BAD0006AE070E04AE050E00E943D5CC801C29616
:10BAE00060E070E00E94AC9EC80187539F4F60E009
:10BAF00070E00E94AC9EC8018D519C4F60E070E0E8
:10BB00000E94AC9EF801E45BFB4F80819181843000
:10BB1000910571F08530910524F48230910541F54D
:10BB20001BC08830910551F08031910509F50EC098
:10BB3000C8018D579E4F6DEA72E005C0C8018D5750
:10BB40009E4F6DEF72E00E94D3A212C0C8018D57C4
:10BB50009E4F6EE473E0F7CFC8018D579E4F6FE99B
:10BB600073E00E94D3A2C8010E945C5C188236C0B8
:10BB70000E94CC730E9466520E94FA440E94D767CA
:10BB8000C0E0D0E08C2F60E00E94BA812196C530E1
:10BB9000D105C1F78091710F9091720F813091059D
:10BBA00019F483E090E009C08330910559F4C8018D
:10BBB00049960E94555182E090E09093720F8093D5
:10BBC000710F0CC08230910549F4C80180559F4F18
:10BBD0000E9455511092720F1092710FDF91CF9108
:10BBE0001F910F91FF90EF900895DF92EF92FF92D7
:10BBF0000F931F93DF93CF93CDB7DEB7E6970FB6C2
:10BC0000F894DEBF0FBECDBF7C01D62E60E070E0A1
:10BC10000E94015C82E090E060E00E94979C082F07
:10BC200087E795E10E94ED78802F8095881F88270F
:10BC3000881F0E94FC7B87ED99E161E00E94C8CBE0
:10BC40008BED99E10E94E3C7D7011D921D921D92D1
:10BC50001C92139721E024BD25BD17BC18BC10927F
:10BC60006E001092900039E0309391001092920093
:10BC700080E090E1909399008093980082E0809317
:10BC800071001092B0009AE09093B1001092B3004E
:10BC90001092B40080937000109220013093210123
:10BCA000109229011092280110922B0110922A0162
:10BCB00010927300209380008BE08093810010929B
:10BCC00089001092880010928B0010928A001092C6
:10BCD0006F002093A0008093A1001092A900109201
:10BCE000A8001092AB001092AA00109272000E945D
:10BCF00096A1F701808F882389F187010D571E4F88
:10BD0000C8010E94F1A286E591E060E00E94979C44
:10BD1000882321F4B701685E7C4F03C0B7016E5FD2
:10BD20007C4FC8010E948BA2DD2049F08FEF9BE77A
:10BD3000A2E981509040A040E1F700C00000B701A7
:10BD400069597E4FC8010E94DBA1C8010E9475A2FB
:10BD5000AB01BC01C70104960E9427CBC70160E07C
:10BD600070E040E050E00E943D5CDD2009F47EC0C0
:10BD70008E010F5F1F4FC80168E679E147E00E941E
:10BD8000E9C8C80161E00E941EC98E01095F1F4F0A
:10BD9000C8016AE679E141E00E94E9C8C80161E0B2
:10BDA0000E941EC98E01035F1F4FC8016AE679E138
:10BDB00040E00E94E9C8C80161E00E941EC98E01EE
:10BDC0000D5E1F4FC80162E779E141E00E94E9C8BA
:10BDD000C80161E00E941EC98E01075E1F4FC801A5
:10BDE00068E679E147E00E94E9C8C80161E00E9485
:10BDF0001EC98E01015E1F4FC80162E779E140E074
:10BE00000E94E9C8C80161E00E941EC98E010B5D55
:10BE10001F4FC80168E779E146E00E94E9C8C80100
:10BE200061E00E941EC98E01055D1F4FC80168E7D1
:10BE300079E145E00E94E9C8C80161E00E941EC99D
:10BE40000E9458750E949462F701E75BFB4F1082D5
:10BE5000F701E45BFB4F11821082C7018B5B9B4FA4
:10BE60000E94B14DF701E25BFB4F1082C70149967A
:10BE70000E943451C70180559F4F0E9434518E015A
:10BE80000F5C1F4FC8016AE779E144E00E94E9C8EE
:10BE9000C80161E00E941EC9C70181539C4F0E94E6
:10BEA0009AC987010D511C4FC8010E94729DC7019C
:10BEB000C29660E070E00E94AC9EC70187539F4F1E
:10BEC00060E070E00E94AC9EC80160E070E00E94FB
:10BED000AC9E0E94C774F701E65BFB4F1082E696AA
:10BEE0000FB6F894DEBF0FBECDBFCF91DF911F918B
:10BEF0000F91FF90EF90DF9008951F920F920FB671
:10BF00000F920BB60F9211240F931F932F933F9311
:10BF10004F935F936F937F938F939F93AF93BF9351
:10BF2000EF93FF93DF93CF93CDB7DEB76297DEBF7A
:10BF3000CDBF8091210B9091220BA091230BB0914A
:10BF4000240B80589F4FAF4FBF4F8093210B90938E
:10BF5000220BA093230BB093240B8091810F90911F
:10BF6000820F9C012F5F3F4F3093820F2093810FF0
:10BF70008138910508F4B3C01092820F1092810F9E
:10BF800080917B0F90917C0F1816190614F401977D
:10BF90003DC08091770F9091780F8130910509F520
:10BFA00080917D0F90917E0F019690937E0F8093EC
:10BFB0007D0F82E090E09093780F8093770F82E17D
:10BFC00090E090937C0F80937B0F8E010F5F1F4F4B
:10BFD000C80168E679E147E00E94E9C8C80160E06D
:10BFE00048C08230910539F58091740F90E020911E
:10BFF0007D0F30917E0F281739076CF083E090E0B9
:10C000009093780F8093770F80E590E090937C0F6A
:10C0100080937B0F30C081E090E09093780F809305
:10C02000770F82E190E090937C0F80937B0F8E01DD
:10C03000095F1F4F16C083309105E9F410927E0FFF
:10C0400010927D0F81E090E09093780F8093770FAE
:10C0500082E190E090937C0F80937B0F8E01035FD1
:10C060001F4FC80168E679E147E00E94E9C8C801AE
:10C0700061E00E94F14C80917F0F9091800F181623
:10C08000190634F401979093800F80937F0F27C097
:10C090008091790F90917A0F8130910571F482E04F
:10C0A00090E090937A0F8093790F8091750F809331
:10C0B0007F0F1092800F81E010C08230910579F4DB
:10C0C00081E090E090937A0F8093790F8091760FC2
:10C0D00080937F0F1092800F80E00E94F3A1629600
:10C0E000DEBFCDBFCF91DF91FF91EF91BF91AF91B7
:10C0F0009F918F917F916F915F914F913F912F9180
:10C100001F910F910F900BBE0F900FBE0F901F90BD
:10C1100018951F920F920FB60F920BB60F92112423
:10C120002F933F934F935F936F937F938F939F933F
:10C13000AF93BF93EF93FF930E94DF62FF91EF9164
:10C14000BF91AF919F918F917F916F915F914F912F
:10C150003F912F910F900BBE0F900FBE0F901F902D
:10C160001895882321F080912001806203C080917E
:10C1700020018F7C8093200108950F931F93DF93FC
:10C18000CF9300D000D000D0CDB7DEB7062F1FB7B9
:10C19000F89480E00E94B160CE0101966AE779E1EF
:10C1A00044E00E94E9C861E0002309F460E0CE01A8
:10C1B00001960E94F14C1FBF26960FB6F894DEBF81
:10C1C0000FBECDBFCF91DF911F910F910895FC015C
:10C1D000EC5BFB4F60830895CF92DF92EF92FF926A
:10C1E0000F931F93DF93CF93CDB7DEB72C970FB686
:10C1F000F894DEBF0FBECDBFC62EDFB6F8943AE787
:10C20000E32E39E1F32E8E010F5F1F4FC801B701F6
:10C2100045E00E94E9C8C80161E00E941EC98E0184
:10C22000095F1F4FC801B70145E00E94E9C8C80176
:10C230006C2D0E94F14CDFBE2C960FB6F894DEBF39
:10C240000FBECDBFCF91DF911F910F91FF90EF9067
:10C25000DF90CF90089583E89FE06CE779E140E0BC
:10C260000E94E9C881E29BE00E94475A08958091AC
:10C270009A0F0895FC019B018281938160817181F5
:10C2800086179707B8F44281538184819581840F82
:10C29000951F0E948FCC880F991FA681B781A80F88
:10C2A000B91F11963C932E938281938101969383BB
:10C2B0008283089581E080870895CF93DF939C0166
:10C2C000EB018091FA0F9091FB0F4091F80F509184
:10C2D000F90F4817590751F088EF9FE0B9010E9404
:10C2E0003A6182E090E1BE010E943A61DF91CF9114
:10C2F00008950F931F93CF93DF93EC018B018091EF
:10C30000990F882321F0CE010E945D61ACC08AE4C0
:10C3100091E061E00E94979C882309F4A4C081E029
:10C3200080939A0F8093990F89E89FE060E00E94C4
:10C33000F14C89E89FE061E00E941EC99E0140E047
:10C3400050E060E072E18AE790E00E94B6CCDA014A
:10C35000C901B695A795979587950197A109B10948
:10C3600080939F0F9093A00FA093A10FB093A20F63
:10C370008F3F9105A105B10509F008F444C0DA0129
:10C38000C901F4E0B695A79597958795FA95D1F7E9
:10C390000197A109B1098F3F9105A105B105A9F147
:10C3A000A0F1DA01C901E7E0B695A79597958795C1
:10C3B000EA95D1F70197A109B1098F3F9105A10530
:10C3C000B10529F120F1DA01C90179E0B695A79507
:10C3D000979587957A95D1F70197A109B1098F3F74
:10C3E0009105A105B105A9F0A0F0DA01C9016BE042
:10C3F000B695A795979587956A95D1F70197A10965
:10C40000B10925E007C021E005C022E003C023E018
:10C4100001C024E0285F25BD87BD88BD82E08093F0
:10C420006E00BE0180E090E0660F771F881F991FA5
:10C43000980140E050E00E9470CC28EE33E040E0EC
:10C4400050E00E94D8CC20939B0F30939C0F4093D8
:10C450009D0F50939E0F1092A30F1092A40F109255
:10C46000A50F1092A60FDF91CF911F910F91089504
:10C470000F931F93CF93DF9300E010E0C82FD0E01D
:10C480000EC08EEE91E06CE271E00E94796188EB63
:10C4900091E06CE271E00E9479610F5F1F4F0C1711
:10C4A0001D077CF3DF91CF911F910F91089580E7D5
:10C4B00093E06CEB70E00E94796180E090E06CEBBF
:10C4C00070E00E94796180EE96E06CEB70E00E9473
:10C4D000796180E090E06CEB70E00E94796188EB1C
:10C4E00097E06CEB70E00E94796180E090E06CEB8B
:10C4F00070E00E9479618DE298E06CEB70E00E9440
:10C50000796189EA98E06CEB70E00E94796180E0E3
:10C5100090E06CEB70E00E94796180EC9DE06DE44E
:10C5200071E00E947961089580EC9DE060E271E025
:10C530000E94796180E090E06CEB70E00E9479618C
:10C5400083E591E16CEB70E00E94796180E090E01E
:10C550006CEB70E00E9479618BE592E161EB71E038
:10C560000E9479610895CF93DF93FC0182819381CA
:10C57000009729F481E0818720E030E01CC08481AD
:10C58000958120813181B9010E948FCC880F991F3C
:10C59000C681D781C80FD91F848195810196B901C1
:10C5A0000E948FCC958384838281938101979383AA
:10C5B000828328813981C901DF91CF910895CF937A
:10C5C000DF9380919B0F90919C0FA0919D0FB09154
:10C5D0009E0F0097A105B10511F16091A70F81E0B1
:10C5E00068276093A70F89E89FE00E94F14C809133
:10C5F0009B0F90919C0FA0919D0FB0919E0F009763
:10C60000A105B10569F10197A109B10980939B0FBB
:10C6100090939C0FA0939D0FB0939E0F21C01092FA
:10C620006E0018BC17BC89E89FE060E00E94F14CE6
:10C630001092990F8091FA0F9091FB0F009771F073
:10C6400088EF9FE00E94B362EC0182E090E10E94DB
:10C65000B362BC01CE010E94796102C010929A0FB0
:10C66000DF91CF9108958CE090E16CE779E140E0B3
:10C670000E94E9C889E89FE062E779E145E00E940D
:10C68000E9C88FE89FE00E9423CB84E190E090937B
:10C69000F90F8093F80F1092FB0F1092FA0F10927F
:10C6A000FD0F1092FC0F28EA3FE03093FF0F20931C
:10C6B000FE0F1092001010920110909303108093BF
:10C6C0000210109205101092041010920710109290
:10C6D000061080ED9FE0909309108093081010924F
:10C6E0000A1010920B1008958F929F92AF92BF92F2
:10C6F000CF92DF92EF92FF920F931F93CF93DF932E
:10C70000EC016B01009709F46BC0FC01EA5BFF4F81
:10C71000808182FD65C0EAA0FBA00CA11DA1FB01E8
:10C72000B2A0A3A094A085A0C801B701D501F401CF
:10C730002B2F3A2F4F2F5E2F0E944D4018160CF4CE
:10C740004FC0C801B701A80197010E94B53D7B0108
:10C750008C012EA53FA548A959A95058CA01B90175
:10C760000E94573D2AA53BA54CA55DA50E94B53D5D
:10C770009B01AC01C801B7010E94843D0E9446CED6
:10C780008B017C01A5019401652F742F832F922FBB
:10C79000202F312F4E2D5F2D0E941D4087FF04C09A
:10C7A0000B2D1A2DE92CF82CA5019401652F7A2D5B
:10C7B000832F982D202F312F4E2D5F2D0E948D3FDE
:10C7C000882371F0802F912FAE2DBF2DF60182A30B
:10C7D00093A3A4A3B5A3EA5BFF4F8081826080830B
:10C7E000DF91CF911F910F91FF90EF90DF90CF904D
:10C7F000BF90AF909F908F90089580939405089577
:10C80000453010F550E0222381F024E130E0429FD2
:10C81000F001439FF00D529FF00D1124EE5EFF4E8C
:10C820006483758386839783089524E130E0429F73
:10C83000F001439FF00D529FF00D1124EE5EFF4E6C
:10C8400060877187828793870895CF93DF93453000
:10C85000D0F450E024E130E0429FE001439FD00D4E
:10C86000529FD00D1124CE5EDF4E0E947D40288164
:10C8700039814A815B810E94B53D0E94E13B6C8712
:10C880007D878E879F87DF91CF9108952F923F926A
:10C890004F925F926F927F928F929F92AF92BF92D0
:10C8A000CF92DF92EF92FF920F931F93DF93CF937C
:10C8B000CDB7DEB72E970FB6F894DEBF0FBECDBF53
:10C8C0009E878D871B01DC015E96AD90BD90CD905B
:10C8D000DC909197D696ED90FD900D911C91D99793
:10C8E000C801B7010E942F413B014C01ED85FE8537
:10C8F00062A173A184A195A1A60195010E94AF3EFA
:10C900009B01AC01C401B3010E94B53D0E94E8CD7A
:10C910000E94E13B262F372F482F592F29833A8336
:10C920004B835C83D1016D917D918D919C91A6018A
:10C9300095010E94AF3E9B01AC01C401B3010E946E
:10C94000B53D0E94E8CD0E94E13B9B01AC0119017D
:10C950002A0189819A81AB81BC8188379105A10523
:10C96000B10540F488E790E0A0E0B0E089839A83C5
:10C97000AB83BC83283731054105510528F438E7DE
:10C98000232E312C412C512C69817A818B819C8101
:10C990009B01AC010E9470CC6D837E838F8398874E
:10C9A000C201B101A20191010E9470CC69877A870E
:10C9B0008B879C87C801B701A80197010E9470CCA2
:10C9C0003B014C01ED85FE85EE5BFF4FE080F18081
:10C9D00002811381EE0CFF1C001F111FE114F104F2
:10C9E0000105110579F02D813E814F815885621B2B
:10C9F000730B840B950BA80197010E94D8CC5901A9
:10CA00006A0103C0AA24BB24650122273327A90198
:10CA10002E193F09400B510B59F069857A858B859A
:10CA20009C8566197709880999090E94D8CC03C0AA
:10CA300020E030E0A901AD85BE8554968D919C9192
:10CA400055973C0188249924D401C3018A199B0974
:10CA5000AC09BD09821B930BA40BB50BB7FF3AC001
:10CA600057016801AA0CBB1CCC1CDD1CA114B1042D
:10CA7000C104D104D9F0C801B701A40193010E94F7
:10CA800070CC2D813E814F815885621B730B840BC6
:10CA9000950B29853A854B855C85620F731F841F32
:10CAA000951FA60195010E94D8CC03C020E030E07C
:10CAB000A90159016A0157FF03C0AA24BB246501DB
:10CAC0006A147B048C049D0414F46401530180E017
:10CAD00090E0DC014FB7F8949501ED85FE85B78AAB
:10CAE000A68A280F391F318F208F89819A81AB81C7
:10CAF000BC8182AF93AFA4AFB5AFFE9620823182E6
:10CB0000428253824FBF81E02E960FB6F894DEBF6B
:10CB10000FBECDBFCF91DF911F910F91FF90EF908E
:10CB2000DF90CF90BF90AF909F908F907F906F904D
:10CB30005F904F903F902F9008954F925F926F9229
:10CB40007F928F929F92AF92BF92CF92DF92EF929D
:10CB5000FF920F931F93CF93DF9380911A159091BB
:10CB60001B1550901C1580901D15850D891B882163
:10CB7000823008F487C010911A1560901E157090CD
:10CB80001F1587E4189F70011124E60CF71C5A94B6
:10CB900042E0442E01C07E01150D182187E4189F44
:10CBA000E0011124C60DD71D209709F466C00EA11F
:10CBB000BFA0A8A499A46AA17BA18CA19DA1202FAC
:10CBC0003B2D4A2D592D0E948D3F882309F455C0D5
:10CBD000FE01EA5BFF4F8081882309F04EC0F70118
:10CBE000C2A0D3A0E4A0F5A0602F7B2D8A2D992DA3
:10CBF000A70196010E94ED3F87FD33C0C701B60132
:10CC0000A70196010E94B53D6B017C012EA53FA5B1
:10CC100048A959A95058CA01B9010E94573D2AA5EF
:10CC20003BA54CA55DA50E94B53D9B01AC01C7018C
:10CC3000B6010E94843D0E9446CEE62EC72EF82EF5
:10CC4000D92E602F7B2D8A2D992D2E2D3C2D4F2DE9
:10CC50005D2D0E941D4087FD04C00E2DBC2CAF2C05
:10CC60009D2C802F9B2DAA2DB92D8AA39BA3ACA30D
:10CC7000BDA3FE01EA5BFF4F408280911B15181790
:10CC800009F089CFDF91CF911F910F91FF90EF9025
:10CC9000DF90CF90BF90AF909F908F907F906F90DC
:10CCA0005F904F900895CF92DF92FF920F931F9362
:10CCB000DF93CF930F92CDB7DEB7F0901B15CC2446
:10CCC000DD2480E090E047E415C05F2D549F900183
:10CCD000112400911E1510911F15020F131FB6018C
:10CCE00049830E947463F39480911D15F822C60154
:10CCF0006801498120911A15F21639F7B6010E9490
:10CD000074630F90CF91DF911F910F91FF90DF908F
:10CD1000CF900895CF92DF92FF920F931F93DF93EE
:10CD2000CF930F92CDB7DEB7F0901B15CC24DD2446
:10CD300027E42EC03F2D329FC001112400911E1503
:10CD400010911F15080F191FC114D104E1F0F6014D
:10CD5000EA5BFF4F808181FD08C0F801EA5BFF4F6D
:10CD6000908191FF10C080FD0EC0B8016E5D7F4FB5
:10CD7000C60129830E944664F601EA5BFF4F808169
:10CD80008D7F80832981F39480911D15F82268019D
:10CD900080911A154F2D552747FD509590E0481763
:10CDA000590741F6B6016E5C7F4FC6010E9446648A
:10CDB000F601EA5BFF4F80818D7F808381E00F90D9
:10CDC000CF91DF911F910F91FF90DF90CF90089549
:10CDD0000E949D650E9453660E948A660895909104
:10CDE0001A1520911B159F5F80911D15982381E0D6
:10CDF000921380E0089520911A1590911B1581E0FF
:10CE0000291380E0089580914E15882349F42091DC
:10CE10001A1590911B1581E0291719F480E00895E7
:10CE200080E0089590911B1587E4989FC00111241C
:10CE300020911E1530911F15280F391FC901089523
:10CE400080911B158F5F90911D15892380931B1571
:10CE500008952F923F924F925F926F927F928F929E
:10CE60009F92AF92BF92CF92DF92EF92FF920F9379
:10CE70001F93DF93CF9300D00F92CDB7DEB7CFB61D
:10CE8000C982F89472E6C72E71E0D72E1B821A82EF
:10CE90006AE0862E912CA12CB12C52E0452E512C0B
:10CEA000612C712CC60140E050E0BA010E94D19C77
:10CEB0007B018C0180E295E16A817B810E94FA719D
:10CEC0001C01C801B701A50194010E94D8CCCA0178
:10CED000B901A30192010E94D8CCF10120833183D2
:10CEE000428353832A813B812F5F3F4F3B832A83B9
:10CEF00084E090E0C80ED91E2330310599F602E097
:10CF000010E080E295E1B8010E94FA71FC01108204
:10CF10001182128213820F5F1F4F0530110589F7AE
:10CF200000E010E084E395E1B8010E94FA717C0111
:10CF300080E295E1B8010E94FA71FC018081918143
:10CF4000A281B381B095A095909581959F4FAF4FE9
:10CF5000BF4FF70180839183A283B3830F5F1F4F7D
:10CF600005301105F9F6F981FFBF0F900F900F9072
:10CF7000CF91DF911F910F91FF90EF90DF90CF90B5
:10CF8000BF90AF909F908F907F906F905F904F90E9
:10CF90003F902F900895813019F484E395E102C009
:10CFA00080E295E1909349158093481508950F9379
:10CFB0001F93DF93CF93CDB7DEB764970FB6F89486
:10CFC000DEBF0FBECDBF0E944A7B8E010F5F1F4F99
:10CFD000C8010E94AA7BAEE7B0E1F80184E10190AC
:10CFE0000D928150E1F70E94296780E00E94CB6793
:10CFF00080E090E0DC018093921090939310A093D6
:10D000009410B09395108093961090939710A093DE
:10D010009810B093991080939A1090939B10A093BE
:10D020009C10B0939D1080939E1090939F10A0939E
:10D03000A010B093A1108093A2109093A310A0937E
:10D04000A410B093A5108093A6109093A710A0935E
:10D05000A810B093A91010921A1510921B158EE605
:10D0600091E061E00E94979C91E0882309F490E0B0
:10D070009093940510924A1510924B1510924C15EE
:10D0800010924D1510924E1564960FB6F894DEBFAF
:10D090000FBECDBFCF91DF911F910F91089582E612
:10D0A00091E04FEF5FEF6FEF7FEF0E94D19C6F3FFA
:10D0B0002FEF72072FEF82072FEF920711F40E94D4
:10D0C0006C5087E897E4ACEBB2E480931210909335
:10D0D0001310A0931410B093151080932610909302
:10D0E0002710A0932810B093291080E090E0A8ECBE
:10D0F000B3E480933A1090933B10A0933C10B0930C
:10D100003D1087EE9CE8A0ECB2E480934E10909323
:10D110004F10A0935010B0935110809362109093D1
:10D120006310A0936410B093651088E891E06FEFEE
:10D130000E94979C803811F00E943F4F80E791E059
:10D1400068EB7BE00E94B09CBC0180E090E00E9414
:10D150007D40609376107093771080937810909351
:10D16000791082E791E068EB7BE00E94B09CBC0103
:10D1700080E090E040E00E94256484E791E068EB65
:10D180007BE00E94B09CBC0180E090E041E00E9406
:10D19000256486E791E068EE73E00E94B09CBC01D4
:10D1A00080E090E042E00E94256488E791E068EB2F
:10D1B0007BE00E94B09CBC0180E090E043E00E94D4
:10D1C00025648AE791E068EB7BE00E94B09CBC019B
:10D1D00080E090E044E00E9425648CE791E040E02C
:10D1E00050E060EA71E40E94F29C609355157093E0
:10D1F0005615809357159093581580E891E040E0BC
:10D2000050E060E87FE30E94F29C60934A107093C4
:10D210004B1080934C1090934D1082E891E040E0C9
:10D2200050E060E771E40E94F29C60935E1070939E
:10D230005F10809360109093611084E891E040E06B
:10D2400050E060E771E40E94F29C6093721070936A
:10D250007310809374109093751086E891E06FE0DE
:10D2600070E00E94B09CBC0180E090E00E942F41E1
:10D2700060937A1070937B1080937C1090937D1054
:10D2800084E991E040E65AEE60E070E00E94D19CB3
:10D2900042E021E00E94006460E070E0CB0142E0E7
:10D2A00020E00E9400640E94D7670895AEE7B0E1D5
:10D2B000282F392FF90124E101900D922150E1F737
:10D2C0000E94867B80E090E0DC0180939210909336
:10D2D0009310A0939410B093951080939610909310
:10D2E0009710A0939810B093991080939A109093F0
:10D2F0009B10A0939C10B0939D1080939E109093D0
:10D300009F10A093A010B093A1108093A2109093AF
:10D31000A310A093A410B093A5108093A61090938F
:10D32000A710A093A810B093A9100895282F392F03
:10D33000D901EEE7F0E124E101900D922150E1F7EF
:10D340000895CF92DF92EF92FF920F931F93DF9396
:10D35000CF93CDB7DEB7C954D0400FB6F894DEBF37
:10D360000FBECDBF8C01FC0110821182628361501F
:10D3700063835583448320E037E46E010894C11C25
:10D38000D11C1FC0239FC0011124F801E480F58047
:10D39000E80EF91EC60129962FAF29972A963FAFAE
:10D3A0002A970E949B71D701F60187E42A963FAD28
:10D3B0002A9729962FAD299701900D928150E1F778
:10D3C0002F5FF80182812817E8F2C75BDF4F0FB6A5
:10D3D000F894DEBF0FBECDBFCF91DF911F910F91AB
:10D3E000FF90EF90DF90CF900895EF92FF920F9310
:10D3F0001F937B018C0120E030E0A9010E94BD3F1A
:10D40000181624F017FB109517F910956E2D7F2D27
:10D41000802F912F1F910F91FF90EF9008952F92E1
:10D420003F924F925F926F927F928F929F92AF92B4
:10D43000BF92CF92DF92EF92FF920F931F93DF93F1
:10D44000CF93CDB7DEB7CE54D0400FB6F894DEBF41
:10D450000FBECDBF8BAB9CAB4DAB59AF6AAF7BAFB3
:10D46000290190911A1587E4989FC0011124009119
:10D470001E1510911F15080F191FF801EA5BFF4FC9
:10D480001082F8013BA92CA9832F922FDC0184E1A3
:10D490000D9001928150E1F7C20160E070E00E94BE
:10D4A000F271DC01CD90DD90ED90FC901397F7FECA
:10D4B00008C0F094E094D094C094C11CD11CE11C2D
:10D4C000F11CC20160E070E00E94F271FC01608119
:10D4D0007181828193810E947D4020911210309150
:10D4E000131040911410509115100E94AF3E762EEB
:10D4F00079A78DA799AB472F382F292F862F942FE7
:10D50000A32FB22F89839A83AB83BC83C20161E0CE
:10D5100070E00E94F271DC018D909D90AD90BC9006
:10D520001397B7FE08C0B094A09490948094811C87
:10D53000911CA11CB11C8C149D04AE04BF0414F4F6
:10D5400046015701C20161E070E00E94F271FC01E6
:10D5500060817181828193810E947D40209126109B
:10D560003091271040912810509129100E94AF3E11
:10D57000662E272E382E9AAB292F862F922DA32D7B
:10D58000B22F8D839E83AF83B887C20162E070E0C3
:10D590000E94F271FC0180819181A281B381B7FF69
:10D5A00007C0B095A095909581959F4FAF4FBF4F05
:10D5B00088169906AA06BB0614F44C015D01C20147
:10D5C00062E070E00E94F271DC016D917D918D91BD
:10D5D0009C910E947D4020913A1030913B104091E7
:10D5E0003C1050913D100E94AF3EF62EE72ED82EF3
:10D5F000C92EA7019601852F942FA32FB22F8987BB
:10D600009A87AB87BC8781149104A104B10409F403
:10D6100046C049A53DA529A9672D742F832F922FB8
:10D62000F901272D342F4F2F5E2F0E94B53D69A79A
:10D630007AA78BA79CA72AA9662D722D832D922FDE
:10D64000262D322D432D592F0E94B53D9B01AC0153
:10D6500069A57AA58BA59CA50E94573D69A77AA7C5
:10D660008BA79CA7A7019601652F742F832F922F5C
:10D67000D701F6012B2F3A2F4F2F5E2F0E94B53D79
:10D680009B01AC0169A57AA58BA59CA50E94573D7D
:10D690000E9446CE6DA77EA78FA798AB07C020E05B
:10D6A00030E0A9012DA73EA74FA758ABC20163E008
:10D6B00070E00E94F271DC01CD90DD90ED90FC9065
:10D6C0001397F7FE08C0F094E094D094C094C11C66
:10D6D000D11CE11CF11CC814D904EA04FB0414F4A5
:10D6E00075016401C20163E070E00E94F271FC0107
:10D6F00060817181828193810E947D4020914E10D2
:10D7000030914F1040915010509151100E94AF3EF7
:10D71000B62EA72E882E792EA501852F942FA82D01
:10D72000B72D8D879E87AF87B88B6DA57EA58FA5FA
:10D7300098A920E030E0A9010E945D3F882359F4B8
:10D74000A501652F742F882D972D0E94F5696DA76F
:10D750007EA78FA798ABC20164E070E00E94F271CF
:10D76000FC0180819181A281B381B7FF07C0B09590
:10D77000A095909581959F4FAF4FBF4FC9A6DAA650
:10D78000EBA6FCA6C816D906EA06FB0624F489A770
:10D790009AA7ABA7BCA7C20164E070E00E94F27137
:10D7A000DC016D917D918D919C910E947D40209135
:10D7B00062103091631040916410509165100E9486
:10D7C000AF3E7B01D82EC92E9601862F9F2DA32F09
:10D7D000B22F898B9A8BAB8BBC8B6DA57EA58FA549
:10D7E00098A920E030E0A9010E945D3F882359F408
:10D7F00096016E2D7F2D832F922F0E94F5696DA7C4
:10D800007EA78FA798AB29A53AA54BA55CA52115A6
:10D8100031054105510509F493C32DA939AD4AAD30
:10D820005BADF22EE32ED42EC52E80919405882375
:10D83000A9F5F8017BA96CA9872F962FDC0184E15B
:10D840000D9001928150E1F760E472E48FE090E086
:10D850000E94B6CCD801D6962D933D934D935C9300
:10D86000D99757961C921E925697E9A5FAA55596F8
:10D87000FC93EE9354975996FC93EE9358975A96CF
:10D880001D921D921D921C925D9780911A158F5FBB
:10D8900090911D15892380931A154EC30E94CF764F
:10D8A000882301F569A57AA58BA59CA52F2D3E2D72
:10D8B0004D2D5C2D0E9470CC6031B7E27B07B0E04B
:10D8C0008B07B0E09B0770F460E177E280E090E0C6
:10D8D00029A53AA54BA55CA50E94B6CCF22EE32E55
:10D8E000D42EC52E6F2D7E2D8D2D9C2D29A53AA5CC
:10D8F0004BA55CA50E9470CC0E942F419B01AC01FE
:10D9000060E074E284E799E40E94AF3E862E772EB1
:10D91000682E392E69A57AA58BA59CA50E942F415A
:10D920006DAB7EAB8FAB98AF60E070E080E89FE3BB
:10D930002DA53EA54FA558A90E94AF3E9B01AC0165
:10D940006DA97EA98FA998AD0E94B53D262E79AF0D
:10D950008AAF9BAF6DA57EA58FA598A9282D372DE1
:10D96000462D532D0E94B53D69AB7AAB8BAB9CAB7A
:10D9700060E472E48FE090E02F2D3E2D4D2D5C2D64
:10D980000E94B6CCF80126AB37AB40AF51AF7E0159
:10D990000894E11CF11CA5E1CA2ED12CCC0EDD1E91
:10D9A0005601D7016D917D918D919D917D01E82D5D
:10D9B000F72DA62DB32D9F01AD010E94B53DF601B7
:10D9C00061937193819391936F01EA14FB0449F77A
:10D9D00049AD3AAD2BAD622D742F832F922F20913C
:10D9E00076103091771040917810509179100E9404
:10D9F000B53D0E94E8CD0E94E13B382F25966FAFE0
:10DA0000259726967FAF26978CAF27969FAF2797AF
:10DA1000FEE1CF2EF0E1DF2EEE24FF24C8018601C7
:10DA2000332E6C01C201B7010E94F2715C01D80172
:10DA30006D907D908D909C9025966FAD2597269644
:10DA40007FAD2697832D27969FAD27970E942F4164
:10DA50006CAF7DAF8EAF9FAFF50160817181828128
:10DA6000938197FF07C090958095709561957F4F42
:10DA70008F4F9F4F0E947D402DA93EA94FA958ADC1
:10DA80000E94AF3E9B01AC016CAD7DAD8EAD9FADF4
:10DA90000E94B53D0E94E13B66167706880699060E
:10DAA00050F425966FAE259726967FAE2697382C94
:10DAB00027969FAE27970894E11CF11C0C5E1F4F20
:10DAC000F5E0EF16F10409F0ADCF86013CAE2596E6
:10DAD0006FAD259726967FAD2697832D27969FAD10
:10DAE00027970E942F41A9ADFAADEBAD222D3A2F19
:10DAF0004F2F5E2F0E94AF3E262F372F482F592FD2
:10DB00002F962CAF3DAF4EAF5FAF2F97D6019E96AD
:10DB10002D933D934D935C93D19725966FAD2597AB
:10DB200026967FAD2697832D27969FAD279722E4D3
:10DB30003FE040E050E00E94B6CCF601228F338FE8
:10DB4000448F558FF0917A10FDAB20917B1029AF57
:10DB500030917C103AAF40917D104BAF422F2BADEE
:10DB60006F2F742F832F922FB9A9AAA9FBA9ECA913
:10DB70002B2F3A2F4F2F5E2F0E941D4087FF05C08D
:10DB8000FDA8E9ACDAACCBAC04C0F9A8EAA8DBA8E4
:10DB9000CCA890911A1580911B15981709F4FCC018
:10DBA0006091A6107091A7108091A8109091A91073
:10DBB00020E030E0A9010E94BD3F18160CF0ECC037
:10DBC0008091921090919310A0919410B091951023
:10DBD00024968CAF9DAFAEAFBFAF24976D897E8981
:10DBE0008F89988D24962CAD3DAD4EAD5FAD2497B9
:10DBF0000E94843D9B01AC010E94B53DB62EA72E2C
:10DC0000382E292E2091961030919710409198101F
:10DC1000509199102B962CAF3DAF4EAF5FAF2B9725
:10DC2000698D7A8D8B8D9C8D0E94843D9B01AC010A
:10DC30000E94B53D462E672E782E892EB501C10172
:10DC4000272F362F492F582FCA01B901242D362DE1
:10DC5000472D582D0E94573D0E9446CE2B013C0176
:10DC600024966CAD7DAD8EAD9FAD249720E030E065
:10DC7000A9010E948D3F882369F42B966CAD7DAD80
:10DC80008EAD9FAD2B9720E030E0A9010E948D3F23
:10DC9000882321F0F9A8EAA8DBA8CCA88090551524
:10DCA00090905615A0905715B0905815C301B20129
:10DCB000A50194010E94BD3F1816A4F4C501B4014A
:10DCC000A30192010E94AF3E9B01AC01D701F60176
:10DCD0006B2F7E2D8F2F9C2D0E94B53DF62EE72EAB
:10DCE000D82EC92EEAE92E2EE0E13E2EAE01435E8B
:10DCF0005F4F29965FAF4EAF29978AE490E1229655
:10DD00009FAF8EAF2297D1016D917D918D919D91A5
:10DD10001D012996EEADFFAD2997219131914191D9
:10DD200051912996FFAFEEAF29970E94843D0E9442
:10DD3000F5692B013C012296AEADBFAD22978D90C7
:10DD40009D90AD90BC90A50194010E94BD3F181616
:10DD5000A4F4C501B401A30192010E94AF3E9B014E
:10DD6000AC01D701F6016B2F7E2D8F2F9C2D0E94C9
:10DD7000B53DF62EE72ED82EC92E2296EEADFFAD7C
:10DD8000229774962296FFAFEEAF2297F6EA2F16EF
:10DD9000F0E13F0609F0B7CFA7019601852F9E2D30
:10DDA000A32FBC2DF80186A397A3A0A7B1A75DA9B7
:10DDB00049AD3AAD2BAD652F742F832F922FDA0129
:10DDC000F9012B2F3A2F4F2F5E2F0E94B53D4B01AB
:10DDD0005C012F962CAD3DAD4EAD5FAD2F975058E9
:10DDE000CA01B9010E94573D2DA53EA54FA558A9CE
:10DDF0000E94B53D9B01AC01C501B4010E94843D68
:10DE00000E9446CE862EB72EA82E492EA701960137
:10DE1000652F7E2D832F9C2D282D3B2D4A2D542D93
:10DE20000E941D4087FD04C0F82CEB2CDA2CC42C7A
:10DE3000A7019601852F9E2DA32FBC2DF80182A34B
:10DE400093A3A4A3B5A359A94AA93BA92CA9652FBB
:10DE5000742F832F922F282D3B2D4A2D542D0E9455
:10DE60004D40F801EA5BFF4F18161CF0808184607A
:10DE700002C080818B7F8083F801EA5BFF4F808145
:10DE800082608083A2E9B0E1FE01759684E1019091
:10DE90000D928150E1F759A94AA93BA92CA9852FD8
:10DEA000942FA32FB22F8093A6109093A710A09326
:10DEB000A810B093A9102DA53EA54FA558A9D8012B
:10DEC0009A962D933D934D935C939D97E9A5FAA562
:10DED0005596FC93EE9354973BA92CA9A32FB22FF0
:10DEE000F801868F978FA0A3B1A3EE5BFF4F259615
:10DEF0002FAD2597208326963FAD269731834CADD5
:10DF0000428327965FAD279753835DA949AD3AAD0C
:10DF10002BAD852F942FA32FB22FF80182AB93AB9B
:10DF2000A4ABB5AB80911A158F5F90911D15892315
:10DF300080931A150E94E8660E94FF8181E001C06B
:10DF400080E0C25BDF4F0FB6F894DEBF0FBECDBFDF
:10DF5000CF91DF911F910F91FF90EF90DF90CF90C5
:10DF6000BF90AF909F908F907F906F905F904F90F9
:10DF70003F902F9008958F929F92AF92BF92CF9231
:10DF8000DF92EF92FF920F931F93DF93CF93CDB762
:10DF9000DEB7A8970FB6F894DEBF0FBECDBF982EA0
:10DFA000892E7B0140914815509149158E010F5FD4
:10DFB0001F4FC801692D782D0E949672C80162E03A
:10DFC00070E00E94FA71FC0120813181428153810D
:10DFD00080913E1090913F10A0914010B09141105F
:10DFE00082179307A407B50794F4C80162E070E0B4
:10DFF0000E94FA7120913E1030913F1040914010E4
:10E0000050914110FC012083318342835383F701F7
:10E01000A080B180C280D380B5E1EB2EF12CEC0E54
:10E02000FD1EC7018E010F5F1F4FB8014EE750E183
:10E030000E940272C801B601A50197010E940F6AF1
:10E04000AEE7B0E19401832F982DFC0184E10190AB
:10E050000D928150E1F7A8960FB6F894DEBF0FBE7F
:10E06000CDBFCF91DF911F910F91FF90EF90DF9087
:10E07000CF90BF90AF909F908F9008952F923F9236
:10E080004F925F926F927F928F929F92AF92BF92C8
:10E09000CF92DF92EF92FF920F931F93DF93CF9374
:10E0A000CDB7DEB7AE970FB6F894DEBF0FBECDBFCB
:10E0B0007C017AA769A7A42E409148155091491573
:10E0C0006E010894C11CD11CC601B7010E94967252
:10E0D00000E010E02224332421018A2D992787FDB6
:10E0E00090959CA78BA79C2C8D2C8BA59CA5002E76
:10E0F00002C0959587950A94E2F780FF2CC0892D80
:10E10000982DB8010E94FA713C018EE790E1B801A8
:10E110000E94FA71FC01A080B180C280D380C70147
:10E12000B8010E94F271FC0180819181A281B381CA
:10E130008A0D9B1DAC1DBD1DF30180839183A283BD
:10E14000B383C701B8010E94F271FC01A080B180C5
:10E15000C280D3803CC0892D982DB8010E94FA71ED
:10E160003C01C701B8010E94F271FC01A080B1809E
:10E17000C280D3808091481590914915B8010E94C2
:10E18000FA71FC0180819181A281B3818A0D9B1D6E
:10E19000AC1DBD1DF30180839183A283B383892DC0
:10E1A000982DB8010E94FA71FC01A080B180C28054
:10E1B000D3808EE790E1B8010E94FA71FC01808162
:10E1C0009181A281B381A81AB90ACA0ADB0AD7FED3
:10E1D00008C0D094C094B094A094A11CB11CC11CE0
:10E1E000D11C2A143B044C045D0414F415012601CF
:10E1F0000F5F1F4F0530110509F077CF8E010F5FBC
:10E200001F4FC80162E070E00E94FA71FC0120819A
:10E2100031814281538180913E1090913F10A091B5
:10E220004010B091411082179307A407B50794F4EA
:10E23000C80162E070E00E94FA7120913E103091B6
:10E240003F104091401050914110FC0120833183D8
:10E2500042835383E9A5FAA560817181828193810C
:10E26000A20191010E94D8CCA42EC52E15E1E12E69
:10E27000F12CEC0EFD1EC7018E010F5F1F4FB80180
:10E280004EE750E12DA73EA70E940272C8012DA5BE
:10E29000422F3EA5532F6A2D7C2D97010E940F6AB5
:10E2A000AEE7B0E1F80184E101900D928150E1F711
:10E2B000AE960FB6F894DEBF0FBECDBFCF91DF9103
:10E2C0001F910F91FF90EF90DF90CF90BF90AF9094
:10E2D0009F908F907F906F905F904F903F902F9086
:10E2E0000895CF93DF938FE495E16CE779E140E007
:10E2F0000E94E9C88EE790E10E949B71CAEAD0E1D2
:10E30000CE010E949B71C95BDF4F85E1CA31D807FE
:10E31000B9F78AE195E160E14AEA50E10E94A1691A
:10E3200080E295E10E949B7184E395E10E949B71DC
:10E33000DF91CF91089508958F929F92AF92BF92EF
:10E34000CF92DF92EF92FF920F931F93DF93CF93C1
:10E35000CDB7DEB7FC0140835183628373830483AE
:10E36000158326833783C086D186E286F38684862A
:10E370009586A686B7868F859889A989BA89808B64
:10E38000918BA28BB38BCF91DF911F910F91FF9057
:10E39000EF90DF90CF90BF90AF909F908F900895B7
:10E3A000CF92DF92EF92FF920F931F93FC01408375
:10E3B0005183628373830483158326833783C086E6
:10E3C000D186E286F3861486158616861786108A0D
:10E3D000118A128A138A1F910F91FF90EF90DF909C
:10E3E000CF900895660F771F660F771F680F791F0C
:10E3F000CB010895660F771F660F771F680F791F8F
:10E40000CB0108952F923F924F925F926F927F922D
:10E410008F929F92AF92BF92CF92DF92EF92FF9234
:10E420000F931F93DF93CF9300D000D000D0CDB7D0
:10E43000DEB79E838D83DB0114962D903D904D9029
:10E440005C901797FA010481158126813781201A83
:10E45000310A420A530A18966D907D908D909C90D7
:10E460001B970085118522853385601A710A820AFF
:10E47000930A1C96AD90BD90CD90DC901F970485BB
:10E48000158526853785A01AB10AC20AD30A509687
:10E49000ED90FD900D911C915397DA0150968D915E
:10E4A0009D910D90BC91A02DE81AF90A0A0B1B0B47
:10E4B000FB0180819181A281B381FA0120813181A8
:10E4C00042815381821B930BA40BB50BED81FE811E
:10E4D00080839183A283B3832482358246825782CC
:10E4E0006086718682869386A486B586C686D78620
:10E4F000E08AF18A028B138BCF0126960FB6F8942F
:10E50000DEBF0FBECDBFCF91DF911F910F91FF9066
:10E51000EF90DF90CF90BF90AF909F908F907F90C3
:10E520006F905F904F903F902F9008952F923F9261
:10E530004F925F926F927F928F929F92AF92BF9213
:10E54000CF92DF92EF92FF920F931F93CF93DF93BF
:10E55000FC01DA0114962D903D904D905C90179738
:10E56000EB018C819D81AE81BF81280E391E4A1E30
:10E570005B1EDA0118966D907D908D909C901B9794
:10E5800088859985AA85BB85680E791E8A1E9B1E83
:10E59000EA01AC84BD84CE84DF84EB018C859D854B
:10E5A000AE85BF85A80EB91ECA1EDB1EDA015096C5
:10E5B000ED90FD900D911C91539788899989AA89B6
:10E5C000BB89E80EF91E0A1F1B1FEA018881998189
:10E5D000AA81BB81EB01288139814A815B81820F4D
:10E5E000931FA41FB51F80839183A283B3832482CA
:10E5F0003582468257826086718682869386A4869B
:10E60000B586C686D786E08AF18A028B138BCF0146
:10E61000DF91CF911F910F91FF90EF90DF90CF90FE
:10E62000BF90AF909F908F907F906F905F904F9032
:10E630003F902F900895DF93CF9300D000D0CDB7B7
:10E64000DEB795E099836C83882349F481E08B835E
:10E65000842F80959091591589234A7A09C0813079
:10E6600011F583E08B83842F809590915915892330
:10E67000842B8A8384ECBE016F5F7F4F42E00E944F
:10E68000918885E08A95F1F7000084ECBE016D5F0A
:10E690007F4F42E00E94918885E08A95F1F7000063
:10E6A0008A81809359150F900F900F900F90CF9102
:10E6B000DF910895DF93CF9300D0CDB7DEB795E01B
:10E6C0009983262F209590915915882321F0922324
:10E6D0006575962B01C092239A8384ECBE016F5F0F
:10E6E0007F4F42E00E9491888A81809359150F9054
:10E6F0000F90CF91DF910895DF93CF9300D000D09A
:10E70000CDB7DEB795E099831A821C821B826C8399
:10E71000882349F482E08B83842F8095909159154A
:10E7200089234A7A09C0813019F584E08B83842FCC
:10E730008095909159158923842B8A8384ECBE019E
:10E740006F5F7F4F42E00E94918885E08A95F1F7E4
:10E75000000084ECBE016D5F7F4F42E00E94918813
:10E7600085E08A95F1F700008A818093591507C0EA
:10E7700081E0662309F480E0642F0E945A730F90B1
:10E780000F900F900F90CF91DF91089583E060E09C
:10E790004FE30E947C7308950E94C67381E068EC89
:10E7A00043E00E947C7381E062E843E00E941B73B7
:10E7B0000895CF92DF92EF92FF920F931F93DF9312
:10E7C000CF930F92CDB7DEB7F82E162F042F22234A
:10E7D00021F099830E94C67399812F2D2F3F09F450
:10E7E00093E01F3F09F49C600F3F09F4906383E0BE
:10E7F00061E0492F0E947C739F2D915081E09E3FE4
:10E8000008F080E0282F30E0912F91509E3F10F4C7
:10E810002F5F3F4FE02EEA944E2D4E3F18F42230EA
:10E820003105A1F1882389F080E060915A1543E019
:10E8300099830E941B7380E06F2D43E00E947C73DC
:10E8400081E0C82ED12C998102C0CC24DD249E3FCA
:10E8500078F4FC2C8C2D60915A154CE00E941B73AF
:10E860000894C11CD11C8F2D612F4CE00E947C7339
:10E870008E2D8E3F08F06FC08C2D60915A1540E3AD
:10E880000E941B738C2D602F40E363C0EF2DF0E0DE
:10E89000202F30E0DF01A21BB30BB7FF03C0B09500
:10E8A000A195BF4F812F90E0E81BF90BF7FF03C044
:10E8B000F095E195FF4F281B390B37FF03C03095CA
:10E8C00021953F4FAE17BF07C4F4A217B3076CF5ED
:10E8D00080E060915A154CE00E941B7380E0612F2C
:10E8E0004CE00E947C7381E060915A1543E30E94E2
:10E8F0001B7381E06F2D43E32CC0E217F307ACF4E8
:10E9000080E060915A1540E30E941B7380E0602F05
:10E9100040E30E947C7381E060915A154FE00E94B1
:10E920001B7381E0612F4FE014C080E060915A15A5
:10E9300043E00E941B7380E06F2D43E00E947C73D4
:10E9400081E060915A154CE30E941B7381E0612FB6
:10E950004CE30E947C730F90CF91DF911F910F9138
:10E96000FF90EF90DF90CF900895FF920F931F9349
:10E97000F82E062F142F0E94DE4E8F2D602F412F70
:10E9800021E00E94D9731F910F91FF900895EF929B
:10E99000FF920F931F930E94C67380E491E061E0A1
:10E9A0000E94979C182F84E491E04FEF5FEF6FEF88
:10E9B0007FEF0E94D19C133009F44EC0143028F42C
:10E9C000113011F1123098F50BC0153099F0153057
:10E9D00020F1163009F449C0173009F05FC051C06A
:10E9E00081E060915A154FE30E941B7381E064E659
:10E9F0004FE344C081E060915A1540E30E941B73CD
:10EA000081E064E640E33AC081E060915A1543E05A
:10EA10000E941B7381E064E61DC081E060915A157D
:10EA20004CE00E941B7381E064E64CE027C081E06B
:10EA300060915A154CE00E941B7381E062E34CE048
:10EA40000E947C7380E060915A1543E00E941B7322
:10EA500080E068EC43E012C081E060915A1543E326
:10EA60000E941B7381E066E408C081E060915A1542
:10EA700043E30E941B7381E068EC43E30E947C73D4
:10EA80000DC07C0100271127272F382F492F55272C
:10EA9000892F6E2D422F21E00E94D9731F910F9173
:10EAA000FF90EF90089580935A150E94C7740895BF
:10EAB0000E94D0880E94C77408958BE595E16CE7A9
:10EAC00079E140E00E94E9C808950F9380E397E957
:10EAD00063ED77E940E059E927EC39E900E00E946D
:10EAE000A0959093621580936115009779F480E367
:10EAF00097E963ED77E940E059E927EC39E90FEF51
:10EB00000E94A095909362158093611581E02091F9
:10EB10006115309162152115310509F480E00F91DE
:10EB2000089580916115909162150E94C48E9C0198
:10EB3000909364158093631581E02115310509F4E4
:10EB400080E008950F931F93DF93CF93CDB7DEB787
:10EB5000AB970FB6F894DEBF0FBECDBF80916315A3
:10EB60009091641560EF73E08E010F5F1F4FA80155
:10EB70000E941B948091631590916415B8010E94C6
:10EB800007939C01909366158093651581E021158C
:10EB9000310509F480E0AB960FB6F894DEBF0FBEE6
:10EBA000CDBFCF91DF911F910F9108958F929F92CA
:10EBB000BF92CF92DF92EF92FF920F931F93DF935A
:10EBC000CF93CDB7DEB7AB970FB6F894DEBF0FBECD
:10EBD000CDBF7C014A0185E0B82E6E010894C11CAE
:10EBE000D11C062F10E001501040809165159091C6
:10EBF0006615B6010E944A938823E1F0D701F60119
:10EC000080E090E08017910734F42191222319F0DD
:10EC10002D930196F7CFF701E80FF91F10820097A7
:10EC200031F08114910441F0F401808305C0BA945D
:10EC3000E1F602C0F701108280E090E0AB960FB6DB
:10EC4000F894DEBF0FBECDBFCF91DF911F910F9122
:10EC5000FF90EF90DF90CF90BF909F908F9008959E
:10EC60000F931F93CF93DF938C01EB010EC0CE0166
:10EC7000B8010E94B0CD009741F480916515909144
:10EC800066150E94A69481E009C080916515909157
:10EC90006615BE010E944A93882349F7DF91CF9100
:10ECA0001F910F910895EF92FF920F931F93DF939F
:10ECB000CF93CDB7DEB7AB970FB6F894DEBF0FBEDC
:10ECC000CDBF7B018E010F5F1F4FB8010E943076D0
:10ECD000882361F08091631590916415B8010E94BA
:10ECE0006990F7019183808381E001C080E0AB9659
:10ECF0000FB6F894DEBF0FBECDBFCF91DF911F914D
:10ED00000F91FF90EF9008950F931F93DF93CF9390
:10ED1000CDB7DEB7AB970FB6F894DEBF0FBECDBF51
:10ED20008E010F5F1F4FB8010E943076882349F093
:10ED30008091631590916415B8010E94169581E049
:10ED400001C080E0AB960FB6F894DEBF0FBECDBF1A
:10ED5000CF91DF911F910F910895DF93CF93CDB79E
:10ED6000DEB7AB970FB6F894DEBF0FBECDBFBC01C8
:10ED70008091651590916615AE014F5F5F4F0E94BF
:10ED8000B39491E0882309F490E0892FAB960FB6F5
:10ED9000F894DEBF0FBECDBFCF91DF910895809173
:10EDA0006A150895809169150895CF93DF93EC015A
:10EDB00080916715909168150097E1F0BE016E5F34
:10EDC0007F4F488150E00E94C391288180916B154C
:10EDD00090916C15A0916D15B0916E15820F911DDB
:10EDE000A11DB11D80936B1590936C15A0936D15AB
:10EDF000B0936E15DF91CF9108950E94D29688232B
:10EE000091F080916715909168156FE675E141E08A
:10EE100050E00E94B49021E0181619060CF020E092
:10EE200020937015089581E29BE062EF73E041E06A
:10EE30000E94725C1092701508958091701508956B
:10EE4000DF93CF930F92CDB7DEB780916F15898393
:10EE50000E94FD7689810F90CF91DF9108951092E5
:10EE60006A158091671590916815009721F00E94AE
:10EE7000A1900E941497109268151092671508953A
:10EE800080916A15882311F00E942F77809169156F
:10EE9000882311F00E947177809165159091661515
:10EEA000009731F00E9444931092661510926515F8
:10EEB0008091631590916415009731F00E946390E2
:10EEC00010926415109263158091611590916215EE
:10EED000009731F00E94729610926215109261159F
:10EEE000089580916915882381F08091671590912C
:10EEF0006815009721F00E94A1900E94149710922B
:10EF0000681510926715109269150E9440776091FC
:10EF10006B1570916C1580916D1590916E1508951B
:10EF20000E944398882371F40E94D296882329F482
:10EF30000E94407721E030E029C00E94407722E023
:10EF400030E024C00E946575882329F40E94407730
:10EF500023E030E01BC00E949175882329F40E94B1
:10EF6000407724E030E012C00E94A275882329F483
:10EF70000E94407725E030E009C00E94F496882383
:10EF800019F026E030E002C020E030E0C901089529
:10EF9000CF93DF93EC010E9440770E9490779C0111
:10EFA000009719F086309105D9F410926B151092E4
:10EFB0006C1510926D1510926E15109268151092C6
:10EFC0006715CE0167E675E10E945376882331F01C
:10EFD0008091671590916815009731F427E030E033
:10EFE000C901DF91CF91089581E080936A150E9455
:10EFF000FD7620E030E0F4CFEF92FF920F931F9365
:10F00000CF93DF938C010E9440770E949077EC01B0
:10F01000009769F510926B1510926C1510926D1592
:10F0200010926E151092681510926715C8010E9413
:10F030008476C8010E94AD76882389F0C80167E60E
:10F0400075E10E945376882369F08091671590914D
:10F050006815009751F081E08093691508C0C7E0FA
:10F06000D0E005C0C3E0D0E002C0C8E0D0E0CE01EF
:10F07000DF91CF911F910F91FF90EF9008950E9423
:10F0800040770E9490779C01009719F08630910597
:10F0900041F480916515909166150E94A69420E038
:10F0A00030E0C901089581E795E16CE779E140E03E
:10F0B0000E94E9C80895EF92FF920F931F93DF9388
:10F0C000CF93CDB7DEB76E970FB6F894DEBF0FBE05
:10F0D000CDBF8C01EE24FF24C8018E0D9F1D0E9420
:10F0E000DBC886E090E0E80EF91E9EE1E916F10427
:10F0F00099F7C8014E9666E779E145E00E94E9C8B4
:10F1000085E0F80184A37E010894E11CF11CC7018D
:10F1100060E779E143E00E94E9C8D801F70186E0A1
:10F1200001900D928150E1F737E0E32EF12CEC0EC7
:10F13000FD1EC70160E779E147E00E94E9C8D801F8
:10F140001696F70186E001900D928150E1F72DE0CF
:10F15000E22EF12CEC0EFD1EC70168E779E143E0D9
:10F160000E94E9C8D8011C96F70186E001900D9233
:10F170008150E1F793E1E92EF12CEC0EFD1EC70161
:10F1800066E679E145E00E94E9C8D8015296F701A8
:10F1900086E001900D928150E1F789E1E82EF12C93
:10F1A000EC0EFD1EC70166E779E146E00E94E9C862
:10F1B000D8015896F70186E001900D928150E1F751
:10F1C0006E960FB6F894DEBF0FBECDBFCF91DF9124
:10F1D0001F910F91FF90EF900895FF920F931F934F
:10F1E000CF93DF938C01FF2414C08F2D90E0EC01AE
:10F1F000CC0FDD1FC80FD91FCC0FDD1FC00FD11FD3
:10F20000CE0161E00E941EC9CE0161E00E94F14C76
:10F21000F394F80184A1F81640F3025E1F4FC80171
:10F2200061E00E941EC9C80161E00E94F14CDF91BB
:10F23000CF911F910F91FF9008951F93CF93DF936C
:10F24000EC0185E18A95F1F70000CE014E9661E070
:10F250000E94F14C85E18A95F1F7000010E00FC0A3
:10F26000212F30E0C901880F991F820F931F880F4B
:10F27000991F8C0F9D1F61E00E94F14C1F5F8CA1B4
:10F28000181770F385E18A95F1F70000DF91CF91AF
:10F290001F910895CF92DF92EF92FF920F931F93E9
:10F2A000CF93DF93D62EEA01A8E0EA2EF12CF0E806
:10F2B000CF2E8C01025E1F4F8C2D8D2161E009F451
:10F2C00060E0CE010E94F14CC80161E00E94F14C67
:10F2D00085E18A95F1F70000C80160E00E94F14CD9
:10F2E000C6940894E108F108E114F10429F7CE016D
:10F2F00061E00E94F14CCE0160E00E941EC9C8018D
:10F3000061E00E94F14CCE010E94E24CE82EC8015F
:10F3100060E00E94F14CCE0161E00E941EC981E0D4
:10F32000E11080E0DF91CF911F910F91FF90EF905E
:10F33000DF90CF900895EF92FF920F931F93CF939A
:10F34000DF93EC01F62E8A01EE240FC02E2D30E063
:10F35000C901880F991F820F931F880F991F8C0F67
:10F360009D1F60E00E94F14CE3948CA1E81670F3BD
:10F3700085E18A95F1F70000CE014E9660E00E948B
:10F38000F14CCE016F2DA8010E944A79DF91CF91F7
:10F390001F910F91FF90EF9008958CE995E16CE734
:10F3A00079E140E00E94E9C887E795E10E945B7837
:10F3B00008958091D415882349F48091701688238C
:10F3C00029F40E94FB6691E0982701C091E0892F03
:10F3D0000895DF92EF92FF920F931F93CF93DF93E5
:10F3E000809A819A8A9A829A849A859A8E9A869A23
:10F3F00080910701816080930701809107018260FD
:10F4000080930701809108018460809308018091B6
:10F4100007018460809307010A9A0B9A149A0C9A48
:10F420000E9A0F9AA29A9A9A0DED15E162EEE62EC7
:10F4300065E1F62EC0E0D0E082E090E060E00E945E
:10F44000979CD82E84E090E060E00E94979C4C2F1F
:10F4500087FF0AC0282F30E00C2E02C03595279573
:10F460000A94E2F7217001C021E0F80121938F0195
:10F470008D2D90E002C0959587954A95E2F78170B1
:10F480009070F70181937F012196C530D105A1F6D7
:10F4900080910A018D7F80930A018091DD15882378
:10F4A00021F080910B01826003C080910B018D7F60
:10F4B00080930B0180910A018E7F80930A018091D5
:10F4C000DD15882321F080910B01816003C08091BC
:10F4D0000B018E7F80930B0180910A01877F8093BF
:10F4E0000A018091DE15882321F080910B0188604C
:10F4F00003C080910B01877F80930B0180910A01EB
:10F500008B7F80930A018091DE15882321F0809102
:10F510000B01846003C080910B018B7F80930B01F2
:10F5200080910A018F7780930A018091DF158823EB
:10F5300021F080910B01806803C080910B018F77CF
:10F5400080930B0180910A018F7B80930A01809147
:10F55000DF15882321F080910B01806403C0809126
:10F560000B018F7B80930B01C0E0D0E0CE01880FB0
:10F57000991F9E0143E0220F331F4A95E1F7820F46
:10F58000931F8E559A4E6C2F0E941F9C2196C5305A
:10F59000D10561F7DF91CF911F910F91FF90EF900F
:10F5A000DF90089580E090E041E09C01220F331F3E
:10F5B000220F331FF901E951FA4E10821182128293
:10F5C0001382F901E550FA4E1082118212821382E1
:10F5D000215F394EF9011082118212821382FC01DF
:10F5E000E85DF94E4083019685309105F1F6089566
:10F5F0000E94E97908951092D415109270160E9415
:10F60000E9790E94D27A10926B1610926C161092C1
:10F610006D1610926E161092731610927216EDE21D
:10F62000F6E11082118212821382108611861286F0
:10F63000138614821582168217823C9686E1E13584
:10F64000F80779F71092511610925216109253162D
:10F650001092541610925516109256161092571674
:10F660001092581610925E1610925F161092601645
:10F670001092611681E080935D16109266161092CA
:10F680006716109268161092691610926A16809387
:10F690006F1608951092D4151092701610926B1672
:10F6A00010926C1610926D1610926E1610927316C0
:10F6B0001092721610925116109252161092531602
:10F6C0001092541610925516109256161092571604
:10F6D0001092581610925E1610925F1610926016D5
:10F6E0001092611681E080935D161092661610925A
:10F6F0006716109268161092691610926A1680E0CA
:10F7000090E1909399008093980008950F931F9330
:10F71000CF93DF938C01C0E0D0E0C801BE010E940E
:10F72000F271FC0180819181A281B381FE01EE0F13
:10F73000FF1FEE0FFF1FE951FA4E80839183A283D2
:10F74000B3832196C530D10541F7DF91CF911F9149
:10F750000F9108958F929F92AF92BF92CF92DF92B6
:10F76000EF92FF920F931F93CF93DF93EC014091A1
:10F77000E7155091E8156091E9157091EA1500912F
:10F78000EB151091EC152091ED153091EE15C09010
:10F79000EF15D090F015E090F115F090F2158090F3
:10F7A000F3159090F415A090F515B090F615809192
:10F7B000F7159091F815A091F915B091FA1500D0B0
:10F7C00000D0EDB7FEB781839283A383B483CE01CB
:10F7D0000E949C710F900F900F900F90CE01DF91BF
:10F7E000CF911F910F91FF90EF90DF90CF90BF903E
:10F7F000AF909F908F900895809371160895809197
:10F800006A16833008F04EC080916A1690E0FC01C1
:10F81000EE0FFF1FE80FF91FEE0FFF1FEE0FFF1F88
:10F82000E35DF94E84819581A681B781809351165D
:10F8300090935216A0935316B093541680916A1663
:10F8400090E0FC01EE0FFF1FE80FF91FEE0FFF1F06
:10F85000EE0FFF1FE35DF94E80819181A281B3819C
:10F860008093621690936316A0936416B093651606
:10F8700080916A1690E0FC01EE0FFF1FE80FF91F60
:10F88000EE0FFF1FEE0FFF1FE35DF94E80859185A0
:10F89000A285B3858093591690935A16A0935B1650
:10F8A000B0935C1608958091551690915616A091CC
:10F8B0005716B0915816813020E8920720E0A20731
:10F8C00020E0B2072CF08EE190E0A0E0B0E054C060
:10F8D0008091551690915616A0915716B0915816D2
:10F8E0008030E0E29E07E0E0AE07E0E0BE07CCF04B
:10F8F0008091551690915616A0915716B0915816B2
:10F9000080509042A040B04024E0B595A7959795CF
:10F9100087952A95D1F7895D9E4FFC01849190E0EF
:10F9200029C08091551690915616A0915716B09106
:10F93000581680329105A105B10564F480E290E08B
:10F94000A0E0B0E08093551690935616A0935716FA
:10F95000B09358168091551690915616A09157164F
:10F96000B0915816FC01EE0FFF1FE85DF84F25918E
:10F970003491C901A0E0B0E080935E1690935F16C9
:10F98000A0936016B093611610925D160895DF93F0
:10F99000CF93CDB7DEB7CE01059660E070E00E9450
:10F9A000FA712091E7153091E8154091E9155091D1
:10F9B000EA15FC0180819181A281B381821B930BA6
:10F9C000A40BB50B80930F1690931016A0931116ED
:10F9D000B0931216CE01059661E070E00E94FA71B4
:10F9E0002091EB153091EC154091ED155091EE15ED
:10F9F000FC0180819181A281B381821B930BA40BB6
:10FA0000B50B8093131690931416A0931516B0930C
:10FA10001616CE01059662E070E00E94FA71209100
:10FA2000EF153091F0154091F1155091F215FC0150
:10FA300080819181A281B381821B930BA40BB50BB2
:10FA40008093171690931816A0931916B0931A1650
:10FA5000CE01059663E070E00E94FA712091F315E3
:10FA60003091F4154091F5155091F615FC01808107
:10FA70009181A281B381821B930BA40BB50B809360
:10FA80001B1690931C16A0931D16B0931E16CE0144
:10FA9000059664E070E00E94FA712091F7153091AC
:10FAA000F8154091F9155091FA15FC01808191816A
:10FAB000A281B381821B930BA40BB50B80931F16FD
:10FAC00090932016A0932116B093221680910F16C2
:10FAD00090911016A0911116B09112160097A105E1
:10FAE000B105D9F18A9880910F1690911016A091C6
:10FAF0001116B0911216B7FF1BC080910F1690918E
:10FB00001016A0911116B0911216B095A09590956F
:10FB100081959F4FAF4FBF4F80930F169093101654
:10FB2000A0931116B0931216109223168FEF03C0F4
:10FB300081E080932316809328168091E215882314
:10FB400029F08091231691E0892702C08091231625
:10FB5000882311F0889A01C088988091131690919B
:10FB60001416A0911516B09116160097A105B105AF
:10FB7000D9F18E988091131690911416A0911516B4
:10FB8000B0911616B7FF1BC08091131690911416F2
:10FB9000A0911516B0911616B095A09590958195E7
:10FBA0009F4FAF4FBF4F8093131690931416A0939F
:10FBB0001516B0931616109224168FEF03C081E02D
:10FBC00080932416809329168091E315882329F0C9
:10FBD0008091241691E0892702C080912416882301
:10FBE00011F08C9A01C08C9880911716909118167C
:10FBF000A0911916B0911A160097A105B10509F444
:10FC000045C0809108018B7F809308018091171671
:10FC100090911816A0911916B0911A16B7FF1BC033
:10FC20008091171690911816A0911916B0911A1676
:10FC3000B095A095909581959F4FAF4FBF4F809302
:10FC4000171690931816A0931916B0931A161092BF
:10FC500025168FEF03C081E08093251680932A1626
:10FC60008091E415882329F08091251691E0892759
:10FC700002C080912516882321F0809108018160BF
:10FC800003C0809108018E7F8093080180911B162C
:10FC900090911C16A0911D16B0911E160097A105FB
:10FCA000B105D9F1149880911B1690911C16A09162
:10FCB0001D16B0911E16B7FF1BC080911B169091A8
:10FCC0001C16A0911D16B0911E16B095A09590958A
:10FCD00081959F4FAF4FBF4F80931B1690931C167B
:10FCE000A0931D16B0931E16109226168FEF03C018
:10FCF00081E08093261680932B168091E51588234A
:10FD000029F08091261691E0892702C0809126165D
:10FD1000882311F0129A01C0129880911F169091B9
:10FD20002016A0912116B09122160097A105B105C9
:10FD3000D9F1A29880911F1690912016A0912116BA
:10FD4000B0912216B7FF1BC080911F16909120160C
:10FD5000A0912116B0912216B095A095909581950D
:10FD60009F4FAF4FBF4F80931F1690932016A093C5
:10FD70002116B0932216109227168FEF03C081E050
:10FD80008093271680932C168091E615882329F0FE
:10FD90008091271691E0892702C080912716882339
:10FDA00011F0169A01C01698CF91DF9108950F9324
:10FDB0001F93CF93DF931092D415E0917216F091B8
:10FDC0007316309759F0EA5BFF4F80818E7F8083F6
:10FDD0000E94206710927316109272160E94036799
:10FDE000882339F40E94FB6691E098279093D415FC
:10FDF00011C10E9412679093731680937216FC01D2
:10FE0000EA5BFF4F208121622083FC010489158970
:10FE10002DB73EB7245130400FB6F8943EBF0FBE09
:10FE20002DBFADB7BEB7119684E101900D92815000
:10FE3000E1F70E94C77C10926A1610925516109234
:10FE400056161092571610925816E0917216F091AD
:10FE50007316668977898DB79EB744960FB6F89466
:10FE60009EBF0FBE8DBF6115710591F182AD93AD3F
:10FE7000A4ADB5AD8093551690935616A093571622
:10FE8000B0935816CB01A0E0B0E080933116909368
:10FE90003216A0933316B0933416828D938DA48DB1
:10FEA000B58D80932D1690932E16A0932F16B09398
:10FEB000301686A997A9A0ADB1AD80933516909361
:10FEC0003616A0933716B093381621E030E002C002
:10FED00020E030E0408D518D6417750788F52115BD
:10FEE000310561F486A997A9A0ADB1AD80935516EF
:10FEF00090935616A0935716B0935816E901CC0F5D
:10FF0000DD1FC20FD31FCC0FDD1FCC0FDD1FC35D64
:10FF1000D94ECA01861B970BA0E0B0E08C839D836D
:10FF2000AE83BF83188219821A821B8286A997A981
:10FF3000A0ADB1AD88879987AA87BB872F5F3F4F58
:10FF40008489958948175907E8F52115310561F429
:10FF500082AD93ADA4ADB5AD809355169093561672
:10FF6000A0935716B0935816E901CC0FDD1FC20FAE
:10FF7000D31FCC0FDD1FCC0FDD1FC35DD94E8FEF1C
:10FF80009FE7A0E0B0E08C839D83AE83BF83828D2A
:10FF9000938DA48DB58DB095A095909581959F4F2B
:10FFA000AF4FBF4F88839983AA83BB83DF01DE965F
:10FFB0008D919D910D90BC91A02D88879987AA87DE
:10FFC000BB8715C021503040E901CC0FDD1FC20FA7
:10FFD000D31FCC0FDD1FCC0FDD1FC35DD94E8FEFBC
:10FFE0009FE7A0E0B0E08C839D83AE83BF83EA5B94
:10FFF000FF4F80818F7D808380915516909156169A
:020000021000EC
:10000000A0915716B09158160097A105B10521F49B
:100010001092D41580E08AC00E94FF7B0E94537C1E
:1000200081E090E0A0E0B0E08093661690936716C0
:10003000A0936816B093691610926B1610926C1606
:1000400010926D1610926E1620E030E00093D515D8
:100050001093D6152093D7153093D8158091D515C8
:100060009091D615A091D715B091D8158093D91538
:100070009093DA15A093DB15B093DC158091D5151C
:100080009091D615A091D715B091D815B595A79593
:1000900097958795B095A095909581959F4FAF4F77
:1000A000BF4F8093FB159093FC15A093FD15B09363
:1000B000FE158093FF1590930016A0930116B09340
:1000C00002168093031690930416A0930516B0931E
:1000D00006168093071690930816A0930916B093FE
:1000E0000A1680930B1690930C16A0930D16B093DE
:1000F0000E1681E08093D4158091171690911816F2
:10010000A0911916B0911A16813AEFE09E07E0E02F
:10011000AE07E0E0BE071CF080E098E002C080E09F
:1001200090E1909399008093980081E0DF91CF91C6
:100130001F910F9108950F931F93922F732F0FEF1D
:100140001FEF2FEF3FE70093D9151093DA15209397
:10015000DB153093DC1501E010E020E030E0009387
:10016000D5151093D6152093D7153093D815092F90
:10017000172F9A0100935E1610935F162093601656
:100180003093611620E038E0309399002093980076
:100190002FEF3FEF4FEF5FEF2093FB153093FC15F0
:1001A0004093FD155093FE1510920F1610921016E5
:1001B00010921116109212162093FF15309300160C
:1001C00040930116509302161092131610921416B3
:1001D00010921516109216162093031630930416DB
:1001E0004093051650930616109217161092181683
:1001F0001092191610921A162093071630930816AB
:100200004093091650930A1610921B1610921C1652
:1002100010921D1610921E1620930B1630930C167A
:1002200040930D1650930E1610921F161092201622
:10023000109221161092221660FF28C08093231678
:100240009091E215992329F09091231621E09227AD
:1002500002C090912316992311F0889A01C08898C2
:100260008A9821E030E040E050E020930F16309370
:10027000101640931116509312169091231699233D
:1002800011F091E001C09FEF9093281661FF28C004
:10029000809324169091E315992329F090912416C8
:1002A00021E0922702C090912416992311F08C9A94
:1002B00001C08C988E9821E030E040E050E020931F
:1002C00013163093141640931516509316169091EA
:1002D0002416992311F091E001C09FEF9093291605
:1002E00062FF32C0809325168091E415882329F09F
:1002F0008091251691E0892702C0809125168823D8
:1003000021F080910801816003C0809108018E7FF7
:1003100080930801809108018B7F8093080181E020
:1003200090E0A0E0B0E08093171690931816A09389
:100330001916B0931A1680912516882311F081E0C2
:1003400001C08FEF80932A1680915E1690915F1600
:10035000A0916016B091611680936B1690936C1605
:10036000A0936D16B0936E1681E0809370161F9166
:100370000F9108958230C1F0833028F4882341F032
:10038000813049F50BC08330D9F0843021F51EC08F
:10039000662311F48A9A08958A980895662311F4C1
:1003A0008E9A08958E980895662321F4809108010D
:1003B000846003C0809108018B7F809308010895B9
:1003C000662311F4149A089514980895662311F47D
:1003D000A29A0895A2980895853080F4282F30E0DD
:1003E000C901880F991F43E0220F331F4A95E1F797
:1003F000820F931F8E559A4E0E94259C08958091DE
:10040000D415882319F481E08093D41508956F9250
:100410007F928F929F92AF92BF92CF92DF92EF9294
:10042000FF920F931F938091D415882309F4C9C3B9
:100430008091721690917316009729F40E94D77ECE
:10044000882309F4BBC380916B1690916C16A09120
:100450006D16B0916E1680509140A040B0408093D0
:100460006B1690936C16A0936D16B0936E168091D8
:100470006B1690916C16A0916D16B0916E16B7FF29
:1004800018C320916B1630916C1640916D165091E7
:100490006E1680915E1690915F16A0916016B091D5
:1004A0006116820F931FA41FB51F80936B16909344
:1004B0006C16A0936D16B0936E1631E080916B169A
:1004C00090916C16A0916D16B0916E16B7FF31C069
:1004D0008091D9159091DA15A091DB15B091DC15BA
:1004E000432F552747FD5095652F752F48175907FE
:1004F0006A077B07F4F43F5F40916B1650916C16CE
:1005000060916D1670916E1680915E1690915F16D7
:10051000A0916016B0916116840F951FA61FB71F9A
:1005200080936B1690936C16A0936D16B0936E1615
:10053000C5CF80910F1690911016A0911116B09111
:1005400012160097A105B10571F08091231688233A
:1005500031F08091090141E081FD06C004C0809125
:10056000090141E080FF40E080911316909114163C
:10057000A0911516B09116160097A105B10571F05E
:1005800080912416882331F08091090151E083FD88
:1005900006C004C08091090151E082FF50E08091C3
:1005A000171690911816A0911916B0911A16009767
:1005B000A105B10571F080912516882331F02091B5
:1005C0000901221F2227221F05C08091090121E075
:1005D00086FF20E0A0901B16B0901C16C0901D1640
:1005E000D0901E1660901F167090201680902116D5
:1005F0009090221660E0E32FFF27E7FDF095F9C108
:10060000442309F45FC0E090FB15F090FC150091C5
:10061000FD151091FE1580910F1690911016A09166
:100620001116B09112168E0D9F1DA01FB11F809341
:10063000FB159093FC15A093FD15B093FE158091CA
:10064000FB159091FC15A091FD15B091FE15B7FD1D
:1006500039C0899A8091FB159091FC15A091FD15E8
:10066000B091FE15E090D515F090D6150091D715F4
:100670001091D8158E199F09A00BB10B8093FB1513
:100680009093FC15A093FD15B093FE15E090E7152F
:10069000F090E8150091E9151091EA15809128165F
:1006A000992787FD9095A92FB92F8E0D9F1DA01F0B
:1006B000B11F8093E7159093E815A093E915B093C7
:1006C000EA158998552309F45FC0E090FF15F09072
:1006D0000016009101161091021680911316909148
:1006E0001416A0911516B09116168E0D9F1DA01F01
:1006F000B11F8093FF1590930016A0930116B0933D
:1007000002168091FF1590910016A0910116B091EC
:100710000216B7FD39C08D9A8091FF159091001691
:10072000A0910116B0910216E090D515F090D61563
:100730000091D7151091D8158E199F09A00BB10BF8
:100740008093FF1590930016A0930116B0930216A4
:10075000E090EB15F090EC150091ED151091EE1571
:1007600080912916992787FD9095A92FB92F8E0D75
:100770009F1DA01FB11F8093EB159093EC15A093C4
:10078000ED15B093EE158D98222309F467C0E09023
:100790000316F0900416009105161091061680912C
:1007A000171690911816A0911916B0911A168E0D61
:1007B0009F1DA01FB11F8093031690930416A09352
:1007C0000516B09306168091031690910416A09119
:1007D0000516B0910616B7FD41C0809108018260F0
:1007E000809308018091031690910416A09105163C
:1007F000B0910616E090D515F090D6150091D7155A
:100800001091D8158E199F09A00BB10B8093031678
:1008100090930416A0930516B0930616E090EF157A
:10082000F090F0150091F1151091F21580912A16B3
:10083000992787FD9095A92FB92F8E0D9F1DA01F79
:10084000B11F8093EF159093F015A093F115B0931D
:10085000F215809108018D7F80930801A114B104E5
:10086000C104D10409F45FC0E0900716F0900816A7
:100870000091091610910A1680911B1690911C1672
:10088000A0911D16B0911E168E0D9F1DA01FB11FA9
:100890008093071690930816A0930916B0930A1632
:1008A0008091071690910816A0910916B0910A162A
:1008B000B7FD39C0139A8091071690910816A09140
:1008C0000916B0910A16E090D515F090D615009152
:1008D000D7151091D8158E199F09A00BB10B8093D5
:1008E000071690930816A0930916B0930A16E09085
:1008F000F315F090F4150091F5151091F61580910F
:100900002B16992787FD9095A92FB92F8E0D9F1D26
:10091000A01FB11F8093F3159093F415A093F515C4
:10092000B093F6151398611471048104910409F4CD
:100930005FC0E0900B16F0900C1600910D16109110
:100940000E1680911F1690912016A0912116B0913D
:1009500022168E0D9F1DA01FB11F80930B16909322
:100960000C16A0930D16B0930E1680910B16909155
:100970000C16A0910D16B0910E16B7FD39C0179A3E
:1009800080910B1690910C16A0910D16B0910E1639
:10099000E090D515F090D6150091D7151091D81587
:1009A0008E199F09A00BB10B80930B1690930C1618
:1009B000A0930D16B0930E16E090F715F090F81571
:1009C0000091F9151091FA1580912C16992787FD41
:1009D0009095A92FB92F8E0D9F1DA01FB11F809339
:1009E000F7159093F815A093F915B093FA15179889
:1009F0006F5F862F90E08E179F070CF401CE8091D9
:100A0000D9159091DA15A091DB15B091DC15E32E84
:100A1000FF24E7FCF0940F2D1F2D8E199F09A00BCA
:100A2000B10B8093D9159093DA15A093DB15B09391
:100A3000DC158091D9159091DA15A091DB15B09154
:100A4000DC15181619061A061B062CF00E94D77E14
:100A5000882309F4B3C08091511690915216A09149
:100A60005316B09154168E199F09A00BB10B8093A9
:100A7000511690935216A0935316B093541680912A
:100A8000511690915216A0915316B0915416181603
:100A900019061A061B063CF080916A168F5F809338
:100AA0006A160E94FF7B80915D16882311F00E94D8
:100AB000537C8091621690916316A0916416B09158
:100AC00065160097A105B10509F478C02091551667
:100AD00030915616409157165091581680916216D3
:100AE00090916316A0916416B0916516820F931FC2
:100AF000A41FB51F8093551690935616A0935716B2
:100B0000B093581681E080935D16809162169091A3
:100B10006316A0916416B0916516181619061A0688
:100B20001B06ACF42091551630915616409157167D
:100B3000509158168091591690915A16A0915B16B3
:100B4000B0915C1682179307A407B507FCF080915B
:100B5000621690916316A0916416B0916516B7FF66
:100B60002DC0209155163091561640915716509130
:100B700058168091591690915A16A0915B16B09113
:100B80005C16281739074A075B07C4F410926216EF
:100B90001092631610926416109265168091591681
:100BA00090915A16A0915B16B0915C1680935516E1
:100BB00090935616A0935716B09358168091D4155B
:100BC00025C280917016882309F41FC280916B168C
:100BD00090916C16A0916D16B0916E168058904051
:100BE000A040B04080936B1690936C16A0936D1646
:100BF000B0936E1680916B1690916C16A0916D1645
:100C0000B0916E16181619061A061B060CF4F4C1DC
:100C10001092701641E01DC04F5F00916B1610914D
:100C20006C1620916D1630916E1680915E16909123
:100C30005F16A0916016B0916116800F911FA21FE0
:100C4000B31F80936B1690936C16A0936D16B093A0
:100C50006E1600916B1610916C1620916D163091E6
:100C60006E1680915E1690915F16A0916016B091FD
:100C70006116B095A095909581959F4FAF4FBF4F4E
:100C800080179107A207B3073CF630E021E080917E
:100C90000F1690911016A0911116B0911216009790
:100CA000A105B10509F476C0E090FB15F090FC15A4
:100CB0000091FD151091FE1580910F169091101660
:100CC000A0911116B09112168E0D9F1DA01FB11F7D
:100CD0008093FB159093FC15A093FD15B093FE1522
:100CE0008091FB159091FC15A091FD15B091FE151A
:100CF000B7FD50C08091FB159091FC15A091FD159A
:100D0000B091FE15E090D515F090D6150091D7154D
:100D10001091D8158E199F09A00BB10B8093FB156C
:100D20009093FC15A093FD15B093FE1580912316AA
:100D3000882329F08091090181FF28C005C0809196
:100D400009018170821711F5899A8091701620939C
:100D50007016E090E715F090E8150091E9151091F4
:100D6000EA1580912816992787FD9095A92FB92F0C
:100D70008E0D9F1DA01FB11F8093E7159093E8155E
:100D8000A093E915B093EA15899804C08091701674
:100D9000809370168091131690911416A0911516D9
:100DA000B09116160097A105B10509F475C0E09041
:100DB000FF15F09000160091011610910216809117
:100DC000131690911416A0911516B09116168E0D4B
:100DD0009F1DA01FB11F8093FF1590930016A09335
:100DE0000116B09302168091FF1590910016A09104
:100DF0000116B0910216B7FD4FC08091FF1590917A
:100E00000016A0910116B0910216E090D515F09051
:100E1000D6150091D7151091D8158E199F09A00BE2
:100E2000B10B8093FF1590930016A0930116B09319
:100E3000021680912416882329F08091090183FFEE
:100E400027C004C08091090182FF22C08D9A809141
:100E5000701620937016E090EB15F090EC15009151
:100E6000ED151091EE1580912916992787FD909523
:100E7000A92FB92F8E0D9F1DA01FB11F8093EB15B9
:100E80009093EC15A093ED15B093EE158D9804C0DA
:100E90008091701680937016809117169091181695
:100EA000A0911916B0911A160097A105B10509F481
:100EB0007DC0E0900316F090041600910516109185
:100EC00006168091171690911816A0911916B091D8
:100ED0001A168E0D9F1DA01FB11F809303169093AD
:100EE0000416A0930516B0930616809103169091F0
:100EF0000416A0910516B0910616B7FD57C0809153
:100F0000031690910416A0910516B0910616E09074
:100F1000D515F090D6150091D7151091D8158E19CA
:100F20009F09A00BB10B8093031690930416A09316
:100F30000516B093061680912516882329F0809116
:100F4000090187FF2FC004C08091090186FF2AC0D4
:100F5000809108018260809308018091701620932F
:100F60007016E090EF15F090F0150091F1151091CA
:100F7000F21580912A16992787FD9095A92FB92FF0
:100F80008E0D9F1DA01FB11F8093EF159093F0153C
:100F9000A093F115B093F215809108018D7F809395
:100FA000080104C080917016809370163F5F34175B
:100FB0000CF46DCE80917016882311F40E94D767CF
:100FC00020916B1630916C1640916D1650916E16F3
:100FD00080915E1690915F16A0916016B091611697
:100FE000820F931FA41FB51F80936B1690936C16EE
:100FF000A0936D16B0936E1680917016882311F42D
:101000000E94D7678091701601C080E01F910F91F8
:10101000FF90EF90DF90CF90BF90AF909F908F9018
:101020007F906F900895AF92BF92CF92DF92EF9230
:10103000FF920F931F93DF93CF93CDB7DEB76E97D9
:101040000FB6F894DEBF0FBECDBF84E796E16CE724
:1010500079E140E00E94E9C88E01075E1F4FE0E79A
:10106000AE2EE9E1BE2EC801B50143E00E94E9C8F9
:1010700072EAE72E75E1F72E6EECC62E65E0D62EED
:10108000C701B801A6010E94A99B8E010D5E1F4FEA
:10109000C801B50147E00E94E9C8C7010A96B80136
:1010A000A6010E94A99B8E01035F1F4FC80168E73C
:1010B00079E143E00E94E9C8C7014496B801A6015E
:1010C0000E94A99B8E01095F1F4FC80166E679E166
:1010D00045E00E94E9C8C7014E96B801A6010E94EA
:1010E000A99B8E010F5F1F4FC80166E779E146E0BB
:1010F0000E94E9C8C7018896B801A6010E94A99B71
:101100006E960FB6F894DEBF0FBECDBFCF91DF91C4
:101110001F910F91FF90EF90DF90CF90BF90AF9015
:10112000089594EA9093BC009091BC0097FFFCCF87
:101130009091B900987F983069F58093BB0084E85E
:101140008093BC008091BC0087FFFCCF8091B900E8
:10115000887F883109F5862F972FFC0180E090E089
:1011600050E034E80FC021912093BB003093BC00C5
:101170002091BC0027FFFCCF2091B900287F2832A6
:1011800069F401968417950774F384E98093BC0091
:1011900080E0089581E0089582E0089583E0089555
:1011A0001092B90080E28093B800089580917A1679
:1011B000089510927A16089581E040917B1650911F
:1011C0007C1620917D1630917E16421753070CF045
:1011D00080E0089580917B1690917C1620917D1679
:1011E00030917E16821793076CF4E0917F16F09190
:1011F0008016E80FF91F019690937C1680937B165A
:101200008491089580E0089520917F163091801692
:1012100080917B1690917C1640E0682F592FF90140
:10122000E80FF91FE4910196E539B9F7862F952F5C
:1012300001964F5F453089F760937B1650937C167B
:1012400008951F93182F81E080937A1610927C16D0
:1012500010927B161130D9F0113028F0123009F1BC
:101260001330A1F503C028E237E41DC00E94944F5B
:10127000882319F083E797E402C08BE99DE49093FB
:10128000801680937F160E94048911E010C00E948E
:10129000944F882319F023E737E405C02BE93DE498
:1012A00002C023EC33E53093801620937F16E12FA4
:1012B000F0E0EE0FFF1FE752FA4925913491209399
:1012C0007D1630937E1680917A1601C080E01F91C2
:1012D000089510927A16089581E896E16CE779E115
:1012E00040E00E94E9C80895DF93CF9300D0CDB7C6
:1012F000DEB7FC01009769F16230710550F1A08101
:10130000B181660F771F80E090E0268137814085AC
:101310005185620F731F841F951FED91FC91AE01E3
:101320004F5F5F4F22E030E00995882391F02981DB
:101330003A812115310579F08FEF273F380749F0C1
:10134000C90140968730910520F08FEF283F38077C
:1013500010F020E030E0C9010F900F90CF91DF91A5
:1013600008954F925F926F927F928F929F92AF9269
:10137000BF92CF92DF92EF92FF920F931F93DF9372
:10138000CF9300D0CDB7DEB75C018B01009709F495
:1013900049C06230710508F445C0DC0116964D90D5
:1013A0005D906D907C9019974E010894811C911C62
:1013B000000F111F6801EE24FF24C40CD51CE61C8D
:1013C000F71CD501ED91FC910190F081E02DC70152
:1013D000B601A40122E030E00995882319F10981C2
:1013E0001A8101151105E1F0C80140968830910578
:1013F000C8F0BFEF083F1B0710F000E010E01A82B2
:101400001982D501ED91FC910480F581E02DC70191
:10141000B601A40122E030E009950115110541F65D
:1014200081E001C080E00F900F90CF91DF911F917C
:101430000F91FF90EF90DF90CF90BF90AF909F9073
:101440008F907F906F905F904F9008952F923F9272
:101450004F925F926F927F928F929F92AF92BF92C4
:10146000CF92DF92EF92FF920F931F93DF93CF9370
:10147000CDB7DEB72E970FB6F894DEBF0FBECDBF47
:101480006C017A876987009709F4A4C0DC01ED91AB
:10149000FC911197208131813C872B878481958134
:1014A0009C838B8316968D919D910D90BC91A02D60
:1014B0008D839E83AF83B887F601028D138D42849E
:1014C00053846484758476946794579447945E86B5
:1014D0004D86138E128E642E752EEE24FF241E016F
:1014E0000894211C311C4CC00230110528F02D85B8
:1014F0003E850217130710F002E010E04801880C47
:10150000991CAA24BB248D819E81AF81B885880E49
:10151000991EAA1EBB1EC501B401A10122E030E044
:10152000AB85BC85FD010995882309F453C08981E9
:101530009A81009701F56114710421F4F601138F6B
:10154000028F25C0E114F10429F42FEF3FEF3A8315
:10155000298302C0FA82E982C501B401A10122E017
:1015600030E0AB81BC81FD010995882379F10894B5
:101570006108710878010894410851080F5F1F4FF6
:101580004114510409F0B0CF61147104F9F4E985F4
:10159000FA85E230F10500F1FA82E982BF01660FB7
:1015A000771F80E090E02D813E814F815885620F4A
:1015B000731F841F951FAE014F5F5F4F22E030E025
:1015C000AB81BC81FD010995882331F4C601B701C7
:1015D0000E94B189EE24FF24C7012E960FB6F8941D
:1015E000DEBF0FBECDBFCF91DF911F910F91FF9056
:1015F000EF90DF90CF90BF90AF909F908F907F90B3
:101600006F905F904F903F902F90089580E190E011
:101610000895CF93DF93EC010097C1F0623071051C
:10162000A8F06250704080E090E02889398940E05D
:1016300050E00E9470CC9B01AC018A899B89AC89E7
:10164000BD89280F391F4A1F5B1F03C020E030E00F
:10165000A901B901CA01DF91CF910895FC018191DF
:101660004AE0282F30E05191C9019695982F88279C
:101670009795879535952795822B850F415089F74A
:101680000895EF92FF920F931F93DF93CF93CDB7FF
:10169000DEB760970FB6F894DEBF0FBECDBF8C01EA
:1016A00062307105D8F00E94098BAE014F5F5F4F29
:1016B00020E1DA011D922A95E9F7D801ED91FC911C
:1016C000119750962D913C9151970680F781E02D0E
:1016D00006E01BE8EE24FF24099501C080E0609637
:1016E0000FB6F894DEBF0FBECDBFCF91DF911F9133
:1016F0000F91FF90EF9008958F929F92AF92BF92BB
:10170000CF92DF92EF92FF920F931F93DF93CF93CD
:10171000CDB7DEB72D970FB6F894DEBF0FBECDBFA5
:101720008C014A015B016901D901ED90FC90119790
:1017300012968D919C911397809613969C938E93FD
:101740001297F8018081853E11F0882329F4D60193
:1017500014961C921497D0C0F80183858F3009F03D
:101760004AC0D90114968C911497882319F0958555
:10177000891779F08BE2D7011D928A95E9F7F80174
:101780008585D60114968C93F70187A290A6A1A611
:10179000B2A6D8012C9130E02F7330702150304028
:1017A0004DE050E0249FC001259F900D349F900D87
:1017B0001124DE011196E0EDF5E02DE001900D928F
:1017C0002150E1F7DE011196E80EF91E9C01235F1E
:1017D0003F4F8F31910508F08FC04D91F801E40F14
:1017E000F11D4081F70141937F0101968217930714
:1017F00009F482C0EECFD7018C91882341F0C80153
:101800000E942E8BF6019481981709F458C08BE240
:10181000D7011D928A95E9F7F70187A290A6A1A6A4
:10182000B2A6B801D701C80140E0FC015191CF0137
:101830005032A1F05C93F801248523FF0BC09C017A
:1018400021503040F9012081213420F02B3510F453
:10185000505E5C934F5F1196483039F7D7018C91F9
:10186000853011F485EE8C93F8018085803219F172
:10187000D701A40FB11D8EE28C93242F2C5F4F5FF4
:10188000DB0118968C9118978032A9F0D701A40F2C
:10189000B11D8C93F801948594FF08C0FB019085DD
:1018A000913420F09B3510F4805E8C934F5F6F5F16
:1018B0007F4F421729F7F701E40FF11D1082D8017D
:1018C0001B968C911B97F70180A35A968D919C9142
:1018D0005B9792A381A35C968D919D910D90BC9195
:1018E000A02D83A394A3A5A3B6A381E0D60115964A
:1018F0008C93159780E001C081E02D960FB6F89487
:10190000DEBF0FBECDBFCF91DF911F910F91FF9032
:10191000EF90DF90CF90BF90AF909F908F90089501
:101920002F923F924F925F926F927F928F929F92EF
:10193000AF92BF92CF92DF92EF92FF920F931F93DD
:10194000DF93CF93CDB7DEB7A0970FB6F894DEBF85
:101950000FBECDBF8B01009709F418C16115710549
:1019600009F414C1DC01ED91FC9124803580FB0168
:1019700087A090A4A1A4B2A46B01DB010D9000206C
:10198000E9F71197FA2EF61A8F2D90E00C966DE07C
:1019900070E00E94A3CCE62ECE01019660E270E0DA
:1019A0004BE050E00E949ECDC8016EE270E00E94C4
:1019B000DDCD0097F9F09C012F5F3F4FDC011196C0
:1019C0008C9111978823B1F0F90101900020E9F77B
:1019D0003197E21BF30B8E2F8095F80EBE01675FE7
:1019E0007F4F4E2FE43008F043E0CB01B90150E0C7
:1019F0000E9495CDCE010196BF2DB93080F4B6017D
:101A00004F2D50E00E9495CDF80180818E3281F5F6
:101A100081818E3209F48281882349F129C0FC0139
:101A20008C2D9D2DDC0188E00D9001928150E1F715
:101A3000D80191962C919197822F90E0203A38F41A
:101A400044E0959587954A95E1F7805D06C034E0BE
:101A5000959587953A95E1F78F598F83822F8F70EF
:101A60008A3010F4805D01C08F59888701C0EE2450
:101A70008981853E11F485E0898385E1FE013C96EC
:101A8000DF011D928A95E9F7F80180A18C8781A179
:101A900092A19C8F8B8F83A194A1A5A1B6A18D8FBC
:101AA0009E8FAF8FB8A36E2D70E095E0660F771F05
:101AB0009A95E1F780E090E0680D791D8A1D9B1DE5
:101AC0006E010894C11CD11CA60120E230E0F10196
:101AD0000995882309F45AC0C6010E942E8B482E0E
:101AE000FE2C8DE0682E712CBFE05B2E4AC0C60133
:101AF0006FEF70E040E250E00E949ECD8F2D90E0AD
:101B00000197869DF001879DF00D969DF00D1124A3
:101B1000E00FF11F21E0CF01D601A20FB11D3081EE
:101B20003C932F5FD601A20FB11D1C922F5F2B306B
:101B300019F02A3121F402C02EE001C02CE13196C7
:101B4000DC018C91882311F02F3128F3F982FE14E7
:101B500019F48F2D806489835C864E861D861B8ECA
:101B60001C8EC501B401A60120E230E0F101099507
:101B700080E290E0A0E0B0E0880E991EAA1EBB1E95
:101B8000FA94FF2009F0B3CF81E001C080E0A09675
:101B90000FB6F894DEBF0FBECDBFCF91DF911F917E
:101BA0000F91FF90EF90DF90CF90BF90AF909F90FC
:101BB0008F907F906F905F904F903F902F900895FF
:101BC0002F923F924F925F926F927F928F929F924D
:101BD000AF92BF92CF92DF92EF92FF920F931F933B
:101BE000DF93CF9300D00F92CDB7DEB74C019B01AE
:101BF000009709F4AEC04115510509F4AAC0FA01D5
:101C000001900020E9F7CF01841B950B0B966DE046
